:100000000C94AD080C94DE080C94DE080C94DE0809
:100010000C94DE080C94DE080C94DE080C94DE08C8
:100020000C94DE080C94DE080C94DE080C94DE08B8
:100030000C94DE080C94F68C0C94DE080C94DE080C
:100040000C94DE080C94DE080C94DE080C94DE0898
:100050000C94DE080C94DE080C94DE080C948B9350
:100060000C94DE080C946F5B0C94465B0C94DE08D9
:100070000C94DE080C94DE080C94DE080C94DE0868
:100080000C94DE080C94DE080C94DE080C94DE0858
:100090000C941C5B0C94F35A0C94DE080C94098E9F
:1000A0000C94DE080C94DE080C94DE080C94DE0838
:1000B0000C94DE080C94DE080C94DE080C94DE0828
:1000C0000C94DE080C94DE080C94DE080C94C95ADB
:1000D0000C94A05A0C94DE080C94765A0C944D5A49
:1000E0000C94DE085E36573639362337F536F5364A
:1000F000F536F536F536F536F53602256B25CE257F
:100100000B271327E5289F29BD2A5F2C5B2D932DF4
:10011000A82DAC2DF536EE2DFA2D662F21313B3171
:100120006232C1329D331D3424341035F536F53634
:10013000F536F536F536F536F536F536F536F53667
:100140004F35F536F536F536F536F536F5362337CF
:10015000E287C588688986899B89B089C589E389D2
:10016000F8890D8A2B8A408A558A788A17921A92C2
:1001700009920D92139251921E92229228922C92E1
:10018000309236923A923E925192449248924C92D8
:10019000084AD73B3BCE016E84BCBFFDC12F3D6CEE
:1001A00074319ABD56833DDA3D00C77F11BED9E454
:1001B000BB4C3E916BAAAABE000000803F07634281
:1001C00036B79BD8A71A39685618AEBAAB558C1DEE
:1001D0003CB7CC5763BD6DEDFD753EF6177231BF70
:1001E000000000803F08000000BE922449123EAB90
:1001F000AAAA2ABECDCCCC4C3E00000080BEABAA41
:10020000AAAA3E00000000BF000000803F000000DE
:100210000000084178D3BB4387D1133D190E3CC37E
:10022000BD4282AD2B3E68EC8276BED98FE1A93EFD
:100230004C80EFFFBE01C4FF7F3F000000000000C4
:100240004E414E494E495459494E46CDCCCC3D0ABB
:10025000D7233C17B7D13877CC2B329595E6241F9E
:10026000B14F0A000020410000C84200401C462057
:10027000BCBE4CCA1B0E5AAEC59D7400407A10F32A
:100280005A00A0724E18090010A5D4E80000E876C4
:1002900048170000E40B54020000CA9A3B0000001B
:1002A000E1F505000080969800000040420F000034
:1002B00000A08601000000102700000000E80300F5
:1002C0000000006400000000000A000000000001BF
:1002D00000000000002C76D888DC674F0823DFC1BF
:1002E000DFAE59E1B1B796E5E3E453C63AE651997A
:1002F0007696E8E6C28426EB898C9B62ED407C6FA3
:10030000FCEFBC9C9F40F2BAA56FA5F490055A2A59
:10031000F75C936B6CF9676DC11BFCE0E40D47FE65
:10032000F520E6B500D0ED902E030094357705005A
:1003300080841E080000204E0A000000C80C3333E1
:1003400033330F986E12831141EF8D2114893BE6F0
:100350005516CFFEE6DB18D1844B381BF77C1D9079
:100360001DA4BBE424203284725E228100C9F124E2
:10037000ECA1E53D27696E707574204453546361A8
:100380006C6962726174653A0020766F6C746167A3
:10039000653D0023547572626964697479205570F3
:1003A000706572204C696D69743A200020766F6C1C
:1003B000746167653D00235475726269646974797C
:1003C000204C6F776572204C696D69743A20002368
:1003D000547572626964697479204C6F7765722014
:1003E0004C696D69742056696E663A200023566F19
:1003F0006C746167652073656E736F723A00234396
:10040000757272656E742073656E736F723A002335
:100410004F322063616C6962726174696F6E3A2059
:100420000023547572626964697479204C6F776532
:1004300072204C696D69742056313A200057694624
:10044000692049503A00234D5320456E61626C6526
:100450006400234D532044697361626C656400231A
:100460005265737420706172616D6574657273207A
:10047000746F2064656661756C742076616C756557
:1004800073002343757272656E742073656E736FAB
:10049000723A004D6F74696F6E00555620496E7444
:1004A0002E00555620496E74656E73697479004F3D
:1004B0003220436F6E6300434F3220436F6E630000
:1004C00053656E736F72206572726F722100234ED6
:1004D0006F2073656E736F722100434F3220436F3C
:1004E0006E63004D6561737572696E6700234E6FB0
:1004F0002073656E736F7220666F7220504D2100FD
:100500004E6F2073656E736F722100206E672F4CE3
:1005100000504D313A322E353A3130004D6561731D
:100520007572696E672E2E00234E6F205442207321
:10053000656E736F723F00234E6F2073656E736F2D
:10054000722100536F756E64204C6576656C004DAA
:100550006561737572696E672E2E00234E6F20736E
:10056000656E736F722100536F756E64204C6576F3
:10057000656C00234E6F2073656E736F7220666F1B
:10058000722074656D7020262068756D69646974C9
:100590007921004E6F2053656E736F7221002066C3
:1005A0006F722074656D7020262068756D696469AE
:1005B000747921002353656E736F72204572726FD8
:1005C00072200053656E736F72204572726F7221D4
:1005D000002357726F6E672073656E736F722066AB
:1005E0006F722074656D7020262068756D6964696E
:1005F0007479210057726F6E672053656E736F7246
:10060000210054656D702048756D696469747900C6
:100610004C6967687420496E74656E7369747900FB
:10062000466C616D6520495200482D6669656C64B1
:100630000053656172636820446972656374696F11
:100640006E00234E6F2070482073656E736F7221A9
:100650000070482076616C756500496E76616C6942
:1006600064206B65792100204D756C746973656E2B
:10067000736F7273004D756C746973656E736F720E
:10068000730044697361626C6500456E61626C65FC
:1006900000237265706C6965733D00235365747443
:1006A000696E6773206F6620616C6C2073656E7372
:1006B0006F72733A0043616C6962726174696F6E44
:1006C0002050726573737572653D00536561206CCF
:1006D0006576656C20502863616C63293D00234575
:1006E00072726F723A707265737375726520424DE3
:1006F000503038352C20636865636B2077697269E8
:100700006E67210049522054656D702073656E73C9
:100710006F7220666F756E6400504D322E352073F7
:10072000656E736F72206C696B656C7920666F758E
:100730006E6400576946692049503A00456455483F
:100740004B205345534C6F676765720053656E735A
:100750006F7220736C6F7420616E642074797065A1
:100760003A0057656C636F6D6520746F2045645562
:10077000484B0067657453656C66546573744269D1
:100780007428293A20006973496E74657272757015
:1007900074456E61626C65642831293A2000676592
:1007A00074496E746572727570744D617070696EA3
:1007B000672831293A2000676574496E7465727242
:1007C000757074536F757263652831293A2000671C
:1007D0006574496E74657272757074536F75726367
:1007E0006528293A20006765745261746528293AA2
:1007F00020332E31343135393F00616363656C2E0F
:1008000069734C6F77506F77657228293A200061C1
:100810006363656C2E697341736C65657028293A52
:100820002000616363656C2E6973546170536F754A
:100830007263654F6E5A28293A2000616363656CC4
:100840002E6973546170536F757263654F6E5928CA
:10085000293A2000616363656C2E6973546170539B
:100860006F757263654F6E5828293A200061636383
:10087000656C2E69734163746976697479536F7519
:100880007263654F6E5A28293A2000616363656C74
:100890002E69734163746976697479536F757263F5
:1008A000654F6E5928293A2000697341637469764F
:1008B000697479536F757263654F6E5828293A20B1
:1008C000006973546170446574656374696F6E4F39
:1008D0006E5A28293B2066616C73653F200069735E
:1008E000546170446574656374696F6E4F6E5A2805
:1008F000293B20747275653F200069735461704410
:100900006574656374696F6E4F6E5928293B206664
:10091000616C73653F200069735461704465746550
:100920006374696F6E4F6E5928293B207472756528
:100930003F20006973546170446574656374696F26
:100940006E4F6E5828293B2066616C73653F20000E
:100950006973546170446574656374696F6E4F6E3A
:100960005828293B20747275653F200067657453D1
:100970007570707265737342697428293B206661D3
:100980006C73653F20006765745375707072657392
:100990007342697428293B20747275653F20006991
:1009A000734163746976697479416328293A200038
:1009B0006973496E61637469766974795A456E61C9
:1009C000626C656428293A20006973496E6163741A
:1009D000697669747959456E61626C656428293A53
:1009E00020006973496E616374697669747958454A
:1009F0006E61626C656428293A20006973416374F2
:100A000069766974795A456E61626C656428293A21
:100A100020006973416374697669747959456E6120
:100A2000626C656428293A200069734163746976B1
:100A300069747958456E61626C656428293A2000B2
:100A40006765744672656546616C6C447572617465
:100A5000696F6E28293A200067657446726565469D
:100A6000616C6C5468726573686F6C6428293A20F5
:100A70000067657454696D65496E61637469766970
:100A8000747928293A2000676574496E6163746936
:100A9000766974795468726573686F6C642829206C
:100AA0000067657441637469766974795468726526
:100AB00073686F6C6428292000676574446F7562E1
:100AC0006C6554617057696E646F772829200067E0
:100AD0006574446F75626C655461704C6174656EC9
:100AE000637928293A2000676574546170447572EF
:100AF0006174696F6E28293A2000676574417869CE
:100B0000734F66667365742826782C2026792C200E
:100B1000267A293A200067657454617054687265BA
:100B200073686F6C6428293A200058595A2047731B
:100B30003A200058595A20434F554E54533A2000FA
:100B4000736574206761696E735B5D3A0067616904
:100B50006E735F6F7269675B5D3A004E6F2053651D
:100B60006E736F7221004E6F20445320546865727B
:100B70006D6F6D6574657221004453205468657211
:100B80006D2E004D6F74696F6E0046696E64696EFC
:100B900067205769466920495000005EBCE2613F0A
:100BA000DD83C29C7E20A3FD1F41009D23BE46DB4A
:100BB00065F88C11AF32CA57E97469746572617453
:100BC000696F6E3D0073656E736F72233D004375F0
:100BD0007272656E74207374617475733A206379F0
:100BE000636C653D006E6379636C653D006E736593
:100BF0006E736F72733D006D61786E73656E736FA7
:100C000072733D00656E61626C65643D00234D75D5
:100C10006C746973656E736F7273206D6561737543
:100C200072656D656E742073657474696E67733A6E
:100C3000007365703D006976616C3D006E69746596
:100C4000723D00230023616E6F7468657220495203
:100C500020696E7075743D0023456E64206F6620B8
:100C60004D756C746973656E736F72204379636C34
:100C7000652300236B65793D00416E676C65732FBA
:100C8000003E6128782C792C7A292F673A004E6F24
:100C90002073656E736F72210049522054656D7028
:100CA00065726174757265004D6561737572696E08
:100CB000672E2E004E6F2073656E736F723F004972
:100CC000522054656D7065726174757265004D6572
:100CD00061737572696E672E2E00202020202020FF
:100CE0002020202020202020202000202020202024
:100CF0002020202020202020202020004F66662059
:100D00006169722D636F6E642100497427732074CA
:100D10006F6F20636F6F6C210054656D7020697375
:100D20002066696E6521004973206169722D636FC9
:100D30006E64206F6E3F004974277320717569746B
:100D40006520686F74210049742773207665727975
:100D500020686F742120004F6666206169722D63E0
:100D60006F6E6421004974277320746F6F20636F66
:100D70006F6C210054656D702069732066696E6523
:100D800021004973206169722D636F6E64206F6E5C
:100D90003F004974277320717569746520686F740A
:100DA000210049742773207665727920686F742159
:100DB0000054656D702048756D696469747900230D
:100DC0002D2D2D2D2D2D2D2D2D2D2D2D2D2D2D2D53
:100DD0002D2D2D2D2D2D2D2D2D2D2D2D2D2D2D2D43
:100DE0002D2D2D2D00235265736F6C7574696F6EF8
:100DF0003A20202000234D696E2056616C75653ABB
:100E00002020202000234D61782056616C75653AC2
:100E1000202020200023556E697175652049443AD1
:100E20002020202000234472697665722056657266
:100E30003A202020002353656E736F723A202020E1
:100E40002020202000232D2D2D2D204D61676E6543
:100E50007469632053656E736F72202D2D2D2D2DB7
:100E60002D2D2D2D2D2D2D2D2D2D2D2D2D2D2D00DF
:100E7000482D6669656C643A2028002020202020D7
:100E80002020202020202020202020002020202082
:100E90002020202020202020202020200020202072
:100EA0002020202020202020202020200020202062
:100EB0002020202020202020202020200044303A04
:100EC000566F6C746167650044393A437572726598
:100ED0006E7400566F6C746167652B437572726532
:100EE0006E740044383A456C6563747269630044FB
:100EF000373A4D6F74696F6E0044363A445320544C
:100F0000656D700044353A555620496E74656E73B0
:100F10006974790044343A4F3220636F6E632E0057
:100F200044333A434F3220636F6E632E0044323AAB
:100F3000504D28313A322E353A3130290044323A78
:100F4000504D28313A322E353A3130292A00443179
:100F50003A5475726269646974790044303A566F24
:100F60006C7461676500393A6F72203344206163A5
:100F700063656C2E00393A496E636C2E20616E6792
:100F80002E00383A70482076616C756500373A4912
:100F9000522054656D7000373A49522054656D7087
:100FA0002A00363A4D61676E65746963206669652B
:100FB0006C6400353A476173204C6576656C00348B
:100FC0003A495220466C616D6500333A4C69676856
:100FD0007420496E742E00323A616E64204865694F
:100FE00067687400323A54656D702050726573738F
:100FF00075726500313A54656D702048756D69648D
:1010000069747900303A536F756E64204C6576656B
:101010006C00303A536F756E64204C6576656C2AAF
:101020000054696D65206C617073653A00576946BC
:10103000692049503A0000002100240027002A00BE
:101040002D003000330001010000040107010A01F6
:1010500000002200250028002B002E003100340063
:1010600002010000050108010B010000200023001F
:10107000260029002C002F0032000001000003018F
:10108000060109010505050507050808080802020B
:1010900002020A0A08080404040401010101010112
:1010A00001010303030303030303040707070C0CF5
:1010B0000C0C0C0C0C0C02020202060606060606BC
:1010C00006060B0B0B0B0B0B0B0B01021020200861
:1010D0000810204010204080020102010804020193
:1010E0000102040810204080804020100804020102
:1010F000800402018040201008040201080402015B
:1011000001020408102040800102040810204080E1
:1011100000000A0B02090C0D0E0807030401000071
:1011200000000000000000000000000000000000BF
:10113000000000000000000000000000121110007C
:10114000000000000000000000000000000000009F
:10115000000000000000359F95A111241FBECFEFB5
:10116000D1E2DEBFCDBF00E00CBF1DE0A0E0B2E0E9
:10117000E4E2FCE501E00BBF02C007900D92A03253
:10118000B107D9F724E1A0E2BDE001C01D92AF3C58
:10119000B207E1F718E0CCEAD8E000E006C02197FA
:1011A0000109802FFE010E9454ABCB3AD10780E0A9
:1011B0000807A9F70E94B2950C9401AE0C940000A8
:1011C0003F924F925F926F927F928F929F92AF92D7
:1011D000BF92CF92DF92EF92FF920F931F93CF9324
:1011E000DF93CDB7DEB7C654D1090FB6F894DEBF92
:1011F0000FBECDBF10917C14112321F010927C14EE
:101200000C9463248091841390918513019709F0C5
:1012100050C060E070E080E893E10E949E57082E85
:10122000000C990B0E9498AD892B09F442C061E52E
:1012300076E0CE0183960E941559BE016D5D7F4F09
:1012400080E893E10E942654811127C064E37AE08C
:10125000CE0145960E941559BE016B5E7F4F80E816
:1012600093E10E942654811114C063E77CE0CE0113
:1012700001960E941559BE016F5F7F4F80E893E190
:101280000E94265411E0811110E0CE0101960E94C7
:10129000D158CE0145960E94D158CE0183960E9426
:1012A000D158112331F060E873E184E793E10E94A3
:1012B00082588091841390918513049708F041C05F
:1012C00062E878E0CE0101960E941559BE016F5F79
:1012D0007F4F80E893E10E942654182FCE0101969B
:1012E0000E94D158112369F161E070E080E893E138
:1012F0000E949E5780330CF484516AE270E0681BB0
:10130000710987FD7395CE0101960E941B72BE0183
:101310006F5F7F4F80E893E10E949758CE0101965E
:101320000E94D15860E873E184E793E10E948258FB
:1013300080E893E10E943357CB010E947C240C94F7
:10134000632462EC77E0CE0145960E941559BE01F8
:101350006B5E7F4F80E893E10E942654811116C096
:1013600068EC77E0CE0101960E941559BE016F5FCF
:101370007F4F80E893E10E94265411E0811101C063
:1013800010E0CE0101960E94D15801C011E0CE01BB
:1013900045960E94D158112309F483C363EC75E08C
:1013A000CE0101960E941559CE0101960E94157733
:1013B000CE0101960E94D1586FEC75E0CE010196E6
:1013C0000E94155967E574E1CE0101960E942258EA
:1013D000BC01CE0145960E940D59CE0145960E9452
:1013E0001577CE0145960E94D158CE0101960E94F4
:1013F000D1586091BD047091BE048091BF0490915A
:10140000C0040E947CA620E030E048EC52E40E9438
:10141000CCA8AB01BC0122E0CE0145960E94D65873
:1014200065EE75E0CE0101960E941559BE016B5E16
:101430007F4FCE0101960E9422586EE677E00E940F
:101440000B58BC01CE0183960E940D59CE018396A4
:101450000E941577CE0183960E94D158CE01019645
:101460000E94D158CE0145960E94D1584091B904AE
:101470005091BA046091BB047091BC0424E0CE0189
:1014800045960E94D6586AEF75E0CE0101960E94FB
:101490001559BE016B5E7F4FCE0101960E94225806
:1014A000BC01CE0183960E940D59CE0183960E9405
:1014B0001577CE0183960E94D158CE0101960E94E5
:1014C000D158CE0145960E94D1584091AD0450911B
:1014D000AE046091AF047091B00422E0CE018F960B
:1014E0000E94D6584091A5045091A6046091A7048B
:1014F0007091A80423E0CE0189960E94D6584091AD
:10150000B1045091B2046091B3047091B40422E02C
:10151000CE0183960E94D6584091A9045091AA0406
:101520006091AB047091AC0423E0CE0145960E941B
:10153000D65867E176E0CE0101960E941559BE01AA
:101540006B5E7F4FCE0101960E9422586CE276E0DE
:101550000E940B58BE016D5D7F4F0E9422586FE2C2
:1015600076E00E940B58BE01675D7F4F0E942258B3
:101570006CE276E00E940B58BE01615D7F4F0E94D5
:10158000225865E376E00E940B58BC01CE01C59657
:101590000E940D59CE01C5960E941577CE01C596C1
:1015A0000E94D158CE0101960E94D158CE01459695
:1015B0000E94D158CE0183960E94D158CE018996BF
:1015C0000E94D158CE018F960E94D15862E874E0F3
:1015D000CE0101960E940559F09002120F2D0F2C9A
:1015E000000C110B01151105A1F52091031230918A
:1015F0000412409105125091061260E070E080EAFA
:1016000090E40E94CCA8AB01BC0122E0CE018396FD
:101610000E94D6586AE376E0CE0145960E9415599D
:10162000BE016D5D7F4FCE0145960E9422586EE649
:1016300076E00E940B58BC01CE0101960E944158F1
:10164000CE0145960E94D158CE0183960E94D15872
:1016500009C00130110531F465E476E0CE01019650
:101660000E943358C8010297029738F52F2D4AE09F
:101670002402B0011124CE0183960E941B7263E5FF
:1016800076E0CE0145960E941559BE016D5D7F4FF3
:10169000CE0145960E94225861E576E00E940B58E3
:1016A000BC01CE0101960E944158CE0145960E9490
:1016B000D158CE0183960E94D1580430110519F4F7
:1016C0006FE576E005C00530110534F061E776E09E
:1016D000CE0101960E943358BE016F5F7F4FCE014D
:1016E00045960E940D59CE0145960E941577CE0170
:1016F00045960E94D15869E776E0CE0101960E9496
:101700006D588091FF116091001270910112833029
:1017100014F00C945024CE0183960E941B726AE54B
:1017200076E0CE0145960E941559BE016D5D7F4F52
:10173000CE0145960E94225869E876E00E940B5837
:10174000BC01CE0101960E944158CE0145960E94EF
:10175000D158CE0183960E94D158BE016F5F7F4F52
:10176000CE0145960E940D59CE0145960E941577EF
:10177000CE0145960E94D15840910712509108120F
:101780006091091270910A1222E0CE0183960E94A4
:10179000D6586BE876E0CE0145960E941559BE01F9
:1017A0006D5D7F4FCE0145960E94225861EA76E03A
:1017B0000E940B58BC01CE0189960E940D59CE01A2
:1017C00089960E941577CE0189960E94D158CE0144
:1017D00045960E94D158CE0183960E94D1584091DF
:1017E0001D1250911E1260911F127091201222E062
:1017F000CE0183960E94D65868EA76E0CE014596DF
:101800000E941559BE016D5D7F4FCE0145960E9425
:1018100022586BEB76E00E940B58BC01CE018996F2
:101820000E940D59CE0189960E941577CE018996A6
:101830000E94D158CE0145960E94D158CE01839680
:101840000E94D15865E9C62E64E0D62E01E010E072
:1018500079E1F72E80919304909194048017910779
:101860000CF44DC0D601AD90BD906D01B501CE0117
:1018700089960E941B72B801CE0183960E941B724A
:101880006EEB76E0CE0145960E941559BE016D5D66
:101890007F4FCE0145960E94225866EC76E00E946A
:1018A0000B58BE01675D7F4F0E94225869EC76E0BD
:1018B0000E940B58FA9CB001FB9C700D1124655ED0
:1018C0007D4F0E940B58BC01CE018F960E940D598E
:1018D000CE018F960E941577CE018F960E94D15827
:1018E000CE0145960E94D158CE0183960E94D158D0
:1018F000CE0189960E94D1580F5F1F4FABCF8091C8
:10190000491290914A12892B71F46FEC76E0CE0166
:1019100045960E941559CE0145960E941577CE0135
:1019200045960E94D1588091491290914A12019790
:1019300071F46EED76E0CE0145960E941559CE0108
:1019400045960E941577CE0145960E94D158809108
:10195000491290914A12029771F468EE76E0CE0136
:1019600045960E941559CE0145960E941577CE01E5
:1019700045960E94D1586091260570912705CE01A9
:1019800083960E941B726AEF76E0CE0145960E9414
:101990001559BE016D5D7F4FCE0145960E942258BC
:1019A000BC01CE0189960E940D59CE0189960E94F4
:1019B0001577CE0189960E94D158CE0145960E9496
:1019C000D158CE0183960E94D15840911702509170
:1019D00018026091190270911A0222E0CE018396DA
:1019E0000E94D65867E177E0CE0145960E941559CE
:1019F000BE016D5D7F4FCE0145960E9422586FEC6F
:101A000079E00E940B58BC01CE0189960E940D59C5
:101A1000CE0189960E941577CE0189960E94D158F1
:101A2000CE0145960E94D158CE0183960E94D1588E
:101A300040911302509114026091150270911602A8
:101A400022E0CE0183960E94D65867E277E0CE016D
:101A500045960E941559BE016D5D7F4FCE0145969A
:101A60000E9422586FEC79E00E940B58BC01CE0115
:101A700089960E940D59CE0189960E941577CE0154
:101A800089960E94D158CE0145960E94D158CE0128
:101A900083960E94D15810921202CE0101960E94A4
:101AA000D15880918413909185138330910508F06B
:101AB00092C08130910541F460E070E080E893E1EC
:101AC0000E949E57E82E62C0029709F05FC062E84C
:101AD00078E0CE0101960E941559BE016F5F7F4FDD
:101AE00080E893E10E942654182FCE0101960E94AF
:101AF000D158112309F44AC061E070E080E893E115
:101B00000E949E571A8219821C821B821E821D828D
:101B10008D8B1E8ABE016B5E7F4FCE0101960E94A7
:101B20006D58BE016F5F7F4F84E793E10E94975825
:101B3000CE0101960E94D15860E070E080E893E108
:101B40000E949E57E82E8091CE0D8823F9F067E31E
:101B500077E0CE0101960E94155960E873E1CE014D
:101B600001960E94225867E67CE00E940B58BC0157
:101B700088E590E10E947359CE0101960E94D158E8
:101B800064E773E188E590E10E94987C8E2D0E2C2D
:101B9000000C990B0E9498AD892BB1F00E942F4543
:101BA0000E94A48167E67CE0CE0101960E9415594F
:101BB0004AE050E060E070E0CE0101960E942C7493
:101BC000CE0101960E94D1588E2D0E943A8F0E941C
:101BD0007F930C943F2421E030E040E050E060E847
:101BE00073E1CE0101960E942959BE016F5F7F4FBC
:101BF00082E693E10E949758CE0101960E94D15847
:101C00006AE677E0CE0145960E941559BE016B5EEB
:101C10007F4F80E893E10E942654811116C06FE641
:101C20007CE0CE0101960E941559BE016F5F7F4F87
:101C300080E893E10E94265411E0811101C010E078
:101C4000CE0101960E94D15801C011E0CE01459607
:101C50000E94D158112309F4BEC080918413909141
:101C60008513409710F00C94632442E050E060E844
:101C700073E1CE0101960E946782BE016F5F7F4FC4
:101C800082E693E10E949758CE0101960E94D158B6
:101C900062E673E1CE0101960E940D59CE010196D4
:101CA0000E945B73CE0101960E94D15882E693E1B7
:101CB0000E94285720E030E048EC52E40E94DBA666
:101CC0000E9465A9AB01BC014093BD045093BE04C2
:101CD0006093BF047093C004CE0101960E94527DB0
:101CE000CE0101960E945B73CE0101960E94D158ED
:101CF0006091BD047091BE048091BF049091C004B6
:101D00008B019C0100591F452140310901341C49B8
:101D10002105310588F06DE377E0CE0101960E9440
:101D2000155962E673E1CE0101960E94225860E5E2
:101D300077E00E940B58BBC11A821982FE013396CC
:101D400026E0DF011D922A95E9F70E947CA620E09B
:101D500030E048EC52E40E94CCA88E010F5F1F4F88
:101D600022E047E00E94C1A1BC0188E693E10E9405
:101D70006D5860E677E0CE0145960E94155968E6F9
:101D800073E1CE0145960E9422586DE677E00E94ED
:101D90000B58BC0188E693E10E948258CE0145961B
:101DA0000E94D15810927C0D10927B0D8091BD0441
:101DB0009091BE04A091BF04B091C0048093D31150
:101DC0009093D411A093D511B093D61180E090E0F8
:101DD0000E94048175C162E777E0CE0145960E94BA
:101DE0001559BE016B5E7F4F80E893E10E94265437
:101DF000811116C068E777E0CE0101960E9415595F
:101E0000BE016F5F7F4F80E893E10E94265411E08E
:101E1000811101C010E0CE0101960E94D15801C08D
:101E200011E0CE0145960E94D158112309F469C0F2
:101E300026E030E045E050E060E873E1CE01019635
:101E40000E942959BE016F5F7F4F82E693E10E9495
:101E50009758CE0101960E94D15882E693E10E94E4
:101E600033576B017C016FE976E0CE0101960E9449
:101E70001559BE016F5F7F4F80E893E10E94C35305
:101E8000AC014F5F5F4F60E873E1CE0145960E9461
:101E90006782BE016B5E7F4F82E693E10E94975896
:101EA000CE0145960E94D158CE0101960E94D1588C
:101EB00082E693E10E9433579B01E3E9F4E041E0BD
:101EC00050E0A0919304B0919404A417B5075CF07E
:101ED000A281B3812A173B0711F4138212824F5F4C
:101EE0005F4F3296EECF9601220F331FF901ED5668
:101EF000FB4F7183608382E090E00E9489460C94DE
:101F000099196EE777E0CE0145960E941559BE01FA
:101F10006B5E7F4F80E893E10E942654811116C0CA
:101F200064E877E0CE0101960E941559BE016F5F0B
:101F30007F4F80E893E10E94265411E0811101C097
:101F400010E0CE0101960E94D15801C011E0CE01EF
:101F500045960E94D158112339F1E3E9F4E081E07C
:101F600090E020919304309194042817390774F07D
:101F7000863091051CF49383828305C09C012E5FFB
:101F80003F4F3383228301963296EBCF82E090E07D
:101F90000E94894610927C0D10927B0D80E090E0AB
:101FA0000E9404810C942B246AE877E0CE014596C8
:101FB0000E941559BE016B5E7F4F80E893E10E943D
:101FC0002654811116C061E977E0CE0101960E9486
:101FD0001559BE016F5F7F4F80E893E10E94265440
:101FE00011E0811101C010E0CE0101960E94D1588C
:101FF00001C011E0CE0145960E94D1581123F9F09D
:102000008091E50D9091E60D892BA1F481E090E09F
:102010009093E60D8093E50D8EED93E090937C0D0B
:1020200080937B0D0E942D8168EC70E080E090E051
:102030000E944793E0E0F0E019950C942D2468E9A4
:1020400077E0CE0145960E941559BE016B5E7F4F29
:1020500080E893E10E942654811116C060EA77E07F
:10206000CE0101960E941559BE016F5F7F4F80E837
:1020700093E10E94265411E0811101C010E0CE01CD
:1020800001960E94D15801C011E0CE0145960E94F0
:10209000D1581123A1F168EA77E0CE0101960E94A0
:1020A000155961E574E1CE0101960E942258BC01E8
:1020B00088E693E10E948258CE0101960E94D15891
:1020C00065E57CE0CE0101960E94155968E673E152
:1020D000CE0101960E942258BC01CE0145960E9475
:1020E0000D59CE0145960E941577CE0145960E9466
:1020F000D158CE0101960E94D1580C942B2462EB4A
:1021000077E0CE0145960E941559BE016B5E7F4F68
:1021100080E893E10E942654811116C069EB77E0B4
:10212000CE0101960E941559BE016F5F7F4F80E876
:1021300093E10E94265411E0811101C010E0CE010C
:1021400001960E94D15801C011E0CE0145960E942F
:10215000D158112349F067ED75E0CE0101960E9438
:10216000155967E574E19FCF60EC77E0CE014596A5
:102170000E941559BE016B5E7F4F80E893E10E947B
:102180002654811116C066EC77E0CE0101960E94BC
:102190001559BE016F5F7F4F80E893E10E9426547E
:1021A00011E0811101C010E0CE0101960E94D158CA
:1021B00001C011E0CE0145960E94D158112311F1C2
:1021C0006FE574E088E693E10E94475868E673E1A2
:1021D000CE0101960E940D59CE0101960E941577FD
:1021E000CE0101960E94D1580E945F871092120280
:1021F00062EC77E080E893E10E946D580E94E0086D
:102200000C942D246CEC77E0CE0145960E94155974
:10221000BE016B5E7F4F80E893E10E9426548111DE
:1022200016C063ED77E0CE0101960E941559BE01FC
:102230006F5F7F4F80E893E10E94265411E0811187
:1022400001C010E0CE0101960E94D15801C011E0FA
:10225000CE0145960E94D158112309F48FC06FE931
:1022600076E0CE0101960E941559BE016F5F7F4F47
:1022700080E893E10E94C353AC014F5F5F4F60E879
:1022800073E1CE0145960E946782BE016B5E7F4F6F
:1022900082E693E10E949758CE0145960E94D1585C
:1022A000CE0101960E94D15882E693E10E943357F5
:1022B0008B0162E574E088E693E10E9447588091C3
:1022C0006212882331F066E474E088E693E10E94AC
:1022D00047580115110511F40C941D24CE010196E7
:1022E0000E944364CE0101960E941577CE010196AB
:1022F0000E94D1580230110514F40C942B246BE980
:1023000076E0CE0145960E940559BE016B5E7F4F77
:10231000CE0101960E940D59CE0101960E941577BB
:10232000CE0101960E94D158E12CF12C80916412CB
:10233000082E000C990BE816F9068CF4B701CE01B3
:1023400001960E942863CE0101960E941577CE0166
:1023500001960E94D158FFEFEF1AFF0AE7CFCE0196
:1023600045960E94D1580230110511F40C942B248B
:102370008CE291E00E947A810C942B246AED77E044
:10238000CE0145960E941559BE016B5E7F4F80E8D5
:1023900093E10E942654811117C061EE77E0CE01CF
:1023A00001960E941559BE016F5F7F4F80E893E14F
:1023B0000E942654FF24F394811101C0F12CCE0118
:1023C00001960E94D15802C0FF24F394CE01459695
:1023D0000E94D1588E010B5E1F4FFF2009F48DC360
:1023E00060E873E1CE018F5B9F4F0E940D596FE94A
:1023F00076E0CE0101960E941559BE016F5F7F4FB6
:10240000CE018F5B9F4F0E94C353AC014F5F5F4F64
:10241000BE016F5B7F4FCE01CB960E946782CE01DB
:1024200001960E94D158BE016F5B7F4FCE0101968D
:102430000E940D59CE0101960E945B73CE01019658
:102440000E94D1586EED77E0CE0101960E94155999
:10245000BE016F5F7F4FCE01CB960E9487537C01F8
:10246000CE0101960E94D1586FEC7CE0CE01C5965A
:102470000E9415596FEC7CE0CE018F960E94155991
:102480001E141F0494F5A7014F5F5F4F21968EAD78
:102490009FAD21974817590790F4BE01655C7F4FA7
:1024A000CE0101960E946782BE016F5F7F4FCE0111
:1024B000C5960E949758CE0101960E94D158970167
:1024C00040E050E0BE01655C7F4FCE0101960E9466
:1024D0002959BE016F5F7F4FCE018F960E9497589A
:1024E000CE0101960E94D1580DC06FEC7CE0CE0168
:1024F000C5960E946D58BE01655C7F4FCE018F96D8
:102500000E9482588BA99CA9892B09F4E6C2CE01AE
:102510008F960E9433577B0121E0E21AF10848E1CF
:10252000E416F1041CF047E1E42EF12CF7FE03C0A1
:10253000EE24EA94FE2CB701CE0145960E941B7250
:1025400060EE77E0CE0101960E941559BE016B5EE8
:102550007F4FCE0101960E942258BC01CE01839686
:102560000E940D59CE0183960E945B73CE01839623
:102570000E94D158CE0101960E94D158CE014596B5
:102580000E94D158BE016B5C7F4FCE01CB960E945A
:1025900082586EED77E0CE0101960E941559BE017A
:1025A0006F5F7F4FCE01CB960E9487536C01CE01A7
:1025B00001960E94D1586FEC7CE0CE01C5960E9436
:1025C0006D586FEC7CE0CE018F960E946D581C1404
:1025D0001D040CF04FC0A6014F5F5F4F21968EADDA
:1025E0009FAD21974817590790F4BE01655C7F4F56
:1025F000CE0101960E946782BE016F5F7F4FCE01C0
:10260000C5960E949758CE0101960E94D158960116
:1026100040E050E0BE01655C7F4FCE0101960E9414
:102620002959BE016F5F7F4FCE018F960E94975848
:10263000CE0101960E94D158CE0101963C01C12CD9
:10264000D12CA7014F5F5F4F8AE0849F9001859F47
:10265000300D1124D901AE59BD4E5D018E9D900102
:102660008F9D300D1124F901E059FD4E2F012AE212
:10267000322EBBC06FEC7CE0CE01C5960E946D5837
:10268000BE01655C7F4FCE018F960E948258D4CFE9
:10269000CE018F96C114D10409F0B4C02FEFE21619
:1026A000F20609F4AFC00E943E57A114B10439F0FC
:1026B00044E050E0B501CE018F960E94A153B501D0
:1026C000CE0183960E94155965EE77E0C8010E94FD
:1026D0001559BE016D5D7F4FC8010E942258BC0193
:1026E000CE0189960E940D59CE0189960E945B7396
:1026F000CE0189960E94D158C8010E94D158CE01BE
:1027000083960E94D1588BA99CA9029708F473C0A4
:1027100061E070E0CE018F960E949E57082E000C5B
:10272000990B803391050CF44497432D481BD2013B
:102730004C93BFEFCB1ADB0ABE016B5C7F4FCE011F
:10274000CB960E9482586EED77E0CE0145960E94AE
:102750001559BE016B5E7F4FCE01CB960E94875309
:102760004C01CE0145960E94D1586FEC7CE0CE0121
:10277000C5960E946D586FEC7CE0CE018F960E944A
:102780006D58181419040CF043C0A4014F5F5F4F3B
:1027900021968EAD9FAD21974817590790F4BE0141
:1027A000655C7F4FCE0145960E946782BE016B5EDD
:1027B0007F4FCE01C5960E949758CE0145960E9444
:1027C000D158940140E050E0BE01655C7F4FC801E4
:1027D0000E942959B801CE018F960E949758C801CE
:1027E0000E94D158F2E06F0E711C8BA99CA9892B15
:1027F00009F04ECF1BC0CE018F960E943357F201D5
:10280000608397CF0E943357D3016D937C9391CF10
:102810006FEC7CE0CE01C5960E946D58BE01655CF0
:102820007F4FCE018F960E948258DCCFEFEFEE16DD
:10283000FE0609F080C06EED77E0CE0145960E945D
:102840001559BE016B5E7F4FCE01C5960E9487531E
:102850007C01CE0145960E94D158F7FE3EC1E98029
:10286000FA801E141F0444F4F9E1EF16F1043CF061
:1028700098E1E92EF12C03C0EE24E394F12CE092D0
:102880006412B701CE0183960E941B7263EF77E05A
:10289000C8010E941559BE016D5D7F4FC8010E949D
:1028A0002258BC01CE0189960E940D59CE0189960D
:1028B0000E945B73CE0189960E94D158C8010E9484
:1028C000D158CE0183960E94D158C114D10471F120
:1028D0008B819C8197FF02C080E090E0909366120C
:1028E0008093651221E0C216D10401F18D819E8191
:1028F0001816190634F497018E159F0524F49C01CF
:1029000002C021E030E0EE24EA94E20EE092691287
:1029100042E0C416D10451F08F819885181619062B
:1029200014F081E090E0815080936A128CE291E093
:102930000E945181D2C080916312082E000C990B25
:10294000E816F9060CF083C0B601CE0183960E940A
:102950001B726DEF77E0CE0145960E941559BE01BE
:102960006D5D7F4FCE0145960E942258BC01CE017D
:1029700089960E940D59CE0189960E945B73CE0103
:1029800089960E94D158CE0145960E94D158CE0119
:1029900083960E94D1588AE08E9DF0018F9DF00DA4
:1029A0001124EE59FD4E81E0878783E090E0918B02
:1029B000808B938B828BC114D10409F48EC08B81E0
:1029C0009C818038910514F08FE790E080385FEFAC
:1029D000950714F480E89FEF878781E0C816D1043B
:1029E00009F47BC08AE08E9DF0018F9DF00D1124CB
:1029F000EE59FD4E8D819E8197FF02C080E090E0F0
:102A0000918B808B92E0C916D10409F466C08AE0EC
:102A10008E9DF0018F9DF00D1124EE59FD4E8F819A
:102A2000988597FF02C080E090E0938B828B809125
:102A30006412082E000C990BE816F9061CF0E394BA
:102A4000E09264128CE291E00E947A8146C0BE015D
:102A50006B5C7F4FCE0189960E940D596091631285
:102A6000062E000C770BCE0183960E941B7265E048
:102A700078E0CE0145960E941559BE01675D7F4FF3
:102A8000CE0145960E94225866E178E00E940B58DC
:102A9000BE016D5D7F4F0E942258BC01CE01899618
:102AA0000E948258CE0145960E94D158CE0183964D
:102AB0000E94D158BE01675D7F4FCE0145960E94AE
:102AC0000D59CE0145960E941577CE0145960E947C
:102AD000D158CE0189960E94D158CE018F960E947E
:102AE000D158CE01C5960E94D158CE01CB960E94F6
:102AF000D158CE018F5B9F4F54C26AE178E0CE017E
:102B000045960E941559BE016B5E7F4F80E893E1A8
:102B10000E942654811117C06FE178E0CE01019622
:102B20000E941559BE016F5F7F4F80E893E10E94BC
:102B30002654FF24F394811101C0F12CCE0101969B
:102B40000E94D15802C0FF24F394CE0145960E9402
:102B5000D158FF20D9F16FE976E0CE0101960E94AD
:102B60001559BE016F5F7F4F80E893E10E94C35308
:102B7000AC014F5F5F4F60E873E1CE0145960E9464
:102B80006782BE016B5E7F4F82E693E10E94975899
:102B9000CE0145960E94D158CE0101960E94D1588F
:102BA00082E693E10E9433576115710521F481E0BB
:102BB0008093DD0407C06130710511F00C942B2463
:102BC0001092DD040E943F450C942B2464E278E0CF
:102BD000CE0145960E941559BE016B5E7F4F80E87D
:102BE00093E10E942654811117C068E278E0CE017B
:102BF00001960E941559BE016F5F7F4F80E893E1F7
:102C00000E942654FF24F394811101C0F12CCE01BF
:102C100001960E94D15802C0FF24F394CE0145963C
:102C20000E94D158FF2009F424C143E050E060E83D
:102C300073E1CE0101960E946782BE016F5F7F4FF4
:102C400082E693E10E949758CE0101960E94D158E6
:102C500062E673E1CE0101960E940D59CE01019604
:102C60000E945B73CE0101960E94D15810927C0D98
:102C700010927B0D62E673E18DE594E10E9482582B
:102C800062E673E187E594E10E9482588FEE91E15C
:102C9000009739F048E050E0BC018DE594E10E94D6
:102CA000A1538DE492E1009739F04CE050E0BC0173
:102CB00087E594E10E94A15380917B0D90917C0D5A
:102CC0000E9404816CE278E0CE0101960E941559C1
:102CD00067E574E1CE0101960E942258BC01CE0145
:102CE00083960E940D59CE0101960E94D158809181
:102CF000491290914A12892B39F4BE016D5D7F4FC4
:102D000081E89EE00E9473598091491290914A1285
:102D1000029709F09BC067E574E1CE0189960E9495
:102D20000D5964E378E0CE0101960E941559CE0159
:102D300001960E94F09ECE0101960E94D15864EF48
:102D400071E080E090E00E94479367E378E0CE0175
:102D500001960E941559CE0101960E94F09ECE0167
:102D600001960E94D15864EF71E080E090E00E94EB
:102D7000479360E478E0CE0101960E941559CE0198
:102D800001960E94F09ECE0101960E94D15864EFF8
:102D900071E080E090E00E94479369E478E0CE0122
:102DA00001960E941559CE0101960E94F09ECE0117
:102DB00001960E94D15864EF71E080E090E00E949B
:102DC000479367E578E0CE0101960E941559CE0140
:102DD00001960E94F09ECE0101960E94D15864EFA8
:102DE00071E080E090E00E9447936CE278E0CE01D1
:102DF00001960E941559BE01675D7F4FCE01019675
:102E00000E942258BC01CE0145960E940D59CE0168
:102E100001960E94D158CE0145960E943E57BE01B0
:102E20006B5E7F4FCE0101960E940D59CE01019637
:102E30000E94F09ECE0101960E94D158CE01459687
:102E40000E94D158CE0189960E94D1586FEE71E14F
:102E5000CE0101960E941559CE0101960E945B7326
:102E6000CE0101960E94D15810921202CE01839693
:102E700098C065E678E0CE0145960E941559BE01DE
:102E80006B5E7F4F80E893E10E942654811117C04A
:102E90006AE678E0CE0101960E941559BE016F5F87
:102EA0007F4F80E893E10E942654FF24F394811120
:102EB00001C0F12CCE0101960E94D15802C0FF241E
:102EC000F394CE0145960E94D158FF2009F46DC0BD
:102ED00044E050E060E873E1CE0101960E94678211
:102EE000BE016F5F7F4F82E693E10E949758CE014B
:102EF00001960E94D1586FE678E0CE0145960E9477
:102F0000155962E673E1CE0145960E942258BC0134
:102F1000CE0101960E940D59CE0145960E94D158CE
:102F20008091491290914A12892B39F4BE016F5F4A
:102F30007F4F81E89EE00E94735968EB7BE080E060
:102F400090E00E9447938091491290914A12029713
:102F500079F4BE016F5F7F4FCE0145960E940D59F7
:102F6000CE0145960E94F09ECE0145960E94D15812
:102F700068EB7BE080E090E00E944793BE016F5FCA
:102F80007F4FCE0145960E940D59CE0145960E9475
:102F90005B73CE0145960E94D15810921202CE0169
:102FA00001960E94D1580C942D2466E778E0CE015A
:102FB00045960E941559BE016B5E7F4F80E893E1F4
:102FC0000E942654811117C06AE778E0CE0101966D
:102FD0000E941559BE016F5F7F4F80E893E10E9408
:102FE0002654FF24F394811101C0F12CCE010196E7
:102FF0000E94D15802C0FF24F394CE0145960E944E
:10300000D158FF2009F46FC060E873E182E693E1D4
:103010000E94825881E08093120260E873E1CE0141
:1030200001960E940D59CE0101960E945B73CE015C
:1030300001960E94D1588091491290914A120297AC
:1030400009F162E673E181E89EE00E94735968EB42
:103050007BE080E090E00E944793CE0101960E94C1
:10306000FD7BBE016F5F7F4F80E893E10E94975820
:10307000CE0101960E94D15860ED77E080E090E0AB
:103080000E9447938091491290914A12029771F4DD
:1030900062E673E1CE0101960E940D59CE010196C0
:1030A0000E94F09ECE0101960E94D1588091841317
:1030B00090918513892B11F40C942B2465E57CE009
:1030C000CE0101960E94155960E873E1CE01019688
:1030D0000E942258BC01C8010E940D59C8010E94DB
:1030E0001577C80104C86EE778E0CE0145960E94C6
:1030F0001559BE016B5E7F4F80E893E10E94265414
:10310000811117C064E878E0CE0101960E9415593C
:10311000BE016F5F7F4F80E893E10E942654FF2439
:10312000F394811101C0F12CCE0101960E94D15877
:1031300002C0FF24F394CE0145960E94D158FF208F
:1031400009F461C08091491290914A12019711F0DF
:103150000C942B24CE0101960E949D478D819E8167
:10316000009711F40C942724E981FA81208122230D
:1031700011F40C942724079710F40C9427246DE382
:1031800074E0CE0145960E94055948EC50E06FEF7F
:103190007FEFCE0145960E942C74CE0145960E9489
:1031A000D158BE016F5F7F4FCE0145960E940D59E9
:1031B00040ED57E06FEF7FEFCE0145960E94D3813F
:1031C000CE0145960E94D1586AE878E0CE01459636
:1031D0000E94155960E873E1CE0145960E9422587D
:1031E000BC01CE0183960E940D59CE0183960E94A8
:1031F0001577CE0183960E94D158CE0145960E9444
:10320000D1580C94272468E978E0CE0145960E94B5
:103210001559BE016B5E7F4F80E893E10E942654F2
:10322000811117C06DE978E0CE0101960E94155911
:10323000BE016F5F7F4F80E893E10E942654FF2418
:10324000F394811101C0F12CCE0101960E94D15856
:1032500002C0FF24F394C8010E94D158FF20F1F06E
:1032600025E030E044E050E060E873E1CE010196F3
:103270000E942959BE016F5F7F4F82E693E10E9451
:103280009758CE0101960E94D15882E693E10E94A0
:10329000335770934A12609349124BC062EA78E048
:1032A000C8010E941559B80180E893E10E94265494
:1032B000811117C067EA78E0CE0101960E94155986
:1032C000BE016F5F7F4F80E893E10E942654FF2488
:1032D000F394811101C0F12CCE0101960E94D158C6
:1032E00002C0FF24F394C8010E94D158FF2089F145
:1032F00026E030E044E050E060E873E1CE01019662
:103300000E942959BE016F5F7F4F82E693E10E94C0
:103310009758CE0101960E94D15882E693E10E940F
:10332000335770934C1260934B1270932705609340
:10333000260560E873E1CE0101960E940D59CE0189
:1033400001960E945B73CE0101960E94D1580C94A5
:10335000CA0F6CEA78E0C8010E941559B80180E8EC
:1033600093E10E942654811117C063EB78E0CE01EF
:1033700001960E941559BE016F5F7F4F80E893E16F
:103380000E942654FF24F394811101C0F12CCE0138
:1033900001960E94D15802C0FF24F394C8010E94F4
:1033A000D158FF2069F127E030E046E050E060E8C6
:1033B00073E1CE0101960E942959BE016F5F7F4FD4
:1033C00082E693E10E949758CE0101960E94D1585F
:1033D00082E693E10E943357672B19F41092CE0DC9
:1033E00003C081E08093CE0D60E873E1CE010196C9
:1033F0000E940D59CE0101960E945B730C94272404
:103400006AEB78E0CE0183960E941559BE016D5D8E
:103410007F4F80E893E10E942654811129C06DEB13
:1034200078E0C8010E941559B80180E893E10E9434
:103430002654811117C060EC78E0CE0101960E94FD
:103440001559BE016F5F7F4F80E893E10E942654BB
:10345000FF24F394811101C0F12CCE0101960E944A
:10346000D15802C0FF24F394C8010E94D15802C071
:10347000FF24F394CE0183960E94D158FF2009F4D3
:103480004BC1AAE0CA2ED12C412C512C3201AA24C6
:10349000AA94B3E0BB2E6EE170E080E090E00E9461
:1034A0004793809110020E94FD92B5010E9441ABAA
:1034B000072E000C880B990B0E947CA620E030E0C0
:1034C00040EA50E40E94DBA69B01AC01C301B201BB
:1034D0000E9406A82B013C01A1E0CA1AD108D9F626
:1034E00020E030E040E251E40E94CCA84B015C01B6
:1034F00063EC78E0C8010E941559B80180E893E1B7
:103500000E942654811117C067EC78E0CE01019625
:103510000E941559BE016F5F7F4F80E893E10E94C2
:103520002654EE24E394811101C0E12CCE010196D2
:103530000E94D15801C0EF2CC8010E94D158EE2042
:1035400009F44FC020E030E040E650E4C501B4018A
:103550000E94DBA69B01AC0160E070E080E890E493
:103560000E9405A8AB01BC0140930C0250930D02D0
:1035700060930E0270930F0222E0CE0101960E942A
:10358000D658BE016F5F7F4F88E693E10E9497583F
:10359000CE0101960E94D15880910C0290910D02AB
:1035A000A0910E02B0910F028093F7119093F81141
:1035B000A093F911B093FA116BEC78E0CE0101966B
:1035C0000E94155968E673E1CE0101960E942258C7
:1035D000BC0188E693E10E948258CE0101960E94C8
:1035E000D1586AED78E0C8010E941559B80180E809
:1035F00093E10E942654811116C06FED78E0CE0150
:1036000001960E941559BE016F5F7F4F80E893E1DC
:103610000E942654FF24F394811101C0F12CCE01A5
:1036200001960E94D158C8010E94D158FF2009F488
:1036300057C020E030E040E650E4C501B4010E94EC
:10364000DBA69B01AC0160E070E080E291E40E94A7
:1036500005A8AB01BC014093080250930902609396
:103660000A0270930B0222E0CE0101960E94D65806
:10367000BE016F5F7F4F88E693E10E949758CE01AD
:1036800001960E94D15864EE78E0CE0101960E9426
:10369000155968E673E1CE0101960E942258BC01DB
:1036A00088E693E10E948258CE0101960E94D1588B
:1036B0008091080290910902A0910A02B0910B0238
:1036C0008093FB119093FC11A093FD11B093FE1118
:1036D00010927C0D10927B0D80E090E00E9404819E
:1036E00065E57CE0CE0101960E94155968E673E11C
:1036F000CE0101960E942258BC01C8010E940D59BA
:10370000C8010E941577C8010E94D158CE010196C8
:103710000E94D1580C942D2464EF78E0CE010196DC
:103720000E941559BE016F5F7F4F80E893E10E94B0
:103730002654F82ECE0101960E94D158FF2009F49C
:103740006CC08091841390918513079710F40C94AA
:103750002D2446E050E060E873E1CE0101960E941E
:103760006782BE016F5F7F4F82E693E10E949758A8
:10377000CE0101960E94D15882E693E10E9428571B
:10378000AB01BC01409317025093180260931902D9
:1037900070931A0221E0C8010E94D65867E177E0D1
:1037A000CE0101960E941559B801CE0101960E94E2
:1037B00022586FEC79E00E940B58BC0188E693E137
:1037C0000E948258CE0101960E94D158C8010E94E1
:1037D000D15868E673E1CE0101960E940D59CE01E1
:1037E00001960E941577CE0101960E94D1580E9441
:1037F0007F9328EE33E040E050E00E94D4A7CA0156
:10380000B9010E947AA66093200D7093210D8093D8
:10381000220D9093230D0C942D246BEF78E0CE01B4
:1038200001960E941559BE016F5F7F4F80E893E1BA
:103830000E942654F82ECE0101960E94D158FF20F6
:10384000D9F18091841390918513079710F40C940B
:103850002D2446E050E060E873E1CE0101960E941D
:103860006782BE016F5F7F4F82E693E10E949758A7
:10387000CE0101960E94D15882E693E10E9428571A
:10388000AB01BC01409313025093140260931502E4
:103890007093160221E0C8010E94D65867E277E0D3
:1038A000CE0101960E941559B801CE0101960E94E1
:1038B00022586FEC79E005C262E079E0C8010E940D
:1038C0001559B80180E893E10E942654811117C070
:1038D00066E079E0CE0101960E941559BE016F5F46
:1038E0007F4F80E893E10E942654FF24F3948111D6
:1038F00001C0F12CCE0101960E94D15802C0FF24D4
:10390000F394C8010E94D158FF2009F455C080915A
:103910000602909107020E9480666093A90470934A
:10392000AA048093AB049093AC046093E711709366
:10393000E8118093E9119093EA1180E090E0A0E80B
:10394000BFE38093B1049093B204A093B304B09307
:10395000B4048093DF119093E011A093E111B09330
:10396000E2118091CE0D882381F061E274E088E558
:1039700090E10E9481596091A9047091AA048091FC
:10398000AB049091AC040E94374F10927C0D1092C2
:103990007B0D80E090E00E9404814091A904509149
:1039A000AA046091AB047091AC0422E0C8010E94AB
:1039B000D6586AE079E0E4C063E179E0C8010E948A
:1039C0001559B80180E893E10E942654811117C06F
:1039D00069E179E0CE0101960E941559BE016F5F41
:1039E0007F4F80E893E10E942654FF24F3948111D5
:1039F00001C0F12CCE0101960E94D15802C0FF24D3
:103A0000F394C8010E94D158FF2009F4C3C08091EB
:103A10008413909185130797F8F046E050E060E832
:103A200073E1CE0101960E946782BE016F5F7F4FF6
:103A300082E693E10E949758CE0101960E94D158E8
:103A400082E693E10E94285760932C0570932D0520
:103A500080932E0590932F0580910402909105028A
:103A600099270E948765BC01990F880B990B0E94CA
:103A70007CA62DE038E643E55BE30E94DBA66B0104
:103A80007C012091F6043091F7044091F8045091A4
:103A9000F9040E9476A618164CF06091DE0470912D
:103AA000DF048091E0049091E1041BC020910A059D
:103AB00030910B0540910C0550910D05C701B601E1
:103AC0000E94BBA987FF05C0C701B6010E94C27F43
:103AD00008C06091F2047091F3048091F404909115
:103AE000F50420E030E048EC52E40E94DBA66B01D4
:103AF0007C0120E030E0A9010E9476A6181634F07F
:103B0000C12CD12CF8EAEF2EF1E4FF2EC0922C0547
:103B1000D0922D05E0922E05F0922F05C09207124B
:103B2000D0920812E0920912F0920A128091CE0D02
:103B3000882381F06FE074E088E590E10E9481596C
:103B400060912C0570912D0580912E0590912F0587
:103B50000E94374F10927C0D10927B0D80E090E018
:103B60000E94048140912C0550912D0560912E05F5
:103B700070912F0522E0C8010E94D6586FE179E0CC
:103B8000CE0101960E941559B801CE0101960E94FE
:103B9000225899C069E279E0C8010E941559B8011C
:103BA00080E893E10E942654811117C06DE279E00C
:103BB000CE0101960E941559BE016F5F7F4F80E8CC
:103BC00093E10E942654FF24F394811101C0F12C4B
:103BD000CE0101960E94D15802C0FF24F394C8017F
:103BE0000E94D158FF2009F479C0D090020260E011
:103BF0008D2D0E94C192E9E1EE2EF12C812C912CA9
:103C000054018D2D0E94FD92BC01990F880B990BD8
:103C10000E947CA69B01AC01C501B4010E9406A8CC
:103C20004B015C016AE070E080E090E00E94479305
:103C3000B1E0EB1AF10829F720E030E040EA50E467
:103C4000C501B4010E94DBA620E030E040E85AE361
:103C50000E94DBA620E030E048EC51E40E94CCA8B2
:103C6000609328057093290580932A0590932B056E
:103C700060931D1270931E1280931F129093201256
:103C800010927C0D10927B0D80E090E00E940481E8
:103C9000409128055091290560912A0570912B05C6
:103CA00022E0C8010E94D65868EA76E0CE0101966B
:103CB0000E941559B801CE0101960E9422586BEB63
:103CC00076E00E940B58BC0188E693E10E9482587E
:103CD000CE0101960E94D158C801ADC561E379E0DB
:103CE000C8010E941559B80180E893E10E9426544A
:103CF000811117C065E379E0CE0101960E94155944
:103D0000BE016F5F7F4F80E893E10E942654FF243D
:103D1000F394811101C0F12CCE0101960E94D1587B
:103D200002C0FF24F394C8010E94D158FF2009F477
:103D30003FC126E030E044E050E060E873E1CE01AE
:103D400001960E942959BE016F5F7F4F82E693E181
:103D50000E949758CE0101960E94D15882E693E1C5
:103D60000E9433574B015C017B016FE976E0CE0185
:103D700001960E941559BE016F5F7F4F80E893E165
:103D80000E94C353AC014F5F5F4F60E873E1C8010D
:103D90000E946782B80182E693E10E949758C801A9
:103DA0000E94D158CE0101960E94D1583090000255
:103DB00082E693E10E9428572B013C016401E1E077
:103DC000CE1AD1088091CE0D8823B9F065E773E053
:103DD00088E590E10E9481594AE050E0B40188E50D
:103DE00090E10E94025A67E67CE088E590E10E943B
:103DF0004C5AC301B2010E94374F632DC8010E9483
:103E00008E8C18870F831D821E82198289E08A8317
:103E100081E08B838C831C8A1B8ACE0101960E94D1
:103E20008B51CE0101960E941B51CE0101960E943A
:103E300040500E8110E00B30110514F00AE010E044
:103E4000FBE58F16910408F44CC073E5C72E7DE0A6
:103E5000D72E5601412C512C3201E12CF12CE016C9
:103E6000F106BCF46E2DCE0101960E94D04F9B014D
:103E7000AC01D5016D937D938D939D935D01C3013D
:103E8000B2010E9406A82B013C01BFEFEB1AFB0A0E
:103E9000E6CFB801012E000C880B990B0E947CA67E
:103EA0009B01AC01C301B2010E94CCA84B015C0193
:103EB000E12CF12CE016F1060CF057C0F601208140
:103EC000318142815381C501B4010E9405A8D60108
:103ED0006D937D938D939D936D01BFEFEB1AFB0A5C
:103EE000E9CF1E141F040CF50E151F0524F46801FC
:103EF000E1E0CE1AD1086C2DCE0101960E94D04F80
:103F00009B01AC01C601880F991F880F991F8C0176
:103F10000D5A124FC301B2010E9405A8D8016D933A
:103F20007D938D939C93139720C0EF28F1F483E544
:103F3000C82E8DE0D82EE12CF12CE016F106ACF461
:103F40006E2DCE0101960E94D04F9B01AC01C301A2
:103F5000B2010E9405A8F601619371938193919338
:103F60006F01FFEFEF1AFF0AE8CFE3E5FDE0A1E202
:103F7000B2E141915191619171914D935D936D9336
:103F80007D932DE0EB37F207A1F710927C0D109294
:103F90007B0D80E090E00E94048144E050E060E806
:103FA00073E1CE0145960E94678269E379E02DC4F2
:103FB0006AE579E0C8010E941559B80180E893E1EB
:103FC0000E942654811117C061E679E0CE01019666
:103FD0000E941559BE016F5F7F4F80E893E10E94F8
:103FE0002654FF24F394811101C0F12CCE010196D7
:103FF0000E94D15802C0FF24F394C8010E94D158F6
:10400000FF2009F41EC127E030E046E050E060E800
:1040100073E1CE0101960E942959BE016F5F7F4F67
:1040200082E693E10E949758CE0101960E94D158F2
:1040300082E693E10E9433577B016093021280E88D
:1040400093E10E943E5767E67CE0CE0101960E9414
:104050001559BE016F5F7F4F80E893E10E94C35303
:10406000AC014F5F5F4F60E873E1C8010E94678257
:10407000C8010E9428576093031270930412809322
:10408000051290930612C8010E94D158CE010196E4
:104090000E94D1586EEF73E088E693E10E94475882
:1040A00044E0E416F1049CF452E0E516F1040CF04F
:1040B0005CC0E114F104B9F0EA94EF2809F095C06E
:1040C00065E476E088E693E10E94335872C094E09C
:1040D000E916F10409F089C06AE676E088E693E122
:1040E0000E943358A5C020E030E0A901609103127E
:1040F0007091041280910512909106120E9476A68A
:10410000181664F080E090E0A0E8BFE3809303120B
:1041100090930412A0930512B093061220910312FB
:1041200030910412409105125091061260E070E047
:1041300080EA90E40E94CCA8AB01BC0122E0CE0151
:1041400045960E94D6586AE376E0CE0101960E9419
:104150001559BE016B5E7F4FCE0101960E94225819
:104160006EE676E00E940B5856C08AE08E9DB00144
:104170008F9D700D1124C8010E941B7263E576E0CB
:10418000CE0101960E941559B801CE0101960E94F8
:10419000225861E576E00E940B58BC0188E693E165
:1041A0000E944158CE0101960E94D158C8010E9438
:1041B000D15820E030E0A9016091031270910412FF
:1041C00080910512909106120E9476A6811130C04E
:1041D00080E090E4ACE1B5E4809303129093041284
:1041E000A0930512B093061223C060910212062E0E
:1041F000000C770BCE0145960E941B7268E679E0B1
:10420000CE0101960E941559BE016B5E7F4FCE0113
:1042100001960E942258BC0188E693E10E94415811
:10422000CE0101960E94D158CE0145960E94D158E8
:1042300010927C0D10927B0D80E090E00E94048132
:10424000FCC261E779E0C8010E941559B80180E815
:1042500093E10E942654811116C068E779E0CE01EF
:1042600001960E941559BE016F5F7F4F80E893E170
:104270000E94265411E0811101C010E0CE01019688
:104280000E94D15801C011E0CE0145960E94D1583C
:10429000112309F4CDC027E030E046E050E060E8AB
:1042A00073E1CE0101960E942959BE016F5F7F4FD5
:1042B00082E693E10E949758CE0101960E94D15860
:1042C00082E693E10E9433576093FF1180E893E107
:1042D0000E943E5782E693E10E94335761157105B3
:1042E0008105910519F485E090E007C06130710502
:1042F0008105910539F489E190E090930112809352
:10430000001226C067E67CE0CE0101960E94155996
:10431000BE016F5F7F4F80E893E10E94C353AC0101
:104320004F5F5F4F60E873E1CE0145960E94678260
:10433000CE0145960E94335770930112609300128C
:10434000CE0145960E94D158CE0101960E94D158C7
:1043500010927C0D10927B0D80E090E00E94048111
:104360006DEE73E088E693E10E9447588091FF115B
:10437000833034F56091001270910112CE014596A0
:104380000E941B726FE779E0CE0101960E941559D9
:10439000BE016B5E7F4FCE0101960E94225869E8F4
:1043A00076E00E940B58BC0188E693E10E944158D8
:1043B000CE0101960E94D158CE0145960E94D15857
:1043C0008091FF1183300CF438C26091001270911B
:1043D0000112CE0183960E941B726091FF11062E7E
:1043E000000C770BCE0145960E941B7268E679E0BF
:1043F000CE0101960E941559BE016B5E7F4FCE0122
:1044000001960E942258BE016D5D7F4F0E94225886
:10441000BC0188E693E10E944158CE0101960E94BA
:10442000D158CE0145960E94D158CE01839603C241
:104430006AE879E0CE0145960E941559BE016B5E8F
:104440007F4F80E893E10E942654811116C06EE8E8
:1044500079E0CE0101960E941559BE016F5F7F4F32
:1044600080E893E10E94265411E0811101C010E020
:10447000CE0101960E94D15801C011E0CE014596AF
:104480000E94D158112309F456C0809106029091E0
:1044900007020E9480666093A5047093A60480932F
:1044A000A7049093A8046093EB117093EC11809390
:1044B000ED119093EE1180E090E5A3ECB7E48093CA
:1044C000AD049093AE04A093AF04B093B004809376
:1044D000E3119093E411A093E511B093E61180915C
:1044E000CE0D882381F06FEC73E088E590E10E94A7
:1044F00081596091A5047091A6048091A7049091C0
:10450000A8040E94374F10927C0D10927B0D80E022
:1045100090E00E9404814091A5045091A60460910E
:10452000A7047091A80422E0CE0145960E94D658B7
:1045300062E979E06AC16DE979E0CE0145960E94B1
:104540001559BE016B5E7F4F80E893E10E942654AF
:10455000811116C061EA79E0CE0101960E941559D9
:10456000BE016F5F7F4F80E893E10E94265411E007
:10457000811101C010E0CE0101960E94D15801C006
:1045800011E0CE0145960E94D158112309F485C04F
:1045900080918413909185130497F8F044E050E0E3
:1045A00060E873E1CE0101960E946782BE016F5FF1
:1045B0007F4F82E693E10E949758CE0101960E94B8
:1045C000D15882E693E10E9428576093B10470931A
:1045D000B2048093B3049093B4048091B104909199
:1045E000B204A091B304B091B4048093DF1190930E
:1045F000E011A093E111B093E2118091CE0D8823D8
:1046000089F066EB73E088E590E10E948159609142
:10461000B1047091B2048091B3049091B40442E06B
:104620000E94C37D80910602909107020E948066DD
:104630006093A9047093AA048093AB049093AC0494
:104640006093E7117093E8118093E9119093EA1158
:104650008091CE0D882381F06CEA73E088E590E1CB
:104660000E9481596091A9047091AA048091AB04C1
:104670009091AC040E94374F10927C0D10927B0DEC
:1046800080E090E00E9404814091A9045091AA0426
:104690006091AB047091AC04B1C06DEA79E0CE01D9
:1046A00045960E941559BE016B5E7F4F80E893E1ED
:1046B0000E942654811116C061EB79E0CE0101966B
:1046C0000E941559BE016F5F7F4F80E893E10E9401
:1046D000265411E0811101C010E0CE0101960E9424
:1046E000D15801C011E0CE0145960E94D158112346
:1046F00009F4B3C080918413909185130497F8F066
:1047000044E050E060E873E1CE0101960E946782C8
:10471000BE016F5F7F4F82E693E10E949758CE0102
:1047200001960E94D15882E693E10E942857609337
:10473000AD047093AE048093AF049093B004809165
:10474000AD049091AE04A091AF04B091B0048093F9
:10475000E3119093E411A093E511B093E6118091D9
:10476000CE0D882389F063E973E088E590E10E942B
:1047700081596091AD047091AE048091AF04909125
:10478000B00442E00E94C37D80910602909107022E
:104790000E9480666093A5047093A6048093A7048A
:1047A0009093A8046093EB117093EC118093ED113A
:1047B0009093EE118091CE0D882381F069E873E02B
:1047C00088E590E10E9481596091A5047091A6044A
:1047D0008091A7049091A8040E94374F10927C0DFD
:1047E00010927B0D80E090E00E9404814091A5042E
:1047F0005091A6046091A7047091A80422E0CE0114
:1048000045960E94D65865EA79E0CE0101960E944D
:104810001559BE016B5E7F4FCE0101960E94225852
:10482000BC0188E693E10E948258CE0101960E9465
:10483000D158CE0145960E94D15868E673E1CE0169
:1048400001960E940D59CE0101960E941577CE0166
:1048500001960E94D1581092120280911202882370
:1048600071F060E873E1CE0101960E940D59CE010E
:1048700001960E945B73CE0101960E94D1580E945E
:104880007F936093240D7093250D8093260D909354
:10489000270D6FEC7CE080E893E10E946D5813C017
:1048A000CE0183960E941B7268E679E0CE014596A0
:1048B0000E941559BE016D5D7F4FCE0145960E9445
:1048C00022580C94A00BCA5BDF4F0FB6F894DEBFE2
:1048D0000FBECDBFDF91CF911F910F91FF90EF9051
:1048E000DF90CF90BF90AF909F908F907F906F9010
:1048F0005F904F903F9008952F923F924F925F921A
:104900006F927F928F929F92AF92BF92CF92DF92DF
:10491000EF92FF920F931F93CF93DF93CDB7DEB744
:10492000C554D1090FB6F894DEBF0FBECDBF8C01C0
:10493000C0904B0DD0904C0D8091CE0D882349F046
:1049400061E976E088E590E10E948159C8010E9402
:104950001973780125E0E20EF11C35E0E316F1044D
:1049600000F180914B0D90914C0D0817190709F13A
:104970000E94A4810E942F4510934C0D00934B0D73
:10498000B801CE0101960E941B72BE016F5F7F4F7E
:1049900084E793E10E949758CE0101960E94D15876
:1049A00008C00E3F4FEF140721F40E943F450C94BE
:1049B000E5376FEC7CE088E693E10E946D58F5E006
:1049C000EF16F10490F067E67CE0CE0101960E94BC
:1049D00015594AE050E06FEF7FEFCE0101960E943B
:1049E0002C74CE0101960E94D158F8017A96E633D4
:1049F000F10510F00C94F5368827EE58FF4F8F4FD5
:104A00000C9454AB0E94A48189E390E00E942A7721
:104A100020E030E04AE754E40E94DBA6AB01BC0191
:104A200021E0CE0101960E94D65865EB79E0CE01D7
:104A300080960E941559BE016F5F7F4FCE01809610
:104A40000E94225868EB79E00E940B58BC0188E66E
:104A500093E10E948258CE0180960E94D158CE01E7
:104A600001960E94D1586CEB79E082E693E10E94B6
:104A70006D5862E673E1CE0101960E940D594AE03D
:104A800050E068E070E0CE0101960E948773CE018D
:104A900001960E94D15868E673E1CE0101960E940A
:104AA0000D594AE050E06FEF7FEFCE0101960E9472
:104AB000D381CE0101960E94D15862E673E188E667
:104AC00093E10E9441588091830D882311F40C9446
:104AD00023370C94B630E090D204F090D3040E94B7
:104AE000A48189E390E00E942A770E9465A928EEBC
:104AF00033E0269FA001279F500D369F500D1124B3
:104B0000BA01CE0101960E941B7265EB79E0CE01DD
:104B100080960E941559BE016F5F7F4FCE0180962F
:104B20000E94225868EB79E00E940B58BC0188E68D
:104B300093E10E948258CE0180960E94D158CE0106
:104B400001960E94D158C7010E94BA77AB01BC01FF
:104B500023E0CE0101960E94D6586EEE79E0CE0198
:104B600080960E941559BE016F5F7F4FCE018096DF
:104B70000E9422586BEB76E00E940B58BC0188E63D
:104B800093E10E944158CE0180960E94D158CE01F7
:104B900001960E94D15864EC79E067CF8091830D33
:104BA000882309F42CC18EE19FE00E94746E61E0BD
:104BB00080918E040E94C19260E080918C040E94DA
:104BC000C1920E948A710E94D0440E94ED44AB01C0
:104BD000BC0123E0CE0180960E94D658BE01605EE3
:104BE0007F4FCE0101960E940D596BEE79E0CE0108
:104BF00001960E940B58BC0182E693E10E94825804
:104C0000CE0101960E94D158CE0180960E94D158C3
:104C10006EED7BE0CE0101960E94155962E673E1CC
:104C2000CE0101960E942258BC0188E693E10E94C1
:104C30008258CE0101960E94D1580E94ED446B012A
:104C40007C010E9422934B015C016EE170E080E0E8
:104C500090E00E9447930E94ED442B013C010E948A
:104C600022939B01AC01281939094A095B094901C2
:104C70005A0131ED831637E09306A104B1040CF418
:104C800041C0A7019601C301B2010E9405A86B01B2
:104C90007C0120E030E0A9010E94BBA918165CF459
:104CA00026EA3BE944EC5BE3C701B6010E9476A625
:104CB00087FF0BC027C026EA3BE944EC5BEBC7014A
:104CC000B6010E94BBA91816ECF0C501B40128EE8C
:104CD00033E040E050E00E94A8A7CA01B9010E9459
:104CE0007CA64B015C0120E030E04AE754E4C701B8
:104CF000B6010E94DBA6A50194010E94CCA8AB01DD
:104D0000BC0103C040E050E0BA0122E0CE01809631
:104D10000E94D658BE01605E7F4FCE0101960E9470
:104D20000D596DEC79E0CE0101960E940B58BC0143
:104D30008CE593E10E948258CE0101960E94D158E1
:104D4000CE0180960E94D15861ED79E0CE010196A6
:104D50000E9415596CE573E1CE0101960E9422581C
:104D6000BC0188E693E10E944158CE0101960E9461
:104D7000D15867E67CE0CE0101960E9415596CE59A
:104D800073E1CE0101960E942258BC0182E693E1B4
:104D90000E944158CE0101960E94D15863E974E007
:104DA000CE0101960E9405594AE050E060E070E0B3
:104DB000CE0101960E948773CE0101960E94D158C0
:104DC00062E673E1CE0101960E940D5945E050E084
:104DD0006FEF7FEFCE0101960E94D381CE01019645
:104DE0000E94D15865ED79E088E693E10E9433583E
:104DF00060E080918E040E94C1920C9423376091F0
:104E000013027091140280911502909116020E9473
:104E100023490C94233780910002909101020E9453
:104E2000224B0C9423374091020226964FAF2697CF
:104E300060E0842F0E94C1928091830D811109C08E
:104E400080915D1281110EC08FE090E0A0E0B0E093
:104E50000DC023E030E040E050E02CAF3DAF4EAF5E
:104E60005FAF08C083E090E0A0E0B0E08CAF9DAF02
:104E7000AEAFBFAF62EA74E088E693E10E944758A4
:104E800068E673E1CE0101960E940D594AE050E0B8
:104E90006FEF7FEFCE0101960E948773CE010196DE
:104EA0000E94D15821961FAE219725961FAE2597B7
:104EB000212C312CC12CD12C760182E3682E712C4F
:104EC000812C912C540126968FAD26970E94FD923D
:104ED000092E000CAA0BBB0B880E991EAA1EBB1E26
:104EE00065E070E080E090E00E94479391E0691AED
:104EF000710849F7409028055090290560902A05CF
:104F000070902B05C501B4010E947CA620E030E022
:104F100040EA50E40E94DBA620E030E040E85AE39B
:104F20000E94DBA620E030E048E452E40E94CCA8D6
:104F3000A30192010E9405A820E030E040E751E47F
:104F40000E94DBA64B015C01A30192016AE979E9A9
:104F500089E390E40E9405A89B01AC01C501B4015E
:104F60000E94CCA820E030E0A9010E9406A820E021
:104F700030E040E251E40E94DBA64B015C01219647
:104F80002FAD219725963FAD2597A1010E94BBA982
:104F900018163CF421968FAE219725969FAE259743
:104FA000150120E030E0A901B401C5010E9476A6F8
:104FB00087FF04C0812C912CA12CB12C22E0A401EC
:104FC000B501CE0180960E94D658BE01605E7F4F2B
:104FD000CE0101960E940D5968EE79E0CE0101964E
:104FE0000E940B58BC0182E693E10E948258CE01D8
:104FF00001960E94D158CE0180960E94D15862E657
:1050000073E1CE0101960E940D594AE050E060E044
:1050100070E0CE0101960E94D381CE0101960E94DC
:10502000D1580E947F938090280D9090290DA090D8
:105030002A0DB0902B0D24013501A4E64A0E511C17
:10504000611C711C461657066806790610F40C940C
:1050500044370E947F930E947AA62B013C01C50130
:10506000B4010E947CA620E030E048EC51E40E94AC
:1050700006A89B01AC01C301B2010E9476A687FF7E
:1050800002C00C9444376CE370E080E090E00E9432
:105090004793BFEFCB1ADB0AEB0AFB0A2CAD3DAD01
:1050A0004EAD5FAD2C153D054E055F050CF005CFEF
:1050B00064E670E080E090E00E9447930E94A48143
:1050C00064E670E080E090E00E9447936AE974E053
:1050D00082E693E10E94475862E673E1CE010196B1
:1050E0000E940D5944E150E060E070E0CE0101966D
:1050F0000E948773CE0101960E94D15822E021962A
:105100004FAD219725965FAD2597B101CE018096D1
:105110000E94D658BE01605E7F4FCE0101960E946C
:105120000D5968EE79E0CE0101960E940B58BC0142
:1051300082E693E10E948258CE0101960E94D158E6
:10514000CE0180960E94D15862E673E1CE010196AD
:105150000E940D5942E350E06FEF7FEFCE010196C0
:105160000E94D381CE0101960E94D15864E170E083
:1051700080E090E00E9447930E94C5816EE170E05C
:1051800080E090E00E9447936EE170E080E090E064
:105190000E9447936DEE79E0CE0101960E94155969
:1051A00062E673E1CE0101960E94225861EF79E038
:1051B0000E940B5868E673E10E942258BC0188E601
:1051C00093E10E9482580C943436809104029091AD
:1051D000050299270E948765BC01990F880B990BDE
:1051E0000E947CA62DE038E643E55BE30E94DBA647
:1051F0006B017C012091F6043091F7044091F80492
:105200005091F9040E9476A618164CF06091DE04C5
:105210007091DF048091E0049091E1041BC0209123
:105220000A0530910B0540910C0550910D05C70101
:10523000B6010E94BBA987FF05C0C701B6010E9445
:10524000C27F08C06091F2047091F3048091F4046D
:105250009091F50420E030E048EC52E40E94DBA697
:1052600020E030E048EA51E40E94DBA620912C05C2
:1052700030912D0540912E0550912F050E94CCA80C
:105280006B017C016FEA74E082E693E10E9447586B
:1052900062E673E1CE0101960E940D5942E350E0AF
:1052A00060E070E0CE0101960E948773CE01019606
:1052B0000E94D15822E0B701A601CE0101960E94BA
:1052C000D6586BEF79E0CE0180960E941559BE0149
:1052D0006F5F7F4FCE0180960E94225865EF79E084
:1052E0000E940B58BC0188E693E10E948258CE01CF
:1052F00080960E94D158CE0101960E94D15868E64E
:1053000073E1CE0101960E940D5942E350E06FEF28
:105310007FEFCE0101960E94D381CE0101960E94BB
:10532000D1588091830D882311F40C94233760E2C7
:1053300073E080E090E00E9447930C9423370E9432
:10534000A48163EE74E088E693E10E94475868E622
:1053500073E1CE0101960E940D594AE050E060E0F1
:1053600070E0CE0101960E948773CE0101960E94E3
:10537000D1586AED74E082E693E10E94475862E6F4
:1053800073E1CE0101960E940D5944E150E06FEFA8
:105390007FEFCE0101960E94D381CE0101960E943B
:1053A000D1588091300D9091310D8230910549F4A2
:1053B0000E94D59381111AC01092310D1092300DB8
:1053C00015C0892BC9F40E94D593882339F082E057
:1053D00090E09093310D8093300D08C00E94D593DA
:1053E0008111F5CF0E94D5938111F1CF8091300DBD
:1053F0009091310D029741F16EEC74E088E693E1F3
:105400000E94475868E673E1CE0101960E940D594B
:105410004AE050E060E070E0CE0101960E948773A0
:10542000CE0101960E94D15868E673E1CE01019643
:105430000E940D5967E67CE0CE0101960E940B5850
:1054400062E673E10C9490338AE090E00E946B4531
:105450006B017C0120E030E0A9010E9476A61816BD
:1054600034F08AE090E00E946B456B017C01BBE068
:10547000AB2EB12C20E030E042ED53E4C701B60181
:105480000E9476A618168CF031E0A31AB10869F0D4
:1054900068EC70E080E090E00E94479383E090E049
:1054A0000E946B456B017C01E5CF20E030E0A90153
:1054B000C701B6010E9476A618163CF060EC74E0B5
:1054C00088E693E10E94475831C020E030E048EC84
:1054D00052E4C701B6010E9476A687FF02C021E010
:1054E00001C020E0B701A601CE0101960E94D65866
:1054F0006AEF79E0CE0180960E941559BE016F5F78
:105500007F4FCE0180960E9422586FEF79E00E9473
:105510000B58BC0188E693E10E948258CE01809628
:105520000E94D158CE0101960E94D15868E673E1DD
:10553000CE0101960E940D5942E350E06FEF7FEFDC
:10554000CE0101960E94D381CE0101960E94D158CE
:1055500067EB74E082E693E10E94475862E673E1EC
:10556000CE0101960E940D5942E350E060E070E0E8
:10557000CE0101960E948773D0CE0E947F932B01AB
:105580003C018EE19FE00E94746E64E670E080E072
:1055900090E00E94479340E855E260E070E08EE1C1
:1055A0009FE00E94A18064E670E080E090E00E94AD
:1055B00047936CE175E082E693E10E94475862E60A
:1055C00073E1CE0101960E940D5942E350E06FEF66
:1055D0007FEFCE0101960E948773CE0101960E9453
:1055E000D15861E175E082E693E10E94475862E696
:1055F00073E1CE0101960E940D5942E350E06FEF36
:105600007FEFCE0101960E94D381CE0101960E94C8
:10561000D1588091510D9091520D8D7F1CAEA12CCF
:10562000B12CC12CD12CE12CF12C019709F46FC0C5
:10563000AE01405E5F4F59AF48AFCE014E969BAF73
:105640008AAF0E947F93DC01CB0184199509A609DA
:10565000B709883B9B40A105B10508F058C08EE111
:105660009FE00E949D54892B09F44AC02CED35E03F
:1056700040E050E02093220F3093230F4093240FFB
:105680005093250F0E946D8097FD06C082349105CE
:10569000C9F780E090E002C08FEF9FEF892B81F582
:1056A000AE014F5F5F4F1A014A010E946D8097FF64
:1056B00006C089818D3421F520E030E009C0D40195
:1056C0008D934D01E8ADF9ADEA17FB0771F7F1CF06
:1056D000D1018D911D01280F311DEAADFBADAE1733
:1056E000BF07B1F72E5B3F4F8E8D90E0982F882734
:1056F0004F8D840F911D2817390711F40C944837EA
:1057000062E370E080E090E00E9447939ACF0E94AD
:105710007F93DC01CB0184199509A609B709883B61
:105720009B40A105B10518F42CAD2111BDC00E940C
:10573000A48162E673E1CE0180960E940D5942E396
:1057400050E066E070E0CE0180960E948773CE0143
:1057500080960E94D1583CAD332311F40C946137EC
:1057600082E090E09093520D8093510DB501CE01EF
:1057700080960E941B72B601CE0186960E941B7213
:10578000B701CE01C2960E941B72BE016E5C7F4FB4
:10579000CE018C960E940D5962EF78E0CE018C9676
:1057A0000E940B58BE016A5D7F4F0E94225862EF33
:1057B00078E00E940B58BE01605E7F4F0E94225825
:1057C000BC0188E693E10E948258CE018C960E942B
:1057D000D158CE01C2960E94D158CE0186960E9421
:1057E000D158CE0180960E94D15868E673E1CE016F
:1057F00080960E940D594AE050E06FEF7FEFCE0196
:1058000080960E94D381CE0180960E94D1586BE091
:1058100075E083E694E10E948159B501CE0180963E
:105820000E941B72B601CE0186960E941B72B701C0
:10583000CE018C960E941B7263E07AE0CE01C29684
:105840000E941559BE01645D7F4FCE01C2960E9431
:10585000225867E67CE00E940B58BE016A5D7F4FCC
:105860000E94225867E67CE00E940B58BE01605EF1
:105870007F4F0E94225863E17AE00E940B58BC01DE
:1058800088E693E10E948258CE01C2960E94D158C8
:10589000CE018C960E94D158CE0186960E94D15896
:1058A000CE0180960E94D15862E370E080E090E0E3
:1058B0000E9447938EE19FE00E94746EFDC5E090C8
:1058C0000602F090070269E17AE082E693E10E9425
:1058D0006D580E94A48162E673E1CE0101960E9498
:1058E0000D594AE050E06FEF7FEFCE0101960E9424
:1058F0008773CE0101960E94D158C7010E9480662D
:1059000024966CAF7DAF8EAF9FAF24978090A90493
:105910009090AA04A090AB04B090AC04A5019401AF
:105920006091A5047091A6048091A7049091A804A9
:105930000E9405A82B013C0120E030E0A9010E9453
:1059400076A6882309F453C0C090B104D090B20465
:10595000E090B304F090B40420E030E0A901C70166
:10596000B6010E9476A618160CF041C08091AD04D5
:105970009091AE04A091AF04B091B0048CAF9DAFF4
:10598000AEAFBFAF9C01AD01C701B6010E9476A6C4
:10599000882369F1A70196016CAD7DAD8EAD9FADF9
:1059A0000E94CCA80E9401AA6CAF7DAF8EAF9FAFC2
:1059B000A501940124966CAD7DAD8EAD9FAD24976D
:1059C0000E9405A8A30192010E94CCA82CAD3DAD78
:1059D0004EAD5FAD0E94DBA60E9439A99B01AC01D0
:1059E000C701B6010E94DBA66B017C0103C0C12C7C
:1059F000D12C760162E673E1CE0101960E940D5929
:105A00004AE050E060E070E0CE0101960E948773AA
:105A1000CE0101960E94D15820E030E64AEE56E4CD
:105A2000C701B6010E94BBA918163CF468E275E0F4
:105A300088E693E10E94475825C021E0B701A601FE
:105A4000CE0180960E94D65863E27AE0CE0101969C
:105A50000E941559BE01605E7F4FCE0101960E94E3
:105A6000225867E27AE00E940B58BC0188E693E175
:105A70000E948258CE0101960E94D158CE01809694
:105A80000E94D15868E673E1CE0101960E940D593B
:105A90004AE050E06FEF7FEFCE0101960E94D38184
:105AA000CE0101960E94D15864E670E080E090E05B
:105AB0000E94479336CCE090D204F090D3040E9429
:105AC000A48165E070E080E090E00E944793C70108
:105AD0000E94BA77AB01BC0123E0CE0101960E947F
:105AE000D6586EEE79E0CE0180960E941559BE011F
:105AF0006F5F7F4FCE0180960E9422586BEB76E05D
:105B00000E940B58BC0188E693E10E948258CE01A6
:105B100080960E94D158CE0101960E94D1586BE226
:105B20007AE00C94352590914A0D81E08927809385
:105B30004A0D8091830D882331F068E673E181E896
:105B40009EE00E94987C68EC70E080E090E0F3CBEF
:105B50001092830D0C94233781E08093830D809302
:105B60006B1280916212882349F161E878E084E742
:105B700093E10E946D5886EE9FEF90934C0D8093B9
:105B80004B0D2091651230916612809167129091B1
:105B900068128217930724F010926812109267120D
:105BA0001092591210925A1210925B1210925C12BB
:105BB0006CE271E080E090E00E94479364E773E15B
:105BC0008AE793E10E94825880914B0D90914C0D91
:105BD0009093820D8093810D0C94233780917C14D7
:105BE000882321F010927C140C9423370E94B187F3
:105BF0000C9423378BEB9FE00E94746E40E052ECD4
:105C000061E070E08BEB9FE00E94A1808CED95E05D
:105C1000A0E0B0E08093BF0F9093C00FA093C10F9E
:105C2000B093C20F64E670E080E090E00E9447937A
:105C30008091300D9091310D019759F483E090E0FF
:105C40000E94E365811140C01092310D1092300D19
:105C50001AC081E090E00E94E365882339F081E07A
:105C600090E09093310D8093300D0DC083E090E073
:105C70000E94E3658111F3CF83E090E00E94E36529
:105C80008111EDCF06C08091300D9091310D0197BB
:105C9000D9F067E675E082E693E10E94475862E634
:105CA00073E1CE0101960E940D5944E150E06FEF7F
:105CB0007FEFCE0101960E94D381CE0101960E9412
:105CC000D1586BE575E0CEC06FE475E088E693E1EE
:105CD0000E94475868E673E1CE0101960E940D5973
:105CE000CE0101960E945B73CE0101960E94D158AD
:105CF00062E370E080E090E00E94479368E673E121
:105D0000CE0101960E940D5942E350E06FEF7FEF04
:105D1000CE0101960E948773CE0101960E94D15850
:105D200063E475E082E693E10E94475862E673E11E
:105D3000CE0101960E940D5944E150E06FEF7FEFD4
:105D4000CE0101960E94D381CE0101960E94D158C6
:105D50008BEB88A38AEA89A381E08AA3212C312CCA
:105D6000C12CD12C412C512C3201C6016AE070E0CB
:105D70000E9441AB892B49F443E050E0BE01605ED4
:105D80007F4F8BEB9FE00E94425465E070E080E023
:105D900090E00E944793BFEFCB1ADB0AE12CF12C75
:105DA000812C912C54018BEB9FE00E949D54892BF8
:105DB00081F4E4E08E169104A104B10454F094E05F
:105DC000291631046CF4A0E9CA16A1E0DA0669F6D6
:105DD00007C0F6E0EF16F10414F40C948D37EFCF02
:105DE000C301B2010E947CA620E030E040E251E411
:105DF0000E94CCA820E030E040E85EE30E94DBA6F1
:105E00006B017C0120E030E040EA51E40E94BBA934
:105E1000181634F521E0B701A601CE0101960E94C3
:105E2000D6586BED77E0CE0180960E941559BE01E1
:105E30006F5F7F4FCE0180960E94225863E37AE025
:105E40000E940B58BC0188E693E10E948258CE0163
:105E500080960E94D158CE0101960E94D15806C06A
:105E600067E375E088E693E10E94475868E673E1CE
:105E7000CE0101960E940D594AE050E060E070E0CA
:105E8000CE0101960E948773CE0101960E94D158DF
:105E900068E673E1CE0101960E940D5967E67CE049
:105EA000CE0101960E940B5862E673E10E942258CF
:105EB000BC0188E693E10E948258CE0101960E94BF
:105EC000D1588BEB9FE00E94746E2BCA62E076E0A3
:105ED000CE0101960E9405594AE050E06FEF7FEF36
:105EE000CE0101960E94D381CE0101960E94D15825
:105EF0006091D0047091D10480912605909127057E
:105F00000E94E574E4E18E2E912CA12CB12CC12CC1
:105F1000D12CAFEFCA1ADA0AC501B4010E94479327
:105F20006091D0047091D10480912605909127054D
:105F30000E94E5747C01B3E0CB16D10434F08EE10D
:105F4000C816D10444F4EF2851F094E1890E911C55
:105F5000A11CB11CDECFE114F10409F00CC1809149
:105F60002605909127058B309105C9F48091C013C7
:105F70009091C113A091C213B091C3138093E00D0F
:105F80009093E10DA093E20DB093E30D8091BC13CB
:105F90009091BD13A091BE13B091BF131DC0863167
:105FA000910521F30C9701F58091D30D9091D40DBB
:105FB000A091D50DB091D60D8093E00D9093E10D99
:105FC000A093E20DB093E30D8091CF0D9091D00D91
:105FD000A091D10DB091D20D8093DC0D9093DD0D89
:105FE000A093DE0DB093DF0D4091E00D5091E10DD7
:105FF0006091E20D7091E30D21E0CE0101960E94C7
:10600000D65860EF7BE0CE0180960E941559BE0104
:106010006F5F7F4FCE0180960E942258BC0188E6B8
:1060200093E10E948258CE0180960E94D158CE0101
:1060300001960E94D1584091DC0D5091DD0D609188
:10604000DE0D7091DF0D21E0CE0101960E94D65841
:1060500066E37AE0CE0180960E941559BE016F5F1B
:106060007F4FCE0180960E942258BC0188E693E1C2
:106070000E944158CE0180960E94D158CE010196CF
:106080000E94D15868EF79E088E693E10E94335886
:106090006FEC7CE0CE0101960E94155944E150E07E
:1060A00060E070E0CE0101960E948773CE010196F8
:1060B0000E94D158C090E00DD090E10DE090E20D2B
:1060C000F090E30D20E030E0A901C701B6010E9485
:1060D000BBA920E030E040E05FE387FD05C0C701D9
:1060E000B6010E9406A804C0C701B6010E9405A817
:1060F0000E9465A9AB01BC01CE0101960E94527DB0
:10610000BE016F5F7F4F82E693E10E949758CE01F8
:1061100001960E94D15860E087E00E94277D62E6E8
:1061200073E183E694E10E9473596FED83E694E195
:106130000E946C596CE37AE083E694E10E944C5A29
:106140006091DC0D7091DD0D8091DE0D9091DF0D81
:106150000E9465A94AE050E083E694E10E94025A59
:1061600068EF79E083E694E10E944C5A64E670E0BF
:1061700080E090E0E0C8EFEFEE16FE06ACF064EFD2
:1061800075E0CE0101960E9405594AE050E060E0BA
:1061900070E0CE0101960E948773CE0101960E94A5
:1061A000D15861ED75E048C0FEEFEF16FFEFFF0636
:1061B00079F163EC75E0CE0101960E9405594AE041
:1061C00050E060E070E0CE0101960E948773CE013E
:1061D00001960E94D15864EB75E088E693E10E9435
:1061E0004758B701CE0101960E941B72BE016F5F36
:1061F0007F4F88E693E10E944158CE0101960E94AC
:10620000D1586EE975E088E693E10E94AF571BC64E
:1062100063E975E0CE0101960E9405594AE050E01D
:1062200060E070E0CE0101960E948773CE01019676
:106230000E94D15863E775E088E693E10E944758D1
:1062400002C680919004882309F4FDC56FEC7CE0C0
:10625000CE0101960E9415594AE050E061E070E0DD
:10626000CE0101960E948773CE0101960E94D158FB
:106270000E947E90E8C58091830D81110AC08091B3
:106280005D12811106C07EE1472E512C612C712CCC
:1062900005C063E0462E512C612C712C60E176E044
:1062A00088E693E10E94475868E673E1CE010196C3
:1062B0000E940D594AE050E06FEF7FEFCE0101964A
:1062C0000E94D381CE0101960E94D158812C912C3D
:1062D00054011CAE1DAE1EAE1FAE83E20E940C7DAB
:1062E00087E090E00E94077D0E94057D66E970E0EE
:1062F00080E090E00E94479383E20E940C7D80E260
:1063000090E00E94077D0E94057D66E970E080E0D4
:1063100090E00E94479362E070E083E290E00E9488
:10632000526FC12CD12C76018091A80D90E0209164
:10633000A90D821B9109181619066CF485EF90E1DE
:106340000E948B8BFE2CED2CDC2CCC24C80ED11C97
:10635000E11CF11CE9CFC701B6010E947CA62AE925
:1063600039E949E95FE30E94CCA80E9465A9AB0125
:10637000BC0184169506A606B70614F44A015B0113
:10638000CE0180960E94527DBE01605E7F4FCE019D
:1063900001960E940D596FE37AE0CE0101960E94AA
:1063A0000B58BC0182E693E10E948258CE0101960F
:1063B0000E94D158CE0180960E94D15862E673E1C6
:1063C000CE0101960E940D594EE150E060E070E070
:1063D000CE0101960E942C74CE0101960E94D158E4
:1063E0002CAD3DAD4EAD5FAD2F5F3F4F4F4F5F4F7B
:1063F0002CAF3DAF4EAF5FAF421653066406750635
:106400000CF06BCFB501A401CE0180960E94527DA5
:10641000BE01605E7F4FCE0101960E940D596FE371
:106420007AE0CE0101960E940B58BC0182E693E10E
:106430000E948258CE0101960E94D158CE018096CA
:106440000E94D15862E673E1CE0101960E940D5977
:106450004AE050E060E070E0CE0101960E94877350
:10646000CE0101960E94D158B501A401CE0101963A
:106470000E94527D63E47AE0CE0180960E94155915
:10648000BE016F5F7F4FCE0180960E94225866E466
:106490007AE00E940B5868E673E10E942258BC0122
:1064A00088E693E10E948258CE0180960E94D158DE
:1064B000CE0101960E94D15862E370E080E090E046
:1064C0000C949B29E090CE04F090CF0481E080935F
:1064D000300564E670E080E090E00E9447930E94FF
:1064E000A481C7010E94876560E074E0681B790B96
:1064F000CE0101960E941B726BE47AE0CE01809679
:106500000E941559BE016F5F7F4FCE0180960E9499
:106510002258BC0188E693E10E948258CE01809601
:106520000E94D158CE0101960E94D15860E087E0C8
:106530000E94277D60E276E0CE0101960E94055917
:1065400042E350E068E070E0CE0101960E9487735C
:10655000CE0101960E94D15868E673E1CE01019602
:106560000E940D5942E350E06FEF7FEFCE0101969C
:106570000E94D381CE0101960E94D15862E57AE053
:10658000C7C08091CC049091CD040E9487657C01A6
:106590009093330D8093320D62E370E080E090E0E1
:1065A0000E944793B701CE0101960E941B72BE0163
:1065B0006F5F7F4F88E693E10E949758CE01019666
:1065C0000E94D1588091BA139091BB13892B09F482
:1065D0005EC066EB73E1CE0180960E940D59BE014C
:1065E000605E7F4FCE0101960E940D5944E150E05C
:1065F00060E070E0CE0101960E948773CE010196A3
:106600000E94D1586CE57AE0CE0101960E9415599E
:1066100068E673E1CE0101960E942258BC0182E631
:1066200093E10E948258CE0101960E94D15862E601
:1066300073E1CE0101960E940D5944E150E06FEFE5
:106640007FEFCE0101960E94D381CE0101960E9478
:10665000D158BE01605E7F4FCE0101960E940D5958
:1066600067E67CE0CE0101960E940B5862E673E17A
:106670000E942258BC0188E693E10E948258CE0114
:1066800001960E94D158CE0180960C948F2967E61E
:106690007AE082E693E10E946D5862E673E1CE01F2
:1066A00001960E940D5944E150E060E070E0CE0197
:1066B00001960E948773CE0101960E94D1586BE427
:1066C0007AE0CE0101960E94155968E673E1CE0189
:1066D00001960E942258BC0182E693E10E948258F2
:1066E000CE0101960E94D15862E673E1CE01019677
:1066F0000E940D5944E150E06FEF7FEFCE0101960B
:106700000E94D381CE0101960E94D1586CE57AE0B7
:10671000CE0101960E94155968E673E1CE010196FB
:106720000E942258BC0188E693E10E948258CE0163
:1067300001960E94D1580C9491298091900488234D
:1067400009F481C38091830D811104C080915D1291
:10675000882329F082E090E00E94738274C3C09085
:106760001302D0901402E0901502F090160220E07F
:1067700030E040E450E4C701B6010E94BBA91816FE
:106780006CF420E030E04AEF54E4C701B6010E9407
:10679000DBA60E9465A96B017C0106C040E3C42E04
:1067A00045E7D42EE12CF12C0E94A48160E080E02A
:1067B0000E94277D61E376E083E694E10E9481599F
:1067C00061E080E00E94277D69E276E083E694E163
:1067D0000E94815964E670E080E090E00E94479357
:1067E0000E947F9360932C0D70932D0D80932E0D3E
:1067F00090932F0D0E947F9380902C0D90902D0DE3
:10680000A0902E0DB0902F0DDC01CB0188199909B5
:10681000AA09BB098C159D05AE05BF050CF013C375
:1068200083E090E00E9473820E947F9364E170E0B5
:1068300080E090E00E944793DDCF0E94A76681E848
:106840009EE00E943B55FFC261E576E082E693E15F
:106850000E94475862E673E1CE0101960E940D59ED
:106860004AE050E060E070E0CE0101960E9487733C
:10687000CE0101960E94D158309110023CAF809118
:10688000420D811105C00E947F9381E08093420DEB
:1068900080913A0D811105C00E947F9381E0809321
:1068A0003A0D1092390D1092380D2090380D30901D
:1068B000390D48E2241631040CF07CC08CAD0E94E6
:1068C000FD92F101EE0FFF1FE951F24F918380839A
:1068D0000E949D7E20E030E040EA50E40E94DBA66A
:1068E00020E030E040E85AE30E94DBA62B013C01A7
:1068F00080900C0290900D02A0900E02B0900F02BA
:10690000A5019401609108027091090280910A0228
:1069100090910B020E9405A89B01AC0160E070E021
:1069200080EC90E40E9405A86B017C0120E030E03F
:10693000A9010E9476A620E030E040E650E48111F3
:1069400005C0C301B2010E94DBA61EC0C301B20193
:106950000E94DBA6A50194010E9406A820E030E079
:1069600040E850E40E9405A8A70196010E94CCA827
:1069700020E030E040EC50E40E94DBA620E030E074
:1069800040E850E40E9406A86093340D7093350DE2
:106990008093360D9093370D64E170E080E090E0D5
:1069A0000E9447935FEF251A350A3092390D2092E5
:1069B000380D7BCFC090340DD090350DE090360D62
:1069C000F090370D20E030E0A901C701B6010E9428
:1069D000BBA987FD1EC022E0B701A601CE0101962A
:1069E0000E94D6586BE67AE0CE0180960E94155937
:1069F000BE016F5F7F4FCE0180960E942258BC017E
:106A000088E693E10E948258CE0180960E94D15878
:106A100004C262E476E088E693E10E94475801C22E
:106A200080919004882309F40EC28091830D811116
:106A30002BC080915D12811127C0C0901302D090AD
:106A40001402E0901502F090160220E030E04AE7D0
:106A500054E4C701B6010E94DBA60E9465A94B0160
:106A60005C0120E030E040EA50E4C701B6010E943A
:106A7000DBA620E030E040EA50E40E9406A80E9435
:106A800065A9A501940108C021E030E040E050E094
:106A90006AE070E080E090E00E94F369D4C18091E8
:106AA000491290914A120097F1F581E090E090939D
:106AB0004A12809349126FE67AE0CE0101960E9455
:106AC0001559CE0101960E945B73CE0101960E947A
:106AD000D15868E77AE0CE0101960E94155967E522
:106AE00074E1CE0101960E942258BC01CE0180962D
:106AF0000E940D5948EC50E06FEF7FEFCE01809679
:106B00000E948773CE0180960E94D158CE010196D3
:106B10000E94D15881E89EE00E94746E40E052ECE1
:106B200061E070E078C0029799F510924A121092D5
:106B300049126EE77AE0CE0101960E941559CE0106
:106B400001960E945B73CE0101960E94D1586CE8B9
:106B50007AE0CE0101960E94155967E574E1CE01F5
:106B600001960E942258BC01CE0180960E940D59C8
:106B700048EC50E06FEF7FEFCE0180960E94877364
:106B8000CE0180960E94D158CE0101960E94D15824
:106B90008091491290914A120197A9F582E090E004
:106BA00090934A128093491260E97AE0CE010196EF
:106BB0000E941559CE0101960E945B73CE01019689
:106BC0000E94D15861EA7AE0CE0101960E941559DF
:106BD00067E574E1CE0101960E942258BC01CE0106
:106BE00080960E940D5948EC50E06FEF7FEFCE0188
:106BF00080960E948773CE0180960E94D158CE0164
:106C000001960E94D15881E89EE00E94746E40E88F
:106C100055E260E070E081E89EE00E94A180109261
:106C20007C0D10927B0D80E090E00E94048166EA6A
:106C30007AE0CE0101960E94155961E574E1CE011A
:106C400001960E942258BC01CE0180960E940D59E7
:106C500040ED57E06FEF7FEFCE0180960E94D38129
:106C6000CE0180960E94D158CE0101960E94D15843
:106C7000EAC08091E50D9091E60D892BA1F481E0A9
:106C800090E09093E60D8093E50D8EED93E0909368
:106C90007C0D80937B0D0E942D8168EC70E080E07C
:106CA00090E00E944793E0E0F0E01995CCC00E948C
:106CB00093940E94A4810E942F45C5C090916212B6
:106CC00081E0892780936212882369F16AE876E07F
:106CD00088E693E10E9447580E947F93609359127F
:106CE00070935A1280935B1290935C12809165129C
:106CF00090916612181619065CF420916712309173
:106D000068122817390724F010926812109267123F
:106D1000909169128091641298175CF01092691238
:106D200010926A1206C062E876E088E693E10E945B
:106D300047588091621280935D1268E673E1CE013C
:106D400001960E940D594AE050E068E070E0CE01E3
:106D500001960E948773CE0101960E94D15865E783
:106D600076E0CE0101960E9405594AE050E06FEFAF
:106D70007FEFCE0101960E94D381CE0101960E9441
:106D8000D15867E676E088E693E10E94AF5765E563
:106D90007CE0CE0101960E94155968E673E1CE01B0
:106DA00001960E942258BC0188E693E10E94825815
:106DB000CE0101960E94D1588091830D80936B1271
:106DC0008CE291E00E9451818091830D8823D9F15A
:106DD00061E878E084E793E10E946D5886EE9FEFCA
:106DE00090934C0D80934B0D2EC0D0924C0DC092C1
:106DF0004B0D6AE576E088E693E10E9447586FEC18
:106E00007CE0CE0101960E9415594AE050E060E016
:106E100070E0CE0101960E948773CE0101960E9418
:106E2000D15868E673E1CE0101960E940D594AE0FF
:106E300050E06FEF7FEFCE0101960E94D381CE012B
:106E400001960E94D15880916C1390916D13009718
:106E5000A1F0419720F4023011050CF0A3C068E6C0
:106E600073E1CE0101960E940D59CE0101960E9458
:106E70001577CE0101960E94D15864E670E080E05B
:106E800090E00E944793A1C00E94C5810C944328C2
:106E9000EC80F12CFE2CEE248D81E80EF11CCE80CE
:106EA000D12CDC2CCC248F81C80ED11CA884B12C11
:106EB000BA2CAA248985A80EB11C21E02CAF0C9411
:106EC000802B60E075E088E693E10E94475868E611
:106ED00073E1CE0180960E940D594AE050E060E0D7
:106EE00070E0CE0180960E94D381CE0180960E94F0
:106EF000D1586DEE74E088E693E10E944758809186
:106F0000510D9091520D029711F00C94542C109247
:106F1000520D1092510D0C94542C8BEB9FE00E945B
:106F20009D54892B71F08BEB9FE00E947B54E1E034
:106F3000F0E0EC0FFD1FEE0DFF1D80832FEFE21A36
:106F4000F20A65E070E080E090E00E94479336E04E
:106F5000E316F10401F5998188A198131CC09A8168
:106F600089A1981318C09B818AA1981314C08D81A0
:106F700090E0A0E0B0E0BA2FA92F982F88272C81AD
:106F8000820F911DA11DB11D480E591E6A1E7B1E48
:106F90004FEF241A340A5FEF851A950AA50AB50A3D
:106FA0000C94D32E68E673E1CE0101960E940D5930
:106FB0004AE050E06FEF7FEFCE0101960E94D3814F
:106FC000CE0101960E94D1584ACFCB5BDF4F0FB65E
:106FD000F894DEBF0FBECDBFDF91CF911F910F910F
:106FE000FF90EF90DF90CF90BF90AF909F908F90E9
:106FF0007F906F905F904F903F902F9008952F92C9
:107000003F924F925F926F927F928F929F92AF9238
:10701000BF92CF92DF92EF92FF920F931F93CF9385
:10702000DF93CDB7DEB728970FB6F894DEBF0FBE5B
:10703000CDBFFC0187E091E19387828780910411A5
:1070400090E0958784878091D11190E0978786871B
:1070500080910111853009F063C6809109119091EA
:107060000A11885891098D35910588F48091041191
:10707000843041F480910B1190910C1180974797C7
:1070800008F47DC080910411843408F05EC08091C2
:1070900004118A3108F4D5C080910711909108112C
:1070A000843F914050F4118610868FEF9FEFDC01F2
:1070B00084839583A683B7833CC080910911909106
:1070C0000A1185974B9708F0BCC00DE0E02E01E156
:1070D000F02E82E090E040E050E0BA018C010F5FBA
:1070E0001F4F2091041130E0021713076CF4970131
:1070F00022503109D9012D913C9127503109273077
:10710000310508F47FC0C80101979595879591874F
:1071100080870C971CF41186108693C04483558396
:107120006683778384E090E00DC044835583668353
:1071300077838BE090E006C0448355836683778332
:107140008CE090E0918380831EC580910B1190911B
:107150000C11825491098E9708F099CF20E030E00D
:10716000C12CD12C7601A901435F5E4EDA014D910D
:107170005C91495051094930510598F088CF809170
:107180000D1190910E110997099708F07BCF118688
:1071900010868FEF9FEFDC0184839583A683B783EE
:1071A000C2C5B901615F7E4EDB014D915C914751D3
:1071B000510942315105C0F4D701C601880F991F0A
:1071C000AA1FBB1F6C017D016894C0F82C5F3F4F64
:1071D0002038310541F620E230E031872087C48233
:1071E000D582E682F7829FC5DB014D915C914650C6
:1071F00051094730510508F04ACFCC0CDD1CEE1C7C
:10720000FF1CE4CFD7012D913C91235131092F3040
:10721000310550F4440F551F661F771F41600296D9
:10722000B4E0EB0EF11C5ACFD7012D913C912A50BE
:1072300031092930310528F4440F551F661F771F87
:10724000EECF809104118A3108F460C0809107115B
:10725000909108118032934008F425CF8091091154
:1072600090910A11C697869708F050C080910B1133
:1072700090910C11C697869708F048C0BFE0EB2E9E
:10728000B1E1FB2E83E090E040E050E0BA018C01D8
:107290000F5F1F4F2091041130E00217130764F4B1
:1072A000970122503109D9012D913C912C5031097F
:1072B0002B30310560F0C80101979595879591872E
:1072C00080870C970CF031CF118610861FC0D70134
:1072D0002D913C91255231092B31310550F4440F49
:1072E000551F661F771F41600296B4E0EB0EF11C3C
:1072F000CECFD7012D913C912C5031092A30310548
:1073000028F4440F551F661F771FEECF809104119C
:10731000823208F452C08091091190910A110697A7
:10732000079708F04AC04DE0C42E41E1D42E82E018
:1073300090E040E050E0BA018C010F5F1F4F2091B8
:10734000041130E002171307F4F4D6011297ED9000
:10735000FC9011979D01BEE1EB1AF108A7E1EA1636
:10736000F104E0F4440F551F661F771F4160D601FA
:107370002D913C91B4E0CB0ED11C23503109253026
:107380003105C8F0C8010197959587959187808749
:1073900040970CF0D1CE118610860FC0D9012D91E7
:1073A0003C912C5031092B30310538F4440F551FD6
:1073B000661F771FDCCF0296BFCF7F011C821B8226
:1073C00081E090E09A838983809104118D3070F47C
:1073D0001C821B8281E090E09A838983F701848577
:1073E0009585181619060CF474C0D1C029E733E04E
:1073F000AE014D5F5F4FBE016F5F7F4FC7010E94BF
:10740000F894892B29F729E733E0AE014D5F5F4FF0
:10741000BE016F5F7F4FC7010E94F8940197C1F6CC
:1074200029E733E0AE014D5F5F4FBE016F5F7F4FD5
:10743000C7010E94F894892B59F6812C912C540194
:1074400000E010E08091041190E029813A81281732
:10745000390794F529E733E0AE014D5F5F4FBE0178
:107460006F5F7F4FC7010E94F8946C0129E733E0FA
:10747000AE014D5F5F4FBE016F5F7F4FC7010E943E
:10748000F894F1E0CF16D10451F4892B09F0A0CF84
:10749000880C991CAA1CBB1C689480F80AC0CD28D3
:1074A00009F096CF019709F093CF880C991CAA1C7C
:1074B000BB1C0F5F1F4FC6CFD70119961C930E93AD
:1074C0001897F70184829582A682B78281E090E0C6
:1074D00039CE0284F385E02D82E090E09A8389839F
:1074E0008281938189974E9708F051C083E090E0A4
:1074F0009A838983848195810B970A9708F047C006
:107500002CEB31E0AE014D5F5F4FBE016F5F7F4FEF
:10751000C7010E94F894892BD1F52CEB31E0AE0124
:107520004D5F5F4FBE016F5F7F4FC7010E94F894B0
:10753000019769F5412C512C320100E010E0F70170
:107540002485358589819A81821793070CF02FC194
:107550002CEB31E0AE014D5F5F4FBE016F5F7F4F9F
:10756000C7010E94F8945C010330110509F0E5C0E1
:107570002CEB31E0AE014D5F5F4FBE016F5F7F4F7F
:10758000C7010E94F894A816B90609F4D6C0D7011D
:107590001A96ED91FC911B9782819381C6978697ED
:1075A000E0F4848195814B974597B8F4DF011696F6
:1075B0006F0126ECC20ED11C20E030E040E050E02C
:1075C00060E070E080E090E00D911C91119709500F
:1075D00011090830110508F4F4C0809104118933B1
:1075E00070F182819381895791098335910508F45F
:1075F0001BC125C0D90112966D917C9113976651DC
:1076000071096131710508F037C1D501C401880FD6
:10761000991FAA1FBB1F4C015D01689480F84E5F43
:107620005F4F2C5F3F4F4B33510509F40CC1D9011B
:107630006D917C916A50710969307105D8F2809121
:107640000411823231F4828193810A97099708F4F8
:1076500023C1828193818957910983359105D0F4A3
:10766000809104118132B0F084819581CA97899705
:1076700088F49F012A5F3F4F812C912C540143E0F5
:1076800050E0D9016D917C916A50710969307105A2
:1076900008F41EC1828193818C549109C59778F4B6
:1076A00080910411843031F48481958180974797CB
:1076B00008F46CC180910411843408F04EC18091AB
:1076C0000411863460F1828193810C970B9708F442
:1076D000A9C125C0D90112966D917C9113976E5165
:1076E00071096731710508F0D1C1D501C401880F56
:1076F000991FAA1FBB1F4C015D01689480F84E5F63
:107700005F4F2C5F3F4F4534510509F4A6C1D901A5
:107710006D917C916C5071096B307105D8F280913C
:107720000411883508F4E4C1828193818558910958
:107730008B35910508F4BAC1DBC12CEB31E0AE0109
:107740004D5F5F4FBE016F5F7F4FC7010E94F8948E
:107750006C010330110579F42CEB31E0AE014D5F83
:107760005F4FBE016F5F7F4FC7010E94F894C8163C
:10777000D90609F00CCFA114B10459F4CA94CD284C
:1077800009F005CF440C551C661C771C689440F822
:107790000BC0AA94AB2809F0FACECD2809F0F7CE99
:1077A000440C551C661C771C0F5F1F4FC8CE1187F9
:1077B0000087F701448255826682778282E090E0FA
:1077C000C1CC12960D911C911397015111090D30E6
:1077D0001105E0F401E00E945CAB21601496AC1549
:1077E000BD0509F0F1CEF701248335834683578325
:1077F00000E20E9477AB2283338385E090E091839F
:10780000808380E390E091878087BDC112960D91BF
:107810001C911397045011090530110508F0DDCEB5
:1078200001E00E945CABDACF84819581CA97899789
:1078300008F005CF9F012A5F3F4F812C912C540106
:1078400043E050E0F4CE9F012A583F4FD9012D91DB
:107850003C912A5031092930310508F0F0CE2CE155
:1078600030E0F70131872087D70184829582A68294
:10787000B7828AE090E085C1D90112966D917C9122
:107880001397665071096730710508F0D8CE880CDF
:10789000991CAA1CBB1CC3CE20910411CF01820FDE
:1078A000911D820F911DDC0112978D919C910A9779
:1078B000099708F0CECEF701118610868FEF9FEF63
:1078C000DC0184839583A683B78386E090E03ACC7D
:1078D000D90112966D917C911397665171096131AE
:1078E000710558F5D501C401880F991FAA1FBB1F48
:1078F0004C015D01689480F84E5F5F4F2C5F3F4FF5
:107900004332510509F0BDCE9F012A5B3F4FD9019B
:107910002D913C912A5031092930310508F0BACE19
:1079200020E130E0F70131872087D70184829582FA
:10793000A682B78286E090E024C1D90112966D91AB
:107940007C911397665071096730710508F0A2CEDB
:10795000880C991CAA1CBB1CCFCF848195818954AB
:107960009109C39708F0ABCE9F012A5F3F4FAF014B
:107970004A575F4F812C912C5401D9016D917C9114
:107980006950710969307105B8F099CE8681978187
:107990000997099708F08ECED70119961C921E926E
:1079A00018978FEF9FEFDC01F70184839583A683FF
:1079B000B78387E090E0C6CBD90112966D917C9198
:1079C00013976651710961317105E0F4D501C40165
:1079D000880F991FAA1FBB1F4C015D01689480F896
:1079E0002C5F3F4F2417350741F620E230E0F701C6
:1079F00031872087D70184829582A682B78287E06B
:107A000090E0BFC0D90112966D917C91139766509A
:107A100071096730710508F052CE880C991CAA1CB8
:107A2000BB1CDECF848195810997099708F077CE3A
:107A3000868197818C974F9708F071CE80859185CC
:107A400089974D9708F06BCE9F01265F3F4F812CA1
:107A5000912C540145E050E05ACE9F0126573F4FEC
:107A6000D9012D913C912C5031092B30310508F072
:107A700056CE20E230E0F70131872087D70184829B
:107A80009582A682B78288E090E07BC0D9011296E9
:107A90006D917C911397695071096930710508F0F7
:107AA0003ECE880C991CAA1CBB1C29CE84819581D2
:107AB000825491098E97E0F48F01045C1F4F8DE191
:107AC00090E040E050E02091041130E02450310972
:107AD000821793070CF063C0980122503109D90135
:107AE0002D913C91295031092830310508F46EC0A0
:107AF00080910411803209F07EC0828193810697C3
:107B0000069708F078C0848195810997099708F055
:107B100072C09F012A5F3F4FAF01425C5F4F812CD3
:107B2000912C5401D9016D917C9166507109663098
:107B3000710508F060C0D90112966D917C91139780
:107B4000695171096331710508F0D5C0D501C401CF
:107B5000880F991FAA1FBB1F4C015D01689480F814
:107B60002C5F3F4F24173507E9F62EE030E0F70190
:107B700031872087D70184829582A682B7828FE0E1
:107B800090E08D939C9381E090E0D0C0D8012D913E
:107B90003C91285131092231310550F1CB01019737
:107BA00095958795D70119969C938E9318978A97E8
:107BB0000CF49ECF052E000C660B770BF701448367
:107BC00055836683778389E090E0BCCABC016F5F10
:107BD0007F4FD8012D913C91275031092730310535
:107BE000A8F6440F551F416002960C5F1F4F6BCFE4
:107BF000440F551FF9CFD7011C962D903C901D972F
:107C0000B6E02B1631040CF486C08F010E5F1F4FB7
:107C100075EC872E7DE9972E7CE1A72E71E8B72EB3
:107C2000E3E0CE2ED12CF8016481758160807180F3
:107C300080E090E00E947AA66D837E838F83988790
:107C4000B30180E090E00E947AA62B013C012DEC6C
:107C50003CEC4CE45FE30E94DBA69B01AC016D8130
:107C60007E818F8198850E9476A687FD19C02DECB4
:107C70003CEC4CE45FE36D817E818F8198850E94AE
:107C8000DBA69B01AC01C301B2010E9476A6E82FDE
:107C9000880FFF0BEE27FF0FEE1FFF27319602C064
:107CA000E0E0F0E0A501940163E971E080E091E09B
:107CB0000E941EAB4F01FF0FAA08BB08862697261D
:107CC000A826B926FFEFCF1ADF0A0E5F1F4F2C142C
:107CD0003D0409F0A8CFD70114968D929D92AD92E4
:107CE000BC92179780E290E019969C938E93189718
:107CF0008FEF9FEF46CFD90112966D917C9113972C
:107D0000695071096930710508F075CF880C991CAC
:107D1000AA1CBB1C25CF82E0809301111092041194
:107D200080E090E003C083E090E00CCA28960FB694
:107D3000F894DEBF0FBECDBFDF91CF911F910F91A1
:107D4000FF90EF90DF90CF90BF90AF909F908F907B
:107D50007F906F905F904F903F902F9008954F923B
:107D60005F926F927F929F92AF92BF92CF92DF927B
:107D7000EF92FF920F931F93CF93DF93CDB7DEB7B0
:107D8000A9970FB6F894DEBF0FBECDBF982E8823FB
:107D900051F08091CE0D882331F06FEC7CE088E5C6
:107DA00090E10E947F7D0E94E97160E08DE20E9477
:107DB000467360E18DE20E94467368E08DE20E94A6
:107DC00046734090CC135090CD136090CE137090BA
:107DD000CF13498E5A8E6B8E7C8EC090D013D0906C
:107DE000D113E090D213F090D313CD8EDE8EEF8EB0
:107DF000F8A28091D4139091D513A091D613B0918D
:107E0000D7138EA39FA3A8A7B9A789A39AA3ABA3AF
:107E1000BCA39920C9F18091CE0D8823A9F16DE40E
:107E20007BE0CE0101960E940559CE0101960E9489
:107E30005B73CE0101960E94D1588E01075E1F4FE1
:107E40005E0195E2A90EB11CD8016D917D918D91D5
:107E50009D918D0146E00E94C37D67E67CE088E548
:107E600090E10E944C5AA016B10671F76FEC7CE0CD
:107E7000CE0101960E941559CE0101960E945B73B6
:107E8000CE0101960E94D15823E938E144E85FE32E
:107E9000C301B2010E94DBA62B013C016D877E87E6
:107EA0008F87988B22E430E645E85FE3C701B6018F
:107EB0000E94DBA66B017C01698B7A8B8B8B9C8B80
:107EC00025E83BEE41E95FE36EA17FA188A599A576
:107ED0000E94DBA66D8B7E8B8F8B988F4092CC138C
:107EE0005092CD136092CE137092CF13C092D013E4
:107EF000D092D113E092D213F092D3136093D413A3
:107F00007093D5138093D6139093D713992009F4C7
:107F1000A0C08091CE0D882309F49BC060E47BE073
:107F2000CE0101960E940559CE0101960E945B7315
:107F3000CE0101960E94D1588E01035F1F4F6E0142
:107F4000B9E1CB0ED11C7801F80161917191819159
:107F500091918F0142E00E94C37D67E67CE088E555
:107F600090E10E944C5AC016D10671F76FEC7CE08C
:107F7000CE0101960E941559CE0101960E945B73B5
:107F8000CE0101960E94D15848ED53E166E070E0C1
:107F900082E30E94DF72A090D813B090D913C090F2
:107FA000DA13D090DB130091DC131091DD1363E33F
:107FB0007BE088E590E10E9481594AE050E0B501FC
:107FC00088E590E10E94025A67E67CE088E590E14E
:107FD0000E944C5A4AE050E0B60188E590E10E94C8
:107FE000025A67E67CE088E590E10E944C5A4AE03C
:107FF00050E0B80188E590E10E94025A6FEC7CE005
:1080000088E590E10E947F7DCE0101960E94464F57
:108010006AE27BE088E590E10E9481598E010F5F62
:108020001F4FD8016D917D918D919D918D014AE0F9
:108030000E94C37D67E67CE088E590E10E944C5A8F
:108040000E151F0571F76FEC7CE088E590E10E944A
:108050007F7D61E08DE10E9446739920B1F08091AF
:10806000CE0D882391F066E17BE088E590E10E94E7
:108070008159AE014B5D5F4F61E070E08DE10E9480
:10808000DF728DA190E00E94197362E08EE10E9480
:10809000467363E08FE10E94467364E080E20E94D1
:1080A0004673992009F450C08091CE0D882309F4BD
:1080B0004BC06AEF7AE088E590E10E948159AE01F9
:1080C0004B5D5F4F61E070E08EE10E94DF72CDA0FA
:1080D000D12CAE014B5D5F4F61E070E08FE10E94FB
:1080E000DF72EDA0F12CAE014B5D5F4F61E070E0FF
:1080F00080E20E94DF720DA110E04AE050E0B6017C
:1081000088E590E10E94025A67E67CE088E590E10C
:108110000E944C5A4AE050E0B70188E590E10E9485
:10812000025A67E67CE088E590E10E944C5A4AE0FA
:1081300050E0B80188E590E10E94025A6FEC7CE0C3
:1081400088E590E10E947F7D65E081E20E944673B0
:108150009920B1F08091CE0D882391F067EE7AE0FE
:1081600088E590E10E948159AE014B5D5F4F61E06F
:1081700070E081E20E94DF728DA190E00E9419738D
:1081800066E082E20E9446739920B1F08091CE0DA4
:10819000882391F06FEC7AE088E590E10E948159A4
:1081A000AE014B5D5F4F61E070E082E20E94DF72E2
:1081B0008DA190E00E94197367E083E20E944673EC
:1081C0009920B1F08091CE0D882391F069EB7AE08F
:1081D00088E590E10E948159AE014B5D5F4F61E0FF
:1081E00070E083E20E94DF728DA190E00E9419731B
:1081F00068E084E20E9446739920B1F08091CE0D30
:10820000882391F061EA7AE088E590E10E94815943
:10821000AE014B5D5F4F61E070E084E20E94DF726F
:108220008DA190E00E94197369E085E20E94467377
:108230009920B1F08091CE0D882391F067E87AE023
:1082400088E590E10E948159AE014B5D5F4F61E08E
:1082500070E085E20E94DF728DA190E00E941973A8
:108260006AE086E20E9446739920B1F08091CE0DBB
:10827000882391F061E77AE088E590E10E948159D6
:10828000AE014B5D5F4F61E070E086E20E94DF72FD
:108290008DA190E00E9419736BE088E20E94467302
:1082A0009920B1F08091CE0D882391F068E57AE0B5
:1082B00088E590E10E948159AE014B5D5F4F61E01E
:1082C00070E088E20E94DF728DA190E00E94197335
:1082D0006CE089E20E944673992009F479C080918C
:1082E000CE0D882309F474C060E47AE088E590E15B
:1082F0000E948159AE014B5D5F4F61E070E089E201
:108300000E94DF728DA190E00E94197369E27AE009
:1083100088E590E10E94815966E070E087E20E9462
:108320002C7390E00E94197362E17AE088E590E195
:108330000E94815965E070E087E20E942C7390E012
:108340000E9419736BEF79E088E590E10E948159F2
:1083500064E070E087E20E942C7390E00E94197341
:1083600062EE79E088E590E10E94815962E070E078
:1083700087E20E942C7390E00E94197369EC79E007
:1083800088E590E10E94815961E070E087E20E94F7
:108390002C7390E00E94197360EB79E088E590E11E
:1083A0000E94815960E070E087E20E942C7390E0A7
:1083B0000E9419736FE979E088E590E10E94815984
:1083C00063E070E087E20E942C7390E00E941973D2
:1083D00041E067E070E087E20E94EA4E41E063E03E
:1083E00070E087E20E94EA4E41E063E070E08AE2DA
:1083F0000E94EA4E992091F08091CE0D882371F071
:1084000066E879E088E590E10E94815963E070E0D8
:108410008AE20E942C7390E00E94197340E063E0AE
:1084200070E08AE20E94EA4E992091F08091CE0D90
:10843000882371F06CE679E088E590E10E9481592B
:1084400063E070E08AE20E942C7390E00E9419734E
:1084500041E062E070E08AE20E94EA4E992091F0E9
:108460008091CE0D882371F060E579E088E590E198
:108470000E94815962E070E08AE20E942C7390E0D1
:108480000E94197340E062E070E08AE20E94EA4EC6
:10849000992091F08091CE0D882371F063E379E00B
:1084A00088E590E10E94815962E070E08AE20E94D2
:1084B0002C7390E00E94197341E061E070E08AE261
:1084C0000E94EA4E992091F08091CE0D882371F0A0
:1084D00067E179E088E590E10E94815961E070E010
:1084E0008AE20E942C7390E00E94197340E061E0E0
:1084F00070E08AE20E94EA4E992091F08091CE0DC0
:10850000882371F06AEF78E088E590E10E94815954
:1085100061E070E08AE20E942C7390E00E9419737F
:1085200041E060E070E08AE20E94EA4E992091F01A
:108530008091CE0D882371F06EED78E088E590E1B2
:108540000E94815960E070E08AE20E942C7390E002
:108550000E94197340E060E070E08AE20E94EA4EF7
:10856000992091F08091CE0D882371F061EC78E034
:1085700088E590E10E94815960E070E08AE20E9403
:108580002C7390E00E94197341E066E070E087E28E
:108590000E94EA4E41E065E070E087E20E94EA4E08
:1085A00041E064E070E087E20E94EA4E40E062E071
:1085B00070E087E20E94EA4E40E061E070E087E20E
:1085C0000E94EA4E40E060E070E087E20E94EA4EDE
:1085D000992009F475C08091CE0D882309F470C0EC
:1085E00069EA78E088E590E10E94815966E070E0F0
:1085F0008BE20E942C7390E00E9419736BE878E084
:1086000088E590E10E94815965E070E08BE20E946C
:108610002C7390E00E9419736DE678E088E590E194
:108620000E94815964E070E08BE20E942C7390E01C
:108630000E94197364E578E088E590E10E94815911
:1086400062E070E08BE20E942C7390E00E9419734C
:108650006BE378E088E590E10E94815961E070E089
:108660008BE20E942C7390E00E94197362E278E022
:1086700088E590E10E94815960E070E08BE20E9401
:108680002C7390E00E9419736FE078E088E590E128
:108690000E94815963E070E08BE20E942C7390E0AD
:1086A0000E9419736AEF77E088E590E10E94815992
:1086B00064E070E08CE20E942C7390E00E941973D9
:1086C00040E064E070E08CE20E94EA4EAE014B5D57
:1086D0005F4F61E070E08CE20E94DF726DA1607F0D
:1086E00066608CE20E944673992009F45FC0809115
:1086F000CE0D882309F45AC066EE77E088E590E154
:108700000E948159AE014B5D5F4F61E070E08CE2E9
:108710000E94DF726DA16F7070E066507109072EC4
:10872000000C880B990B0E947CA69B01AC0160E0B9
:1087300070E080E090E40E9474AA20E030E048EC11
:1087400050E40E94DBA60E94374F6FEC77E088E58B
:1087500090E10E948159AE014B5D5F4F61E070E096
:1087600080E30E94DF726DA14AE050E088E590E16D
:108770000E941C4F67EB77E088E590E10E948159E9
:1087800061E070E080E30E942C7390E00E94197316
:108790006EE977E088E590E10E94815961E070E040
:1087A0008FE20E942C7390E00E94197341E061E017
:1087B00070E08FE20E94EA4E992091F08091CE0DF8
:1087C000882371F066E877E088E590E10E9481599E
:1087D00061E070E08EE20E942C7390E00E941973B9
:1087E00041E061E070E08EE20E94EA4E40E067E026
:1087F00070E081E30E94EA4E992009F455C080910F
:10880000CE0D882309F450C063E777E088E590E156
:108810000E94815967E070E081E30E942C7390E030
:108820000E94197364E97BE088E590E10E944C5A4C
:10883000AE014B5D5F4F61E070E080E00E94DF724F
:108840008DA10E94E58D6FEC7CE088E590E10E94AF
:108850007F7D0DE110E060ED7AE088E590E10E9417
:108860004C5A40E150E0B80188E590E10E94025A7C
:1088700068E97BE088E590E10E944C5AAE014B5DCF
:108880005F4F61E070E0802F0E94DF728DA10E9437
:10889000E58D6FEC7CE088E590E10E947F7D0F5FC5
:1088A0001F4F0A331105B9F6A9960FB6F894DEBF2B
:1088B0000FBECDBFDF91CF911F910F91FF90EF9031
:1088C000DF90CF90BF90AF909F907F906F905F9020
:1088D0004F9008950F931F9360E080918E040E9443
:1088E000939283E090E00197F1F761E080918E042C
:1088F0000E94939283E290E00197F1F760E080910B
:108900008E040E94939280918C0490918D049927FB
:10891000FC01E653FF4E6491FC01EC57FF4EE491DD
:10892000F0E0EE0FFF1FE659FF4E8591949100E4B1
:1089300012E42FE030E0462F0E946D95611571051D
:108940008105910549F0DC01CB010196A11DB11D06
:10895000BC01CD019F7003C060E070E0CB010E94BC
:108960007AA620E030E048EC52E40E94CCA82091A6
:108970007D0D30917E0D40917F0D5091800D0E94B4
:10898000DBA620E030E44CE156E40E94CCA820E0D5
:1089900030E040E05FE30E94DBA61F910F91089555
:1089A00023E333E948E853E40E94CCA820E030E018
:1089B00040E85FE30E9406A80E94C4AA26E636EAC1
:1089C00045EA53E40E94DBA660937D0D70937E0D13
:1089D00080937F0D9093800D0895CF92DF92EF9258
:1089E000FF9278DF6B017C0120E030E040E050E452
:1089F0000E94BBA918161CF46DDF6B017C0120E0FE
:108A000030E040E050E4C701B6010E94BBA918164F
:108A10001CF460DF6B017C0120E030E040E050E4BA
:108A2000C701B6010E94BBA918161CF453DF6B01E5
:108A30007C0120E030E040E050E4C701B6010E9434
:108A4000BBA918162CF4FF90EF90DF90CF9042CF87
:108A5000C701B601FF90EF90DF90CF90089581E0BD
:108A60008093DC048091DD04882341F088E08093CA
:108A70006E1460E083E694E10C94B88C08958091C4
:108A8000DD0481110FC081E08093DD048093DC045C
:108A900080916914982F9460909369148C600E945F
:108AA000167D18C08091DC048823A1F010926E140A
:108AB00060E083E694E10E94B88C1092DC0480911F
:108AC00069148B7F8093691488600E94167D1092D0
:108AD000DD040895C4CF2F923F924F925F926F9220
:108AE0007F928F929F92AF92BF92CF92DF92EF923E
:108AF000FF920F931F93CF93DF93CDB7DEB76697A7
:108B00000FB6F894DEBF0FBECDBF1C018BEB9FE00C
:108B10000E94746E40E855E260E070E08BEB9FE0ED
:108B20000E94A18064E670E080E090E00E9447939C
:108B30008CED95E0A0E0B0E08093BF0F9093C00F64
:108B4000A093C10FB093C20F64E670E080E090E0A4
:108B50000E9447938FEF8A8781E08B8786E88C8716
:108B60001D861E861F86188A198A89E78A8BC1018D
:108B7000880F991F9E8B8D8BC12CD12CE12CF12C51
:108B8000412C512C32018BEB9FE0E214F3046CF585
:108B9000ED89FE89CE16DF0644F50E946C540897D5
:108BA0004CF049E050E0BE01665F7F4F8BEB9FE0E9
:108BB0000E94425465E070E080E090E00E9447939C
:108BC00000E010E0812C912C54018BEB9FE00E947F
:108BD0009D54892B31F4F4E08F169104A104B10463
:108BE000ACF50230110594F535C00E94746EE114A5
:108BF000F10409F47101C301B2010E947CA64B018A
:108C00005C01B701FF0C880B990B0E947CA69B01AD
:108C1000AC01C501B4010E94CCA866960FB6F894C9
:108C2000DEBF0FBECDBFDF91CF911F910F91FF909F
:108C3000EF90DF90CF90BF90AF909F908F907F90FC
:108C40006F905F904F903F902F9008958FEFC81ACC
:108C5000D80A99CF8BEB9FE00E949D54892B69F035
:108C60008BEB9FE00E947B54E1E0F0E0EC0FFD1FF6
:108C7000E00FF11F80830F5F1F4F65E070E080E021
:108C800090E00E9447930230110569F599818A8529
:108C9000981329C09A818C85981325C0CE0103961C
:108CA0009C8B8B8B8BEB9FE00E949D54892B31F426
:108CB00094E089169104A104B1043CF50930110532
:108CC000C1F48B8190E0982F88272C81820F911D11
:108CD000092E000CAA0BBB0B480E591E6A1E7B1EE8
:108CE000EFEFEE1AFE0AFFEF8F1A9F0AAF0ABF0AD4
:108CF0006CCF8BEB9FE00E947B54EB89FC898193C6
:108D0000FC8BEB8B0F5F1F4FCDCF0430110544F36D
:108D1000D8CF2F923F924F925F926F927F928F9215
:108D20009F92AF92BF92CF92DF92EF92FF920F93FA
:108D30001F93CF93DF936C01C7E3D5E085E9882EBD
:108D400084E0982E03ED11E1EE24E394F12C22E16E
:108D5000222E312C33E1432E512C40E1642E712C14
:108D600051E1A52EB12C80919304909194048E151D
:108D70009F050CF4CFC021E0C216D10439F4F801EC
:108D800082AD93ADF401918380830AC0F2E0CF16E7
:108D9000D10431F4F40180819181F80193AF82AF65
:108DA000F40180819181009739F48A819B819093AD
:108DB000D3048093D20422C08130910539F48A8192
:108DC0009B819093D1048093D00418C08230910588
:108DD00039F48A819B819093CF048093CE040EC096
:108DE000039761F48A819B819093CD048093CC0496
:108DF0006FEC7CE086EB93E10E946D58F401819169
:108E000091914F018430910539F42A813B8130934F
:108E100011022093100221C08530910539F42A8176
:108E20003B81309307022093060217C086309105DC
:108E300039F42A813B813093CB042093CA0417C0B4
:108E40008730910539F42A813B81309305022093C4
:108E5000040217C08A309105F1F18531910539F48A
:108E60002A813B81309303022093020234C0863171
:108E7000910539F42A813B8130930102209300024D
:108E80002AC08731910539F52A813B812830310587
:108E900049F470928F0460928E04B0928D04A09277
:108EA0008C0419C02730310549F430928F04209288
:108EB0008E0450928D0440928C040DC026303105F2
:108EC00051F421E030E030938F0420938E0410920F
:108ED0008D0410928C049C012B5031092A303105ED
:108EE00090F42A813B813093CD042093CC0439E166
:108EF000389FB001399F700D1124655E7D4F86EB60
:108F000093E10E946D588FEFE81AF80A22960E5FDF
:108F10001F4F29CFDF91CF911F910F91FF90EF90BD
:108F2000DF90CF90BF90AF909F908F907F906F9089
:108F30005F904F903F902F9008956F927F928F9205
:108F40009F92AF92BF92CF92DF92EF92FF920F93D8
:108F50001F93CF93DF93CDB7DEB768970FB6F89422
:108F6000DEBF0FBECDBF7C018091491290914A12A5
:108F7000019731F06FEC7CE0C7010E9415594DC19B
:108F80006BE97BE0CE010D960E941559BE01635F2F
:108F90007F4F81E89EE00E9473596CE271E080E0AF
:108FA00090E00E944793CE0143960E94FD7B64E6C9
:108FB00070E080E090E00E944793C12CD12C85E0C6
:108FC000A82EB12C9AE0892E912C66EA7BE0CE0186
:108FD00001960E9415598F89988D892B69F06B88AD
:108FE0007C8869817A81C3010E94E7AD009721F0F6
:108FF0008C010619170902C00FEF1FEFCE01019671
:109000000E94D158A8014F5F5F4FBE016D5E7F4F38
:10901000CE0101960E946782BE016F5F7F4FCE0135
:109020000D960E949758CE0101960E94D1588989C9
:109030009A89892B69F060E070E0CE010D960E945C
:109040009E57082E000C990BC0970A9708F4CEC0C3
:1090500010E06AE87BE0CE0101960E94055944E1E8
:1090600050E06FEF7FEFCE0101960E942C74CE018D
:1090700001960E94D1588FEFC81AD80A62E370E0B7
:1090800080E090E00E944793C601B5010E9441AB89
:10909000019771F5CE0101960E94C07A8D819E8163
:1090A000892B59F0BE016F5F7F4F80E893E10E94EA
:1090B00082580E94E00811E017C0E4E1CE16D10406
:1090C0009CF0C601B4010E9441AB892B69F4BE013A
:1090D000635F7F4F81E89EE00E94735968EC70E007
:1090E00080E090E00E944793CE0101960E94D15803
:1090F000CE0101960E94FD7BBE016F5F7F4FCE01C6
:1091000043960E949758CE0101960E94D15862E37F
:1091100070E080E090E00E944793F4E6CF16D1041F
:1091200019F0112309F451CF8091CE0D8823F1F06D
:1091300065E57CE0CE0101960E941559BE01635F92
:109140007F4FCE0101960E942258BC01CE010796A6
:109150000E940D59CE0107960E941577CE01079601
:109160000E94D158CE0101960E94D15889899A89CE
:10917000892B61F060E070E0CE010D960E949E5751
:10918000082E000C990BC0970A9730F068EA7BE034
:10919000C7010E94155921C064EB7BE0CE01019606
:1091A0000E941559BE016F5F7F4FCE010D960E9440
:1091B0002654182FCE0101960E94D1581111E6CFE6
:1091C000F701118210821382128215821482BE016D
:1091D000635F7F4FC7010E949758CE0143960E945C
:1091E000D158CE010D960E94D15817C064EB7BE098
:1091F000CE0101960E941559BE016F5F7F4FCE01CF
:109200000D960E942654082FCE0101960E94D15837
:1092100011E0002309F41DCF1BCFC70168960FB6DC
:10922000F894DEBF0FBECDBFDF91CF911F910F919C
:10923000FF90EF90DF90CF90BF90AF909F908F9076
:109240007F906F9008954F925F926F927F928F926E
:109250009F92AF92BF92CF92DF92EF92FF92CF9305
:10926000DF93CDB7DEB768970FB6F894DEBF0FBEB9
:10927000CDBF6B017C010E947F93698B7A8B8B8BB6
:109280009C8B8EE19FE00E94746E61E080918E0461
:109290000E94C19260E080918C040E94C1920E9461
:1092A0008A717EDB9ADB6D877E878F87988B0E9421
:1092B00022934B015C016AE070E080E090E00E9444
:1092C00047936CEB7BE088E693E10E946D5820E0C9
:1092D00030E04AE754E4C701B6010E94DBA66D8B7B
:1092E0007E8B8F8B988F412C512C3201C12CD12C2D
:1092F0007601C701B6010E947CA62D893E894F895F
:10930000588D0E9476A687FF83C10E947F9329898A
:109310003A894B895C89621B730B840B950B0E9405
:109320007AA620E030E04AE754E40E94CCA8AB01E2
:10933000BC0123E0CE0101960E94D658BE016F5FAA
:109340007F4F82E693E10E949758CE0101960E94DA
:10935000D15843DB6B017C010E9422939B01AC013D
:10936000281939094A095B0949015A0131ED831667
:1093700037E09306A104B1040CF441C020E030E0D2
:10938000A901C701B6010E94BBA918165CF426EA20
:109390003BE944EC5BE3C701B6010E9476A687FF78
:1093A0000BC02DC026EA3BE944EC5BEBC701B601DC
:1093B0000E94BBA918161CF1C501B40128EE33E0C8
:1093C00040E050E00E94A8A7CA01B9010E947CA613
:1093D0004B015C012D853E854F855889C701B6013B
:1093E0000E9405A820E030E04AE754E40E94DBA692
:1093F000A50194010E94CCA84B015C0103C0812C03
:10940000912C540162E673E1CE0101960E940D5940
:109410006FEC79E0CE0101960E940B58BC0182E608
:1094200093E10E948258CE0101960E94D15823E018
:10943000B701A601CE0101960E94D658BE016F5F0A
:109440007F4FCE0107960E940D596AED7BE0CE0159
:1094500007960E940B58BC018CE593E10E9482584C
:10946000CE0107960E94D158CE0101960E94D15894
:1094700022E0B501A401CE0107960E94D65866E706
:109480007CE0CE0101960E94155962E673E1CE019F
:1094900001960E9422586DED7BE00E940B586CE50E
:1094A00073E10E94225862ED79E00E940B58BE01E0
:1094B000695F7F4F0E9422586DEC79E00E940B5843
:1094C000BC0188E693E10E944158CE0101960E94BA
:1094D000D158CE0107960E94D15820E030E0A90172
:1094E000C501B4010E94BBA987FD06C067E67CE008
:1094F0008CE593E10E94335822E0B501A401CE012E
:1095000001960E94D658BE016F5F7F4FCE0107962D
:109510000E940D596DEC79E0CE0107960E940B5820
:10952000BC018CE593E10E944158CE0107960E9450
:10953000D158CE0101960E94D15868E673E1CE0160
:1095400001960E940D59CE0101960E941577CE0119
:1095500001960E94D158C301B20125E030E040E0FD
:1095600050E00E94A8A7672B682B692B21F563E8C0
:109570007BE0CE0101960E94055945E050E060E095
:1095800070E0CE0101960E948773CE0101960E9481
:10959000D1586CE573E1CE0101960E940D5945E06A
:1095A00050E06FEF7FEFCE0101960E94D381CE0194
:1095B00001960E94D1586FEC7CE088E693E10E940E
:1095C0006D5865E070E080E090E00E9447930E9453
:1095D0007F936B017C0129893A894B895C89C21A86
:1095E000D30AE40AF50AF9D96D877E878F87988BAD
:1095F0000E9422934B015C016AE070E080E090E001
:109600000E9447933FEF431A530A630A730A71CECD
:1096100060E080918E040E94C19268960FB6F89423
:10962000DEBF0FBECDBFDF91CF91FF90EF90DF90F7
:10963000CF90BF90AF909F908F907F906F905F90F2
:109640004F9008954F925F926F927F92AF92BF9228
:10965000CF92DF92EF92FF920F931F93CF93DF93FE
:10966000CDB7DEB7EA970FB6F894DEBF0FBECDBF19
:10967000F82E6FEC7CE0CE01C5960E9415598E0144
:109680000B5E1F4F6F2DC8010E948E8C18870F83B1
:109690001D821E82198289E08A8381E08B838C83FC
:1096A0001C8A1B8ACE01019636D6CE010196C3D5FF
:1096B000CE010196E5D40E8110E00330110509F4C6
:1096C0006DC169E77BE0CE01C5960E9447586FECFB
:1096D0007CE088E693E10E946D58BE016B5C7F4F91
:1096E000CE0183960E940D594AE050E060E070E0A0
:1096F000CE0183960E948773CE0183960E94D15833
:1097000061E080E00E94277D60EF7BE0CE01C5969E
:109710000E946D5883E5A82E8DE0B82ECC24C3940A
:10972000D12CE12CF12CE016F1060CF0EDC06E2DE1
:10973000CE01019635D4F50121913191419151919C
:109740005F010E9406A82B013C0120E030E04CEFB5
:1097500052EC0E9476A687FF24C0B601CE018996FE
:109760000E941B7265E378E0CE0183960E94155932
:10977000BE01675D7F4FCE0183960E94225861EE45
:109780007BE00E940B58BC0188E693E10E9441589F
:10979000CE0183960E94D158CE0189960E94D1585D
:1097A00048C022E0B301A201CE018F960E94D65894
:1097B000B601CE0189960E941B7265E378E0CE0166
:1097C00083960E941559BE01675D7F4FCE01839637
:1097D0000E9422586FE976E00E940B58BE01615D3D
:1097E0007F4F0E942258BC018CE593E10E94825871
:1097F000CE0183960E94D158CE0189960E94D158FD
:10980000CE018F960E94D1586CE573E1CE0183960C
:109810000E940D5967E67CE0CE0183960E940B58AA
:10982000BC0188E693E10E944158CE0183960E94D4
:10983000D1580130110559F4E114F10409F05DC06B
:1098400068E673E1CE01C5960E94825856C0023088
:10985000110511F522E0B301A201CE0183960E9409
:10986000D658BE016D5D7F4FCE0189960E940D597D
:1098700067E67CE0CE0189960E940B58BC01CE01C0
:10988000C5960E944158CE0189960E94D158CE01BA
:1098900083960E94D15831C00330110571F16CE5F7
:1098A00073E1CE0183960E940D5944E150E06FEFC1
:1098B0007FEFCE0183960E94D381CE0183960E94D2
:1098C000D15863E77CE0CE0183960E941559CE0102
:1098D00083960E94566ECE0183960E94D158809145
:1098E000DD04882351F08091DC04882331F060EDA1
:1098F00077E080E090E00E944793FFEFEF1AFF0AC5
:109900008FEFC81AD80A0FCFCE01C5960E943E57D6
:1099100088E693E10E943E5701151105C9F466E6F9
:109920007BE088E693E10E9447586BE57BE0CE013F
:1099300083960E9405594AE050E06FEF7FEFCE0119
:1099400083960E94D381CE0183960E94D158EAC0AB
:10995000043011050CF0FFC0BE016B5C7F4FCE01DF
:1099600083960E940D594AE050E06FEF7FEFCE01E1
:1099700083960E94D381CE0183960E94D15863E7DB
:109980007CE0CE0183960E941559CE0183960E94F9
:10999000566ECE0183960E94D158DDC06DEE7BE0FD
:1099A000CE01C5960E946D58BE016B5C7F4FCE0103
:1099B00083960E940D594AE050E060E070E0CE01CD
:1099C00083960E948773CE0183960E94D1586FECD4
:1099D0007CE088E693E10E946D5868E673E1CE0171
:1099E000C5960E94825800E010E0602FCE010196DB
:1099F000D7D26B017C0122E0AB01BC01CE01839682
:109A00000115110551F40E94D658BE016D5D7F4FBE
:109A100083E694E10E94735918C00E94D658BE0193
:109A20006D5D7F4FCE0189960E940D5967E67CE0FF
:109A3000CE0189960E940B58BC01CE01C5960E94AA
:109A40004158CE0189960E94D158CE0183960E943A
:109A5000D15822E0B701A601CE0183960E94D658C4
:109A6000BE016D5D7F4FCE0189960E940D5967E65C
:109A70007CE0CE0189960E940B58BC0188E693E1F8
:109A80000E944158CE0189960E94D158CE018396FA
:109A90000E94D1580F5F1F4F0330110509F0A5CF69
:109AA000CE01C5960E943E57BE016B5C7F4FCE0132
:109AB00083960E940D594AE050E06FEF7FEFCE0190
:109AC00083960E94D381CE0183960E94D15863E78A
:109AD0007CE0CE0183960E941559CE0183960E94A8
:109AE000566ECE0183960E94D15888E693E10E947B
:109AF0003E5763EF7BE0CE0183960E94155968E6DE
:109B000073E1CE0183960E9422586DEF7BE00E94A4
:109B10000B58BC0188E693E10E948258CE018396DF
:109B20000E94D158CE01C5960E94D158EA960FB630
:109B3000F894DEBF0FBECDBFDF91CF911F910F9183
:109B4000FF90EF90DF90CF90BF90AF907F906F909D
:109B50005F904F9008956DEF7BE088E693E10E945F
:109B60003358E0CF96E0899FD0011124A252BC4E19
:109B700090967C936E935F9791E091969C939197CA
:109B800090914A14E0914B14F0914C14992339F0C0
:109B9000309751F0811108C08091FA1304C03097BA
:109BA00019F05C968C9119940895BF92CF92DF9230
:109BB000EF92FF920F931F93CF93DF93EC016B0112
:109BC0008D85811105C0CE010E94578C811105C081
:109BD0001B861D861C8680E060C040E060EFCE01E1
:109BE0000E94B15B01E0E12CB12C11E0CE010E949A
:109BF000048CF82ECE010E94048C91E0F91203C06F
:109C00008130B1F434C02E2D30E0F8121BC08B85AA
:109C1000181738F4FE01E20FF31F8381802341F40B
:109C200002C0811729F0F12C193058F41C8709C0A3
:109C3000FE01EE0DF11D8381802B8383FF24F394BD
:109C400009C0B12EFE01E20FF31F9381802F809592
:109C5000892383836F2DCE010E94288C1F5F000F04
:109C600011F4E39401E087E08E1508F0BFCF1134C2
:109C700008F4AECFBB86B11002C081E08D878B8126
:109C8000882309F4A5CFDE011396F6012B968D915A
:109C90008193CA17DB07D9F781E0DF91CF911F913C
:109CA0000F91FF90EF90DF90CF90BF900895DF92DB
:109CB000EF92FF920F931F93CF93DF937C018B0161
:109CC000D42EDC011696ED91FC911797138615861C
:109CD0001486DF011B9633961E92EA17FB07E1F705
:109CE000C0E0B801F701868197815FDFD82F882314
:109CF00071F0DC1209C067E0C8010E94995BD801CD
:109D000017969C91891721F0CF5FDC1650F7D0E0B1
:109D10008D2FDF91CF911F910F91FF90EF90DF90EA
:109D200008950F931F93CF93DF93C82FD62F86E00C
:109D3000C89FF0011124E252FC4E11A2878D90A120
:109D400081309105D1F040F082309105A1F1039767
:109D5000E1F560E070E033C06623B9F161E070E0E6
:109D60008C2F00DF0E947F9360933614709337141A
:109D7000809338149093391428C00E947F930091E7
:109D80003614109137142091381430913914AB01E6
:109D9000BC01401B510B620B730B809148149091D6
:109DA0004914A0E0B0E084179507A607B70718F498
:109DB00062E070E004C0D11108C063E070E08C2F55
:109DC000DF91CF911F910F91CDCEDF91CF911F9158
:109DD0000F910895FF920F931F93CF93DF931F92DC
:109DE000CDB7DEB7182F062FF42EAE014F5F5F4FB1
:109DF00061E070E00E94DF724981FF2049F021E0BC
:109E000030E001C0220F0A95EAF7242B298309C00C
:109E100081E090E001C0880F0A95EAF780958423DD
:109E200089836981812F0E9446730F90DF91CF91C2
:109E30001F910F91FF9008950F931F93CF93DF937E
:109E4000EC019A01452B11F4CAD506C0462F50E00B
:109E500060E070E00E94BA598C01CE010E94947CAF
:109E6000800F911FDF91CF911F910F910895CF9394
:109E7000DF9342E00E94C37DEC0188E590E10E94FF
:109E8000947C8C0F9D1FDF91CF9108958F929F92AC
:109E9000AF92BF92CF92DF92EF92FF920F931F93F8
:109EA000CF93DF9300D000D0CDB7DEB75C0148ED93
:109EB00053E166E070E082E30E94DF728091D81384
:109EC0009091D9139A8389838091DA139091DB134F
:109ED0009C838B838091DC139091DD139E838D8313
:109EE000CE0101966C018CECE82E83E1F82E850101
:109EF000F601619171916F01F70181909190A190AC
:109F0000B1907F01072E000C880B990B0E947CA654
:109F1000A50194010E94DBA6F801619371938193DE
:109F200091938F01F8EDEF16F3E1FF0609F72696FE
:109F30000FB6F894DEBF0FBECDBFDF91CF911F915A
:109F40000F91FF90EF90DF90CF90BF90AF909F90D8
:109F50008F900895CF93DF93C82F809150140E9463
:109F60000C7D6C2F85EF90E10E94D38B80E00E94E6
:109F7000A97C63E0809150140E94477285EF90E1C4
:109F80000E948B8BEC0185EF90E10E948B8B20E08F
:109F900030E0382FC9018C2B9D2BDF91CF91089594
:109FA0000F931F93CF93DF93CDB7DEB761970FB6B3
:109FB000F894DEBF0FBECDBF8C01462FBE01665F99
:109FC0007F4F75DE811105C060E070E08EEF92EC8E
:109FD0004CC0AE014F5F5F4FBE01665F7F4FC8014F
:109FE0000E94025C882361F12A8130E0C901982F28
:109FF0008827990F990F990F698128E0629FB00116
:10A0000011249C01262B372B8A858031E1F4688549
:10A0100070E08F81AB01481B5109CA019695982FBA
:10A020008827979587950E9441AB60517109207FE1
:10A0300053E0220F331F5A95E1F7620F731F04C0DC
:10A0400060E874EE01C0B901613854EE75070CF494
:10A05000BBCF072E000C880B990B0E947CA620E03A
:10A0600030E040E05CE30E94DBA661960FB6F89416
:10A07000DEBF0FBECDBFDF91CF911F910F9108952D
:10A080009F92AF92BF92CF92DF92EF92FF920F9387
:10A090001F93CF93DF93CDB7DEB761970FB6F894D8
:10A0A000DEBF0FBECDBF8C018CE0F8018183C12CD7
:10A0B000D12C2FE5E22E3FE7B32E4FE1A42E5FE334
:10A0C000952EF801848190E0C816D9060CF0A1C045
:10A0D0004C2DBE01665F7F4FC801E9DDF80181812B
:10A0E000893038F0F82EFCE0F81728F49CE0F92EBF
:10A0F00002C089E0F82E8A85803139F0BE01665FA2
:10A100007F4FC8010E945D5C01C08CE0F81609F425
:10A110007CC0AE014F5F5F4FBE01665F7F4FC801DD
:10A120000E94025C882309F470C08A85803109F49A
:10A130006CC08BE0F81651F0ECE0FE1629F0FAE066
:10A14000FF1206C09D8205C0BD8203C0ED8201C022
:10A15000AD82F801868197810E94578CBE01665FAF
:10A160007F4FF801868197810E94E55B40E06EE4B5
:10A17000F801868197810E94B15B40E06B81F80114
:10A18000868197810E94B15B40E06C81F8018681F5
:10A1900097810E94B15B8A85803139F040E06D8102
:10A1A000F801868197810E94B15BF80186819781D1
:10A1B0000E94578CBE01665F7F4FF80186819781B0
:10A1C0000E94E55BF801408168E4868197810E94E6
:10A1D000B15B64E170E080E090E00E944793F80199
:10A1E0008081882331F06AE070E080E090E00E9496
:10A1F0004793F801868197810E94578CF8018181ED
:10A200008F1508F48F2DF8018183FFEFCF1ADF0A35
:10A2100058CF61960FB6F894DEBF0FBECDBFDF9169
:10A22000CF911F910F91FF90EF90DF90CF90BF9053
:10A23000AF909F9008958F929F92AF92BF92CF92CE
:10A24000DF92EF92FF920F931F93CF93DF93EC0176
:10A250008E819F810E94578C40E06CEC8E819F81A3
:10A260000E94B15B488164E48E819F810E94B15B52
:10A270008A81882309F442C0E981E950E33040F43F
:10A28000F0E0EE0FFF1FE75BFA4F0081118102C083
:10A290000EEE12E08B818823F9F0888181111CC0B9
:10A2A0000E947F934B015C016801110FEE08FF08CB
:10A2B0008E819F810E94048C813001F10E947F93E6
:10A2C000DC01CB018C199D09AE09BF0988159905E0
:10A2D000AA05BB0568F312C0B801110F880B990BD2
:10A2E000DF91CF911F910F91FF90EF90DF90CF9072
:10A2F000BF90AF909F908F900C944793DF91CF9138
:10A300001F910F91FF90EF90DF90CF90BF90AF9093
:10A310009F908F900895EF92FF920F931F93CF938A
:10A32000DF93CDB7DEB728970FB6F894DEBF0FBE28
:10A33000CDBF8C01DC011696ED91FC911797138629
:10A3400015861486DF011B9633961E92EA17FB07CB
:10A35000E1F7F80114821582EE24E394BE016F5FE9
:10A360007F4FD80116968D919C9117971EDC8823FC
:10A3700009F475C067E0CE0101960E94995B98854B
:10A380008913ECCFF8018081811124C086819781E7
:10A390000E94578CBE016F5F7F4FD80116968D913A
:10A3A0009C9117970E94E55B40E064EBF801868181
:10A3B00097810E94B15BD80116968D919C91179759
:10A3C0000E94048CF82EF801868197810E94578C98
:10A3D000FF20B1F1D8011196FC9089818031D9F12B
:10A3E000BE016F5F7F4FC8010E945D5C8F1518F43E
:10A3F000F80181810BC08981803111F48CE006C0A5
:10A40000BE016F5F7F4FC8010E945D5CD80111964D
:10A410008C93119714968C9114978F5F14968C934C
:10A420008981883281F030F4803169F0823209F01C
:10A4300095CF09C08B3339F0823409F08FCF03C038
:10A44000F801E082C7CFD80115968C9115978F5FE0
:10A4500015968C9383CFBCE0BF1550F2CFCF2896D2
:10A460000FB6F894DEBF0FBECDBFDF91CF911F9125
:10A470000F91FF90EF9008956F927F928F929F922D
:10A48000AF92BF92CF92DF92EF92FF920F931F9302
:10A49000CF93DF9381E080934A140E947F930091D1
:10A4A0003A1410913B1420913C1430913D14AB01AF
:10A4B000BC01401B510B620B730B809146149091B1
:10A4C0004714A0E0B0E084179507A607B70708F087
:10A4D000E6C0C0E080914414C81730F0712C812C84
:10A4E000912C5401839440C0E0914014F0914114A8
:10A4F000EC0FF11D62E080810E94C192CF5FEACF34
:10A50000C62DD0E0E0914014F0914114EC0FFD1FF6
:10A5100080810E946B922496CC0FDD1FC252DC4ECC
:10A52000892B09F04BC0888199818C299D299983B9
:10A530008883639480914414681610F3E091421468
:10A54000F0914314E00FF11F61E080810E9493922B
:10A550008091421490914314FC01E00FF11F60E0E0
:10A5600080810E94C192739480914514781658F5A9
:10A57000072D10E0E0914214F0914314E00FF11F19
:10A5800061E080810E94C192E0914214F0914314F5
:10A59000E00FF11F60E080810E949392D501C40119
:10A5A000072C04C0880F991FAA1FBB1F0A94D2F75B
:10A5B0006C017C01E094F094612CBCCF888199817E
:10A5C0008E219F21B4CF2EEDE22E23E1F22EF70152
:10A5D0008FEF9FEF278D30A1232B21F4148E968FC0
:10A5E000858F11A2369624E1EA31F20799F7C0E08F
:10A5F00096E0D92E80914414C81758F5D0E00C2F5E
:10A6000010E0000F111F0A511C4E20914514D21763
:10A61000F0F4F801408151810D2E02C05695479506
:10A620000A94E2F7642F6170C29F900111242D0FEC
:10A63000311DEEEDF3E180E0A58DB68D2A173B07C5
:10A6400009F44DC08F5F36968A30B1F72CC0CF5FCA
:10A65000D1CFC0E0F70181A18111C1E0F6E0EF0E9A
:10A66000F11C2AE1E21624E1F206A1F70E947F9391
:10A6700060933A1470933B1480933C1490933D1470
:10A68000CC2369F08091FF13882349F08091FD135A
:10A690009091FE13019719F48091FA1329C010923A
:10A6A0004A1480E025C040FF1BC0EEEDF3E180E0DE
:10A6B00090E0448D411116C0E0913E14F0913F149A
:10A6C000E20FF31F4081D89EF001D99EF00D1124B6
:10A6D000E252FC4E448F368F258F10A2178E21DB5D
:10A6E000DF5F93CF019636968A30910511F7F8CF48
:10A6F000DF91CF911F910F91FF90EF90DF90CF905E
:10A70000BF90AF909F908F907F906F900895CF9360
:10A71000DF93FC0124813581232B71F0FB01DC01E7
:10A72000CD91DC9160817181CE010E94E7AD0097EF
:10A7300019F08C1B9D0B02C08FEF9FEFDF91CF9123
:10A7400008950F931F93CF93DF93FC01C481D581AC
:10A75000209719F4FB01108211C0415051094C1788
:10A760005D0708F4EA018B01FC0160817181AE0193
:10A77000C8010E94D8ADC00FD11F1882DF91CF91C0
:10A780001F910F910895AF92BF92CF92DF92EF92F7
:10A79000FF920F931F93CF93DF93FC0124813581A8
:10A7A000FB01448155818901041B150B411551059D
:10A7B00051F12115310539F12417350720F1021720
:10A7C000130718F08901015011097B01FC01A080D9
:10A7D000B180C501DFEFCFEF6501C00ED11EC816F5
:10A7E000D906A0F0F701608171810E94E7AD009762
:10A7F00069F09C012A193B090217130710F0D22FA8
:10A80000C32F0196ECCF8FEF9FEF02C08D2F9C2FAF
:10A81000DF91CF911F910F91FF90EF90DF90CF903C
:10A82000BF90AF900895CF93DF931F921F92CDB743
:10A83000DEB769831A8241E050E0BE016F5F7F4F4F
:10A84000BDD30F900F90DF91CF910895FB0144810C
:10A850005581FC01248135812417350778F08081EA
:10A860009181009759F0FB0160817181611571053B
:10A8700029F00E94CAAD21E0892B09F020E0822F47
:10A8800008950895CF92DF92EF92FF920F931F9356
:10A89000CF93DF936C017A018B01C0E0D0E0CE153D
:10A8A000DF0581F0D8016D918D01D601ED91FC910C
:10A8B0000190F081E02DC6011995892B11F02196A8
:10A8C000EECF7E01C701DF91CF911F910F91FF90D5
:10A8D000EF90DF90CF900895FC01538D448D252F8C
:10A8E00030E0842F90E0821B930B541710F0CF962A
:10A8F000089501970895FC01918D828D981761F05C
:10A90000828DDF01A80FB11D5D968C91928D9F5FA6
:10A910009F73928F90E008958FEF9FEF0895FC0151
:10A92000918D828D981731F0828DE80FF11D858D04
:10A9300090E008958FEF9FEF0895FC01918D228D97
:10A94000892F90E0805C9F4F821B91098F7399271C
:10A95000089581E89EE0F1DF21E0892B09F420E0F1
:10A96000822F08958EE19FE0E8DF21E0892B09F432
:10A9700020E0822F08958BEB9FE0DFDF21E0892B21
:10A9800009F420E0822F089588E590E1D6DF21E0E8
:10A99000892B09F420E0822F0895FC01848DDF01CA
:10A9A000A80FB11DA35ABF4F2C91848D90E0019642
:10A9B0008F739927848FA689B7892C93A089B18931
:10A9C0008C91837080648C93938D848D981306C0D2
:10A9D0000288F389E02D80818F7D80830895EF9236
:10A9E000FF920F931F93CF93DF93EC0181E0888F49
:10A9F0009B8D8C8D981305C0E889F989808185FD30
:10AA000025C0F62E0B8D10E00F5F1F4F0F7311271F
:10AA1000E02E8C8DE8120BC00FB607FCFACFE88948
:10AA2000F989808185FFF5CFCE01B7DFF2CF8B8D1D
:10AA3000FE01E80FF11DE35AFF4FF0829FB7F89433
:10AA40000B8FEA89FB89808180620AC09FB7F894E6
:10AA5000EE89FF896083E889F98980818370806449
:10AA600080839FBF81E090E0DF91CF911F910F9194
:10AA7000FF90EF900895CF93DF93EC01888D8823AA
:10AA8000C1F0EA89FB89808185FD05C0A889B98963
:10AA90008C9186FD0EC00FB607FCF5CF808185FF37
:10AAA000F2CFA889B9898C9185FFEDCFCE0175DFF2
:10AAB000E8CFDF91CF91089580E090E0892B19F0E5
:10AAC00063DF811116C080E090E0892B19F053DF1D
:10AAD000811112C080E090E0892B19F043DF8111D1
:10AAE0000EC080E090E0892B79F033DF81110AC03D
:10AAF00008950E940000E7CF0E940000EBCF0E9463
:10AB00000000EFCF0C94000008950E9494ADCF9305
:10AB1000DF93EC0188819981009711F00E942BACA2
:10AB2000198218821D821C821B821A82DF91CF91AA
:10AB300008950F931F93CF93DF93EC018881998140
:10AB4000009729F02A813B812617370788F48B016B
:10AB50006F5F7F4F0E94B4AC009761F09983888348
:10AB60001B830A832C813D81232B11F4FC0110826D
:10AB700081E001C080E0DF91CF911F910F91089596
:10AB8000EF92FF920F931F93CF93DF93EC017B0122
:10AB90008A01BA01CEDF811103C0CE01B8DF07C040
:10ABA0001D830C83B701888199810E94C3ADCE01BA
:10ABB000DF91CF911F910F91FF90EF9008950F9328
:10ABC0001F93CF93DF938C01EB0188E2FB0111927D
:10ABD0008A95E9F74BE050E060E17CE0CE010E940D
:10ABE000D8AD1B8681E090E0A0E0B0E08C879D8727
:10ABF000AE87BF87F80185899689A789B08D888B34
:10AC0000998BAA8BBB8B82E090E0A0E0B0E08C8BAC
:10AC10009D8BAE8BBF8B1CA21DA21EA21FA280E02B
:10AC200090E0A8E4B4E4888F998FAA8FBB8F80E06E
:10AC300090E0A8E4B4EC8C8F9D8FAE8FBF8F8DEC2D
:10AC40009CECACE4BEE388A399A3AAA3BBA3DF91C9
:10AC5000CF911F910F9108954F925F926F927F92C3
:10AC60008F929F92AF92BF92CF92DF92EF92FF921C
:10AC70000F931F93CF93DF938C01EB0184E2FB01D1
:10AC800011928A95E9F78EE10E940C7D83E090E0B5
:10AC90000E94077D0E94057D66E08EE10E9447725A
:10ACA0008091A80D90E02091A90D821B910986301A
:10ACB0009105ECF385EF90E10E948B8B882E85EF58
:10ACC00090E10E948B8B982E85EF90E10E948B8BF8
:10ACD000682E85EF90E10E948B8B782E85EF90E1B6
:10ACE0000E948B8B482E85EF90E10E948B8B582E13
:10ACF000B82CA12CB5016929072E000C880B990BE3
:10AD00000E947CA64B015C01F801658376838783F2
:10AD10009087D42CC12CB6016529072E000C880B16
:10AD2000990B0E947CA6F8016187728783879487BC
:10AD3000F62CE12CB7016729072E000C880B990B24
:10AD40000E947CA6F801658776878787908B118A99
:10AD5000128A138A148A84E290E0A0E0B0E088832B
:10AD60009983AA83BB8385899689A789B08D8C83B3
:10AD70009D83AE83BF8382E090E0A0E0B0E088874F
:10AD80009987AA87BB87188A198A1A8A1B8AC09052
:10AD9000D804D090D904E090DA04F090DB04A70145
:10ADA0009601C501B4010E94CCA820E030E048EC37
:10ADB00052E40E94DBA66C8B7D8B8E8B9F8BA70150
:10ADC0009601F80161857285838594850E94CCA8DF
:10ADD00020E030E048EC52E40E94DBA6688F798FD7
:10ADE0008A8F9B8F2091D4043091D5044091D60452
:10ADF0005091D704F80165857685878590890E94F2
:10AE0000CCA820E030E048EC52E40E94DBA66C8F36
:10AE10007D8F8E8F9F8F81E0DF91CF911F910F915A
:10AE2000FF90EF90DF90CF90BF90AF909F908F906A
:10AE30007F906F905F904F900895862F0C946B9247
:10AE4000862F642F0C949392862F642F0C94C192BA
:10AE5000FC0180819181009711F00C94E0A160E0E9
:10AE600070E0CB010895FC0180819181009711F081
:10AE70000C9400A260E070E0CB010895AF92BF9205
:10AE8000CF92DF92EF92FF920F931F93CF93DF93B6
:10AE9000DC01CD90DC901197C114D10409F443C0BA
:10AEA0001496CD91DC9115972097E9F18C017601EC
:10AEB0005701BFEFAB1ABB0AF7018081082E000CC7
:10AEC000990B0E9446A6892B11F07501F1CF2197AD
:10AED000CC0DDD1D8881082E000C990B0E9446A622
:10AEE000892B29F0CE15DF0510F02197F3CFAE01A5
:10AEF0004F5F5F4F4E195F09D80115965C934E93D3
:10AF00001497CE14DF0420F4B701C6010E94B1AD3E
:10AF1000D801ED91FC91119714968D919C91159704
:10AF2000E80FF91F1082DF91CF911F910F91FF90D1
:10AF3000EF90DF90CF90BF90AF900895FC012481F7
:10AF400035816217730748F480819181009729F059
:10AF5000FC01E60FF71F8081089580E00895EF92CD
:10AF6000FF920F931F93CF93DF936115710511F437
:10AF700080E01DC08B01EC01CB010E942DA2009747
:10AF8000A9F02C813D817C01E20EF31EB701CE01B8
:10AF9000D0DD882369F3288139818C819D81B801B6
:10AFA000820F931F0E9426A2FD82EC8281E0DF9136
:10AFB000CF911F910F91FF90EF900895EF92FF9224
:10AFC0000F931F93CF93DF936115710511F480E008
:10AFD0001BC041155105B9F07B01EC018C819D81AD
:10AFE0008A01080F191FB801CE01A3DD882379F368
:10AFF000288139818C819D81B701820F931F0E9426
:10B00000C3AD1D830C8381E0DF91CF911F910F9120
:10B01000FF90EF900895CF93DF93EC0161157105D8
:10B0200059F0FB0101900020E9F73197AF01461B71
:10B03000570BC4DF811102C0CE0169DDCE01DF9163
:10B04000CF910895CF93DF93EC01FB0144815581AB
:10B0500060817181B3DF811102C0CE0158DDCE0164
:10B06000DF91CF9108956115710549F0FB010190C1
:10B070000020E9F73197AF01461B570B9FCF80E0C7
:10B080000895FB01448155816081718197CFEF92D2
:10B09000FF920F931F93CF93DF93EC018B01611508
:10B0A000710549F0CB010E942DA27C01BC01CE01AB
:10B0B00040DD811103C0CE012ADD07C0FD82EC8294
:10B0C000B801888199810E9426A2CE01DF91CF919B
:10B0D0001F910F91FF90EF900895CF93DF93EC01B4
:10B0E0006115710551F0FB0101900020E9F73197DE
:10B0F000AF01461B570B44DD01C009DDCE01DF91D6
:10B10000CF910895CF93DF93EC01FB01861797074A
:10B1100051F0608171816115710521F04481558183
:10B120002FDD01C0F4DCCE01DF91CF9108950F93A4
:10B130001F93CF93DF938C01EB01FC018081918100
:10B14000009739F06881798161157105A1F40E9439
:10B150002BAC88819981F801918380838A819B81BE
:10B16000938382838C819D81958384831982188245
:10B170001B821A820FC0F801428153812C813D81CC
:10B180004217530720F30E94C3AD8C819D81F801C3
:10B19000958384831D821C82DF91CF911F910F9133
:10B1A0000895FC01808191810C942BACEF92FF9269
:10B1B0000F931F93CF93DF93CDB7DEB7A1970FB651
:10B1C000F894DEBF0FBECDBF7C01CB01BA01F70101
:10B1D00011821082138212821582148242E0420F81
:10B1E0008E010F5F1F4F0E94C1A1BC01C70175DF17
:10B1F000A1960FB6F894DEBF0FBECDBFDF91CF9101
:10B200001F910F91FF90EF900895FC011182108221
:10B2100013821282158214823ACFFC0111821082AD
:10B2200013821282158214826DCFFC01118210826A
:10B2300013821282158214826115710549F0FB0197
:10B2400001900020E9F73197AF01461B570B98CCCE
:10B250000895BF92CF92DF92EF92FF920F931F93C8
:10B26000CF93DF937C016B018A01E9012417350735
:10B2700020F4812F8901C42FD82F6FEC7CE0C70107
:10B28000D4DFD60114968D919C9115970817190754
:10B29000C0F48C179D0708F4EC01D601ED91FC91E8
:10B2A0001197EC0FFD1FB08010826D917C91600FA3
:10B2B000711FC70112DFD601ED91FC91EC0FFD1F4C
:10B2C000B082C701DF91CF911F910F91FF90EF9056
:10B2D000DF90CF90BF900895DC01ED91FC9101903B
:10B2E000F081E02D1994DB0114964D915C91159736
:10B2F0006D917C91DC01ED91FC910280F381E02D58
:10B300001994EF92FF920F931F93CF93DF938C01C9
:10B310007B01C0E0D0E0F701EC0FFD1F64916623D4
:10B3200061F0D801ED91FC910190F081E02DC80110
:10B330001995892B11F02196EECFCE01DF91CF9197
:10B340001F910F91FF90EF9008956115710579F0AD
:10B35000FB0101900020E9F73197AF01461B570B25
:10B36000DC01ED91FC910280F381E02D199480E0E5
:10B3700090E008958F929F92AF92BF92EF92FF92CA
:10B380000F931F93CF93DF93CDB7DEB7A1970FB67F
:10B39000F894DEBF0FBECDBF7C01FA01CB0119A22C
:10B3A000223008F42AE08E010F5D1F4F822E912C6F
:10B3B000A12CB12CBF01A50194010E94D4A7F901D1
:10B3C000CA01015011096A3014F4605D01C0695C62
:10B3D000D8016C93232B242B252B61F7B801C701CF
:10B3E000B4DFA1960FB6F894DEBF0FBECDBFDF91DC
:10B3F000CF911F910F91FF90EF90BF90AF909F90D2
:10B400008F900895CF92DF92EF92FF920F931F9348
:10B41000CF93DF934115510579F4DC01ED91FC9157
:10B420000190F081E02DDF91CF911F910F91FF905E
:10B43000EF90DF90CF9019946B01770FEE08FF0823
:10B440004A305105E9F4F7FE19C0EC016DE244DF22
:10B450008C0144275527BA014C195D096E097F09F3
:10B460002AE0CE0187DF800F911FDF91CF911F91DE
:10B470000F91FF90EF90DF90CF9008952AE001C0E8
:10B48000242FB701A601DF91CF911F910F91FF905B
:10B49000EF90DF90CF906ECF58CF1F920F920FB6E4
:10B4A0000F9211240BB60F922F933F934F935F93FC
:10B4B0006F937F938F939F93AF93BF93EF93FF937C
:10B4C00081E89EE06ADAFF91EF91BF91AF919F9181
:10B4D0008F917F916F915F914F913F912F910F903D
:10B4E0000BBE0F900FBE0F901F9018951F920F92DA
:10B4F0000FB60F9211240BB60F922F933F934F93D9
:10B500005F936F937F938F939F93AF93BF93EF93CB
:10B51000FF9381E89EE00E945292FF91EF91BF91CC
:10B52000AF919F918F917F916F915F914F913F91DB
:10B530002F910F900BBE0F900FBE0F901F9018957C
:10B540001F920F920FB60F9211240BB60F922F93EA
:10B550003F934F935F936F937F938F939F93AF939B
:10B56000BF93EF93FF938EE19FE017DAFF91EF9186
:10B57000BF91AF919F918F917F916F915F914F910B
:10B580003F912F910F900BBE0F900FBE0F901F9009
:10B5900018951F920F920FB60F9211240BB60F92AF
:10B5A0002F933F934F935F936F937F938F939F93CB
:10B5B000AF93BF93EF93FF938EE19FE00E9452926F
:10B5C000FF91EF91BF91AF919F918F917F916F917B
:10B5D0005F914F913F912F910F900BBE0F900FBE37
:10B5E0000F901F9018951F920F920FB60F92112473
:10B5F0000BB60F922F933F934F935F936F937F936D
:10B600008F939F93AF93BF93EF93FF938BEB9FE049
:10B61000C4D9FF91EF91BF91AF919F918F917F918D
:10B620006F915F914F913F912F910F900BBE0F90B3
:10B630000FBE0F901F9018951F920F920FB60F928A
:10B6400011240BB60F922F933F934F935F936F93F9
:10B650007F938F939F93AF93BF93EF93FF938BEB66
:10B660009FE00E945292FF91EF91BF91AF919F9105
:10B670008F917F916F915F914F913F912F910F909B
:10B680000BBE0F900FBE0F901F9018951F920F9238
:10B690000FB60F9211240BB60F922F933F934F9337
:10B6A0005F936F937F938F939F93AF93BF93EF932A
:10B6B000FF9388E590E171D9FF91EF91BF91AF9130
:10B6C0009F918F917F916F915F914F913F912F91BA
:10B6D0000F900BBE0F900FBE0F901F9018951F92EA
:10B6E0000F920FB60F9211240BB60F922F933F9328
:10B6F0004F935F936F937F938F939F93AF93BF937A
:10B70000EF93FF9388E590E10E945292FF91EF91B1
:10B71000BF91AF919F918F917F916F915F914F9169
:10B720003F912F910F900BBE0F900FBE0F901F9067
:10B730001895DC0180E0615098F02D91982F9227A8
:10B74000E92FEF70F0E0E656F44F249192959F7048
:10B75000E92FF0E0E655F44FE491822F8E27EBCFEE
:10B760000895DF92EF92FF920F931F93CF93DF9391
:10B77000EC01D62EE42E08E010E0FF24F39461E003
:10B780008D2D8F2109F460E0CE010E94288CFF0CE2
:10B7900001501109A1F7E11010C0F894E981FA8174
:10B7A00091818881809589238183E981FA819281C1
:10B7B00088818095892382837894DF91CF911F912E
:10B7C0000F91FF90EF90DF900895EF92FF920F930B
:10B7D0001F93CF93DF938C017B0140E065E5C1DFD0
:10B7E000E70188E0E80EF11C699140E0C801B9DF8B
:10B7F000CE15DF05C9F7DF91CF911F910F91FF9013
:10B80000EF9008956F927F928F929F92AF92BF9226
:10B81000CF92DF92EF92FF920F931F93CF93DF931C
:10B82000EC017B018A018E819F810E94578C8823C5
:10B8300099F1B7018E819F81C8DF40E06EEB8E8168
:10B840009F818FDF7801680189E0C80ED11CAE802E
:10B85000BF8088E0882E912C712C66246394C501EA
:10B860000E94048C81117628660CE1E08E1A910802
:10B87000B1F7F70171927F01EC15FD0541F78E815B
:10B880009F810E94578C813039F468E0C80151DFF4
:10B8900091E0F8012085281390E0892FDF91CF9166
:10B8A0001F910F91FF90EF90DF90CF90BF90AF90DE
:10B8B0009F908F907F906F900895CF93DF93CDB737
:10B8C000DEB729970FB6F894DEBF0FBECDBFAE012D
:10B8D0004F5F5F4F97DF882389F08D818F3361F051
:10B8E00020F48F3159F489E00CC08F3519F08F376F
:10B8F00039F004C08BE005C08AE003C080E001C0DD
:10B900008CE029960FB6F894DEBF0FBECDBFDF9155
:10B91000CF9108954F925F926F927F92AF92BF92B4
:10B92000CF92DF92EF92FF920F931F93CF93DF930B
:10B9300000D000D0CDB7DEB781E08093120284E959
:10B940009DE00E94FF37892B09F489C280917C1405
:10B95000882319F010927C1466C610927C14809192
:10B96000CE0D8823A1F165E57CE0CE0101965DDC7A
:10B97000BE016F5F7F4F88E590E1B5DCBE016F5F70
:10B980007F4F81E89EE0AFDCCE0101960ADC40915A
:10B99000980D5091990D60919A0D70919B0D20E139
:10B9A00088E590E1E7DC88E590E10E94947C409195
:10B9B000980D5091990D60919A0D70919B0D20E119
:10B9C00081E89EE0D7DC81E89EE00E94947C809133
:10B9D000980D9091990DA0919A0DB0919B0D883082
:10B9E00025E09207A105B10509F4CCC108F08DC08E
:10B9F000893421E09207A105B10509F4CBC1E0F536
:10BA0000843421E09207A105B10509F49BC1E8F453
:10BA1000813421E09207A105B10509F47BC138F416
:10BA200080349140A105B10509F467C106C2823492
:10BA300021E09207A105B10509F474C18334914056
:10BA4000A105B10509F476C1F8C1863421E0920759
:10BA5000A105B10509F486C108F47CC1873421E051
:10BA60009207A105B10509F485C188349140A1056B
:10BA7000B10509F487C1E1C1823025E09207A10533
:10BA8000B10509F44FC1E8F4843721E09207A1051C
:10BA9000B10509F403C138F482379140A105B1051D
:10BAA00009F406C1CAC1811525E09207A105B105B7
:10BAB00009F423C181309540A105B10509F42AC1DB
:10BAC000BCC1853025E09207A105B10509F442C14A
:10BAD00070F4833025E09207A105B10509F42AC16D
:10BAE00084309540A105B10509F42CC1A6C186306A
:10BAF00025E09207A105B10509F434C187309540CE
:10BB0000A105B10509F436C198C18D3B22E4920725
:10BB10002FEFA207B10509F4E3C008F04AC08F3E39
:10BB200020E192072FEFA207B10509F423C110F518
:10BB3000823325E09207A105B10509F4B9C038F4B4
:10BB400089309540A105B10509F424C176C184333B
:10BB500025E09207A105B10509F4A0C08D3F9240F0
:10BB6000AF4FB10509F069C163E47CE080E893E17F
:10BB7000B4DA8FC08D3D22E292072FEFA207B10504
:10BB800009F48CC038F4873E9841AF4FB10509F4F1
:10BB9000E1C053C18F3C20E392072FEFA207B1050C
:10BBA00009F4D0C0873C9843AF4FB10509F4EAC00F
:10BBB00044C1873928E692072FEFA207B10509F49F
:10BBC000A9C038F58D3A22E592072FEFA207B105FB
:10BBD00009F479C038F4853B9A44AF4FB10509F4B4
:10BBE0008CC02BC1853A2AE592072FEFA207B10539
:10BBF00009F4D0C08D399246AF4FB10509F01DC18F
:10BC000063E47CE080E893E168DA81E08093830D6F
:10BC100040C0873528EA92072FEFA207B105F1F05F
:10BC200078F485382AE792072FEFA207B10509F4C7
:10BC300099C087369849AF4FB10509F473C0FDC06C
:10BC40008F3420EB92072FEFA207B10509F472C0E1
:10BC50008D33924CAF4FB10559F1EFC06CE271E0FA
:10BC600080E090E00E94479382E08093011110925F
:10BC7000041100E010E084E89DE00E94FF37892B6A
:10BC800009F090C00F5F1F4F0536110509F0A4C4DD
:10BC900089C08BEF9FEF0E947C24D5C066E47CE0D6
:10BCA00080E893E11ADA1092830D8CEF9FEFF3CFC7
:10BCB00069E47CE080E893E110DA81E08093830D11
:10BCC0008DEF9FEFE8CF6CE47CE080E893E105DA4C
:10BCD0006CE47CE080E893E100DA8EEF9FEFDBCF4D
:10BCE0006FE47CE080E893E1F8D96FE47CE080E8E1
:10BCF00093E1F3D98FEF9FEFCECF6AEB7BE084E740
:10BD000093E1EBD96AEB7BE080E893E1E6D980E050
:10BD100090E0C1CF60E57CE084E793E1DED981E08B
:10BD200090E0B9CF6DE47CE084E793E1D6D982E07E
:10BD300090E0B1CF6AE47CE084E793E1CED983E080
:10BD400090E0A9CF67E47CE084E793E1C6D984E082
:10BD500090E0A1CF64E47CE084E793E1BED985E084
:10BD600090E099CF69E17CE084E793E1B6D986E081
:10BD700090E091CF6CE17CE084E793E1AED987E07D
:10BD800090E089CF6FE17CE084E793E1A6D988E079
:10BD900090E081CF62E27CE084E793E19ED989E084
:10BDA00090E079CF8091CE0D8823A9F065E47CE006
:10BDB00088E590E1A6DA4091880D5091890D609157
:10BDC0008A0D70918B0D2AE088E590E1D3DA88E541
:10BDD00090E10E94947C8091880D9091890DA091B2
:10BDE0008A0DB0918B0D883025E09207A105B10531
:10BDF00009F4C8C308F0E1C2893421E09207A10523
:10BE0000B10509F4C8C308F08FC2843421E0920759
:10BE1000A105B10509F492C308F06FC2813421E095
:10BE20009207A105B10509F46EC308F058C2803429
:10BE30009140A105B10509F45DC364E670E080E0BE
:10BE400090E00E9447936CE271E080E090E00E94F5
:10BE5000479382E0809301111092041142C0CE01F9
:10BE600001960E94C07ABE016F5F7F4F80E893E128
:10BE70005ED9CE01019695D96AE070E080E090E04D
:10BE80000E9447938091841390918513892B19F018
:10BE90000E94E00818C20E943C52182F882361F1CA
:10BEA00080917C14811156CD6FEC7CE084E793E1A6
:10BEB00014D98091CE0D882369F063E77CE088E592
:10BEC00090E11FDA612F88E590E106DA88E590E1DC
:10BED0000E94947C812F0E943A8F1A3211F01092A6
:10BEE0007C140E947F936093240D7093250D8093A2
:10BEF000260D9093270DE7C180915D12882309F4E8
:10BF000098C1809167129091681297FF04C01092B7
:10BF1000681210926712809165129091661218163D
:10BF200019069CF42091671230916812281739077E
:10BF300064F010925D12109262128CE291E00E9405
:10BF400051811092681210926712E09169128091EB
:10BF50006412E817D4F18091830D811107C080919C
:10BF60006512909166121816190634F50E947F9397
:10BF700028EE33E040E050E00E94D4A7CA01B901A6
:10BF80000E947AA62091200D3091210D4091220D22
:10BF90005091230D0E9405A820911702309118029C
:10BFA0004091190250911A020E94BBA918160CF078
:10BFB0008AC11092691287C11092621210925D12AA
:10BFC0008CE291E00E9451817EC10E2F0E2E000C5A
:10BFD000110B8AE0E802F0011124EE59FD4EE784CE
:10BFE0000E2C000CFF0880916A12A82E880FBB0847
:10BFF0000E947F934090591250905A1260905B12A9
:10C0000070905C12641975098609970928EE33E06F
:10C0100040E050E00E94D4A7CA01B9010E947AA66C
:10C020002B013C016701F7FE04C0CC24DD24CE18AF
:10C03000DF08C501B7FE02C080E090E08C159D05C9
:10C040000CF096C08AE0809FF001819FF00D1124D2
:10C05000EE59FD4E60897189072E000C880B990BF3
:10C060000E947CA69B01AC01C301B2010E94BBA946
:10C0700018160CF028C1F7FE09C080916712909144
:10C080006812B6010E9441AB892B71F48AE0809F4F
:10C09000F001819FF00D1124EE59FD4E8685082E8A
:10C0A000000C990B0E947C240E947F93609359128C
:10C0B00070935A1280935B1290935C1280916A1273
:10C0C0008F5F80936A12082E000C990B8C159D05CA
:10C0D0000CF4F9C080916412082E000C990B0197A2
:10C0E000081719070CF4EFC080916712909168123D
:10C0F000019690936812809367128091830D81114D
:10C1000008C08091651290916612181619060CF0FD
:10C110008AC28CE291E00E94518168E57CE088E669
:10C1200093E10E9447586091671270916812CE01A6
:10C1300001960E941B72BE016F5F7F4F88E693E1FC
:10C140000E944158CE0101962CD86CED75E080E03C
:10C1500090E00E94479368E673E1CE0101965DD8B6
:10C16000CE0101960E941577CE0101961AD8ABC078
:10C170003AE0F32EF09EF001F19EF00D1124EE59FD
:10C18000FD4E62897389072E000C880B990B0E9463
:10C190007CA69B01AC01C301B2010E94BBA9181689
:10C1A0000CF091C010926A12809169128F5F809397
:10C1B0006912082E000C990B20916412022E000CBB
:10C1C000330B8217930704F5F89EF001F99EF00DEA
:10C1D0001124EE59FD4E878587FD06C08685082E01
:10C1E000000C990B0E947C240E947F93609359124B
:10C1F00070935A1280935B1290935C1280916A1232
:10C200008F5F80936A125FC00E947F9328EE33E0B5
:10C2100040E050E00E94D4A7CA01B9010E947AA66A
:10C220006093200D7093210D8093220D9093230D28
:10C230004AC08091830D882309F4D5C10E947F9361
:10C2400028EEC22E23E0D22EE12CF12CA70196017C
:10C250000E94D4A7CA01B9010E947AA62091200D9C
:10C260003091210D4091220D5091230D0E9405A87F
:10C2700020911702309118024091190250911A0230
:10C280000E94BBA918160CF0AEC10E947F93A701B3
:10C2900096010E94D4A7CA01B9010E947AA66093B0
:10C2A000200D7093210D8093220D9093230D80918A
:10C2B000810D9091820D0E947C2464E170E080E009
:10C2C00090E00E9447938091830D882309F4ABC1CD
:10C2D00064E670E080E090E00E944793A4C182345D
:10C2E00021E09207A105B10509F416C183349140FC
:10C2F000A105B10509F419C1A0CD863421E092074A
:10C30000A105B10509F42CC108F421C1873421E04D
:10C310009207A105B10509F42CC188349140A1050B
:10C32000B10509F42FC189CD823025E09207A1051E
:10C33000B10509F4F1C0E8F4843721E09207A105C2
:10C34000B10509F434C138F482379140A105B10533
:10C3500009F436C172CD811525E09207A105B1051A
:10C3600009F4C8C081309540A105B10509F4CBC0DE
:10C3700064CD853025E09207A105B10509F4E7C039
:10C3800070F4833025E09207A105B10509F4CDC012
:10C3900084309540A105B10509F4D0C04ECD86305A
:10C3A00025E09207A105B10509F4DAC08730954070
:10C3B000A105B10509F4DDC040CD8D3B22E4920713
:10C3C0002FEFA207B10509F4FEC008F045C08F3E6B
:10C3D00020E192072FEFA207B10509F4CAC0E8F4E3
:10C3E000823325E09207A105B10509F4E9C038F4CC
:10C3F00089309540A105B10509F4CDC01ECD843327
:10C4000025E09207A105B10509F4D1C08D3F924006
:10C41000AF4FB10509F417CD10CD8D3D22E2920743
:10C420002FEFA207B10509F4C2C038F4873E984146
:10C43000AF4FB10509F48BC000CD8F3C20E39207CC
:10C440002FEFA207B10509F479C0873C9843AF4F9D
:10C45000B10509F497C0F1CC873928E692072FEF90
:10C46000A207B10509F44FC000F58D3A22E5920705
:10C470002FEFA207B10509F4E6CC30F4853B9A44CE
:10C48000AF4FB105B9F1D9CC853A2AE592072FEF24
:10C49000A207B10509F47FC08D399246AF4FB105AF
:10C4A00009F0CBCC87EE9FEFF6CB873528EA9207D1
:10C4B0002FEFA207B10509F477C070F485382AE799
:10C4C00092072FEFA207B10509F44AC087369849B1
:10C4D000AF4FB10509F1B1CC8F3420EB92072FEFAC
:10C4E000A207B10511F18D33924CAF4FB10509F49C
:10C4F00067C0A3CC68E17CE084E793E10E946D58BB
:10C500008AEF9FEFC8CB6BE17CE084E793E10E9468
:10C510006D5889EF9FEFBFCB6EE17CE084E793E13C
:10C520000E946D5888EF9FEFB6CB61E27CE084E714
:10C5300093E10E946D5887EF9FEFADCB64E27CE002
:10C5400084E793E10E946D5886EF9FEFA4CB68E2E9
:10C550007CE084E793E10E946D5885EF9FEF9BCBD1
:10C560006CE27CE084E793E10E946D5884EF9FEFDA
:10C5700092CB60E37CE084E793E10E946D5883EF07
:10C580009FEF89CB64E37CE084E793E10E946D58E0
:10C5900082EF9FEF80CB68E37CE084E793E10E9429
:10C5A0006D5881EF9FEF77CB86EE9FEF74CB6CE3F6
:10C5B0007CE080E893E10E946D5888EE9FEF6BCBA2
:10C5C00089EE9FEF68CB60E47CE080E893E10E9415
:10C5D0006D5884E190E05FCB6EE170E080E090E028
:10C5E0000E94479348CB0E947F930091240D1091A5
:10C5F000250D2091260D3091270DDC01CB01801BEC
:10C60000910BA20BB30B88349E4EA105B10508F423
:10C610005ACE10926E1460E083E694E10E94B88CCA
:10C620001092DC0450CE26960FB6F894DEBF0FBEF3
:10C63000CDBFDF91CF911F910F91FF90EF90DF90D1
:10C64000CF90BF90AF907F906F905F904F90089584
:10C65000BF92CF92DF92EF92FF920F931F93CF93EF
:10C66000DF93CDB7DEB762970FB6F894DEBF0FBE8B
:10C67000CDBF8C016B0167E67CE0CE010D960E9478
:10C68000155963E47CE0C8010E94055976012FEF3B
:10C69000E21AF20AB701CE0101960E941B72BE0196
:10C6A0006F5F7F4FCE0107960E940D5962EF78E0D1
:10C6B000CE0107960E940B58BC01C8010E94415848
:10C6C000CE0107960E94D158CE0101960E94D15802
:10C6D0008AE0B82EBE9CC001BF9C900D1124FC01C5
:10C6E000EE59FD4E7F018081082E000C990B0E94AF
:10C6F000ABAD892B09F4B2C0B701CE0101960E94FF
:10C700001559BE016F5F7F4FCE0107960E940D59EC
:10C7100067EC76E0CE0107960E940B58BC01C80179
:10C720000E944158CE0107960E94D158CE01019631
:10C730000E94D158BC9CC001BD9C900D11249C014D
:10C740002E593D4E7901F9016685062E000C770BB6
:10C75000CE0101960E941B72BE016F5F7F4FCE011A
:10C7600007960E940D5962E57CE0CE0107960E9473
:10C770000B58BE01635F7F4F0E942258BC01C80165
:10C780000E944158CE0107960E94D158CE010196D1
:10C790000E94D1586CE37CE0C8010E94AF57F701BA
:10C7A0006785062E000C770BCE0101960E941B7246
:10C7B000BE016F5F7F4FCE0107960E940D59BE01EB
:10C7C000635F7F4FCE0107960E942258BC01C801CB
:10C7D0000E944158CE0107960E94D158CE01019681
:10C7E0000E94D15866E37CE0C8010E94AF57F70170
:10C7F00060897189CE0101960E941B72BE016F5F34
:10C800007F4FCE0107960E940D59BE01635F7F4F97
:10C81000CE0107960E942258BC01C8010E944158CF
:10C82000CE0107960E94D158CE0101960E94D158A0
:10C8300061E37CE0C8010E94AF57F7016289738908
:10C84000CE0101960E941B72BE016F5F7F4FC8012F
:10C850000E944158CE0101960E94D158CE010D96FA
:10C860000E94D158C80162960FB6F894DEBF0FBE81
:10C87000CDBFDF91CF911F910F91FF90EF90DF908F
:10C88000CF90BF900895EF92FF920F931F93CF9395
:10C89000DF93CDB7DEB768970FB6F894DEBF0FBE53
:10C8A000CDBF8C0167E67CE0CE010D960E94155944
:10C8B00064E57CE0CE0143960E9415596DE07CE072
:10C8C000C8010E940559BE016D5E7F4FC8010E94DC
:10C8D000415864E07CE0C8010E94AF5782E6E82E30
:10C8E00082E1F82EF701608170E0CE0101960E948E
:10C8F0001B72BE016F5F7F4FCE0107960E940D59DC
:10C90000BE01635F7F4FCE0107960E942258BC0193
:10C91000C8010E944158CE0107960E94D158CE010D
:10C9200001960E94D15867EF7BE0C8010E94AF5783
:10C93000F7016181062E000C770BCE0101960E9453
:10C940001B72BE016F5F7F4FCE0107960E940D598B
:10C95000BE01635F7F4FCE0107960E942258BC0143
:10C96000C8010E944158CE0107960E94D158CE01BD
:10C9700001960E94D1586DEE7BE0C8010E94AF572E
:10C98000F7016281062E000C770BCE0101960E9402
:10C990001B72BE016F5F7F4FCE0107960E940D593B
:10C9A000BE01635F7F4FCE0107960E942258BC01F3
:10C9B000C8010E944158CE0107960E94D158CE016D
:10C9C00001960E94D15865EE7BE0C8010E94AF57E6
:10C9D000F70163817481CE0101960E941B72BE0132
:10C9E0006F5F7F4FCE0107960E940D59BE016D5EAD
:10C9F0007F4FCE0107960E942258BC01C8010E94B9
:10CA00004158CE0107960E94D158CE0101960E944E
:10CA1000D1586EEC7BE0C8010E94AF57F7016581E9
:10CA20007681CE0101960E941B72BE016F5F7F4F1F
:10CA3000CE0107960E940D59BE01635F7F4FCE0164
:10CA400007960E942258BC01C8010E944158CE019D
:10CA500007960E94D158CE0101960E94D15865ECEC
:10CA60007BE0C8010E94AF57F7016781062E000CDA
:10CA7000770B6F5F7F4FCE0101960E941B72BE0144
:10CA80006F5F7F4FCE0107960E940D59BE01635F15
:10CA90007F4FCE0107960E942258BC01C8010E9418
:10CAA0004158CE0107960E94D158CE0101960E94AE
:10CAB000D1586AEB7BE0C8010E94AF57F70160854F
:10CAC000062E000C770BCE0101960E941B72BE0150
:10CAD0006F5F7F4FC8010E944158CE0101960E94AE
:10CAE000D158CE0143960E94D158CE010D960E9496
:10CAF000D158C80168960FB6F894DEBF0FBECDBFFF
:10CB0000DF91CF911F910F91FF90EF9008957F9249
:10CB10008F929F92AF92BF92CF92DF92EF92FF924D
:10CB20000F931F93CF93DF93782E8AE0A82EB12C1A
:10CB3000EE24EA9493E0F92E88248A9423E0922E3E
:10CB400000E010E0C12CD12CC0E0D0E0872D0E9485
:10CB5000FD92C816D90628F00817190718F48C0199
:10CB600001C06C018815990528F08E159F0518F4F1
:10CB70007C0101C04C01C80FD91F65E070E080E066
:10CB800090E00E94479381E0A81AB108F9F60C0DD5
:10CB90001D1DCE01801B910B8E199F0988199909C3
:10CBA00066E070E00E942DABCB01DF91CF911F9129
:10CBB0000F91FF90EF90DF90CF90BF90AF909F903C
:10CBC0008F907F9008954F925F926F927F92AF9275
:10CBD000BF92CF92DF92FF920F931F93CF93DF9379
:10CBE00000D000D0CDB7DEB75C018BEB9FE00E9498
:10CBF000746E40E052EC61E070E08BEB9FE00E94CD
:10CC0000A1808CED95E0A0E0B0E08093BF0F909301
:10CC1000C00FA093C10FB093C20F64E670E080E034
:10CC200090E00E944793C12CD12CF12CCA14DB0454
:10CC30000CF051C065E070E080E090E00E94479306
:10CC400000E010E0412C512C3201F1100FC08BEBB1
:10CC50009FE00E949D54892B31F485E148165104D0
:10CC6000610471041CF40330110554F08FEFC81AED
:10CC7000D80A64E670E080E090E00E944793D6CF47
:10CC80008BEB9FE00E949D54892B69F08BEB9FE01A
:10CC90000E947B54E1E0F0E0EC0FFD1FE00FF11F7C
:10CCA00080830F5F1F4F65E070E080E090E00E949E
:10CCB0004793023011054CF089818B3B31F4FF24FE
:10CCC000F3948A818A3A09F0F12C8FEF481A580AB6
:10CCD000680A780ABACF8F2D26960FB6F894DEBF71
:10CCE0000FBECDBFDF91CF911F910F91FF90DF90CD
:10CCF000CF90BF90AF907F906F905F904F900895CE
:10CD00001F93CF93DF93182FC7EEDDE0812F0E9492
:10CD1000FD92899399936CE370E080E090E00E942B
:10CD200047938EE0C733D80789F70E949D7E20E0A5
:10CD300030E040EA50E40E94DBA620E030E040E82A
:10CD40005AE30E94DBA6DF91CF911F910895AF9225
:10CD5000BF92CF92DF92EF92FF920F931F93CF93E8
:10CD6000DF93CDB7DEB72C970FB6F894DEBF0FBEBA
:10CD7000CDBF8091830D811102C00E94A48180915A
:10CD8000910490919204029751F08091510D9091ED
:10CD9000520D009709F48BC1039709F488C168EA22
:10CDA0007CE082E693E10E94475862E673E1CE019F
:10CDB00001960E940D5944E150E060E070E0CE0120
:10CDC00001960E948773CE0101960E94D15869E9AD
:10CDD0007CE082E693E10E94475862E673E1CE016F
:10CDE00001960E940D5944E150E06FEF7FEFCE01B4
:10CDF00001960E94D381CE0101960E94D15887E00E
:10CE00000E94AA4F8C0186E00E94AA4FBC0180E0DC
:10CE100090E00E947AA62AE037ED43EA5CE30E94A4
:10CE2000DBA623E333E948E853E40E9405A86B013D
:10CE30007C0184E0A82EB12C20E030E048EC52E4E4
:10CE4000C701B6010E94BBA9181614F581E0A81A03
:10CE5000B10809F4F2C064E670E080E090E00E945E
:10CE6000479386E00E94AA4FBC0180E090E00E94B8
:10CE70007AA62AE037ED43EA5CE30E94DBA623E3CF
:10CE800033E948E853E40E9405A86B017C01D4CF44
:10CE9000B80180E090E00E947AA62AE037ED43EAEC
:10CEA0005CE30E94DBA623E333E948E853E40E94F5
:10CEB00005A8AB01BC0121E0CE0101960E94D65825
:10CEC00069E67CE0CE0107960E941559BE016F5FAE
:10CED0007F4FCE0107960E942258BC0188E693E15D
:10CEE0000E948258CE0107960E94D158CE01019629
:10CEF0000E94D15868E673E1CE0101960E940D5957
:10CF000042E350E06FEF7FEFCE0101960E94D381A4
:10CF1000CE0101960E94D15863E77CE0CE010196D4
:10CF20000E941559CE010196C1D6CE0101960E94EC
:10CF3000D15862E77CE088E693E10E94335821E013
:10CF4000B701A601CE0101960E94D65860EF7BE0A2
:10CF5000CE0107960E941559BE016F5F7F4FCE012B
:10CF600007960E942258BC018EE693E10E948258E7
:10CF7000CE0107960E94D158CE0101960E94D15849
:10CF800067E67CE0CE0101960E9415596EE673E1DA
:10CF9000CE0101960E942258BC0182E693E10E94D4
:10CFA0008258CE0101960E94D15862E673E1CE010B
:10CFB00001960E940D594AE050E060E070E0CE0119
:10CFC00001960E942C74CE0101960E94D15863E70D
:10CFD0007CE0CE0101960E941559CE01019666D6DD
:10CFE000CE0101960E94D15862E77CE08EE693E183
:10CFF0000E9433586EE673E1CE0101960E940D59EE
:10D0000067E67CE0CE0101960E940B5868E673E16A
:10D010000E942258BC0188E693E10E948258CE010A
:10D0200001960E94D1588091510D9091520D039715
:10D0300009F002C184E090E0FBC06EE87CE082E68B
:10D0400093E10E94475862E673E1CE0101960E9487
:10D050000D594AE050E060E070E0CE0101960E9478
:10D060008773CE0101960E94D15867E57CE0CE011E
:10D0700001960E94155962E673E1CE0101960E9465
:10D080002258BC0188E693E10E948258CE010196A5
:10D090000E94D1588091510D9091520D049721F426
:10D0A0001092520D1092510D81E090E014C18EE16A
:10D0B0009FE01AD664E670E080E090E00E9447931B
:10D0C0006EEC7CE082E693E10E94475862E673E1F1
:10D0D000CE0101960E940D5944E150E060E070E0FD
:10D0E000CE0101960E948773CE0101960E94D1580D
:10D0F0006FEB7CE082E693E10E94475862E673E1C1
:10D10000CE0101960E940D5944E150E06FEF7FEF90
:10D11000CE0101960E94D381CE0101960E94D15882
:10D120008CE400D66B017C0104E010E0A7019601BD
:10D13000C701B6010E9405AB811190C021E0B70183
:10D14000A601CE0107960E94D65869E67CE0CE0182
:10D1500001960E941559BE01695F7F4FCE0101966D
:10D160000E942258BC0188E693E10E948258CE01B9
:10D1700001960E94D158CE0107960E94D15868E6C8
:10D1800073E1CE0101960E940D5942E350E06FEF2A
:10D190007FEFCE0101960E94D381CE0101960E94BD
:10D1A000D15863E77CE0CE0101960E941559CE016B
:10D1B00001967CD5CE0101960E94D15862E77CE0B1
:10D1C00088E693E10E94335886E6ACD56B017C017A
:10D1D00004E010E0A7019601C701B6010E9405AB6B
:10D1E000882309F47DC00150110909F0E0C06FECFB
:10D1F0007CE08EE693E10E946D586EE673E1CE010D
:10D2000001960E940D5967E67CE0CE0101960E94CE
:10D210000B5868E673E10E942258BC0188E693E14E
:10D220000E948258CE0101960E94D15883E090E07E
:10D230009093520D8093510D64E670E080E090E091
:10D240000E9447938091830D882309F4BBC060E25C
:10D2500073E080E090E00E944793B4C00150110950
:10D2600009F09AC064EB7CE082E693E10E944758A3
:10D2700062E673E1CE0101960E940D594AE050E04A
:10D2800060E070E0CE0101960E948773CE010196A6
:10D290000E94D15867E57CE0CE0101960E941559A5
:10D2A00062E673E1CE0101960E942258BC0188E635
:10D2B00093E10E948258CE0101960E94D15880913C
:10D2C000510D9091520D039721F41092520D10922E
:10D2D000510D82E090E09093920480939104ACCF42
:10D2E00021E0B701A601CE0107960E94D65860EF53
:10D2F0007BE0CE0101960E941559BE01695F7F4F08
:10D30000CE0101960E942258BC018EE693E10E9454
:10D310008258CE0101960E94D158CE0107960E94F4
:10D32000D15867E67CE0CE0101960E9415596EE661
:10D3300073E1CE0101960E942258BC0182E693E17E
:10D340000E948258CE0101960E94D15862E673E194
:10D35000CE0101960E940D594AE050E06FEF7FEF39
:10D36000CE0101960E942C74CE0101960E94D158E4
:10D3700063E77CE0CE0101960E941559CE0101962B
:10D3800095D4CE0101960E94D15862E77CE08EE6EA
:10D3900093E10E94335831CF68EC70E080E090E078
:10D3A0000E9447938CE4BED46B017C01BFCE68EC35
:10D3B00070E080E090E00E94479386E6B3D46B0172
:10D3C0007C0108CF2C960FB6F894DEBF0FBECDBF00
:10D3D000DF91CF911F910F91FF90EF90DF90CF9051
:10D3E000BF90AF9008952F923F924F925F926F92AD
:10D3F0007F928F929F92AF92BF92CF92DF92EF92E5
:10D40000FF920F931F93CF93DF93CDB7DEB7C55431
:10D41000D1090FB6F894DEBF0FBECDBF2B013C0182
:10D4200069017A010E947F9322966CAF7DAF8EAF27
:10D430009FAF229720E9421621E052066104710451
:10D4400034F090E9492E55245394612C712C30E12D
:10D45000C31637E2D306E104F1042CF4CDA6DEA610
:10D46000EFA6F8AA08C080E197E2A0E0B0E08DA79F
:10D470009EA7AFA7B8AB8091830D882321F0CDA6DE
:10D48000DEA6EFA6F8AA22966CAD7DAD8EAD9FAD5F
:10D49000229728EE33E040E050E00E94A8A72696AD
:10D4A0002CAF3DAF4EAF5FAF269791E09DAB19A675
:10D4B0001AA61BA61CA68E01035F1F4FCC24DD24D9
:10D4C0007601C418D508E608F708C9AADAAAEBAAB3
:10D4D000FCAAC9A4DAA4EBA4FCA42DA53EA54FA5E3
:10D4E00058A9C216D306E406F5060CF02AC3C701F4
:10D4F000B6010E947CA620E030E04AE754E40E9496
:10D50000CCA8AB01BC0123E0C8010E94D658B801E9
:10D5100082E693E10E949758C8010E94D1588DA5D8
:10D520009EA5AFA5B8A90A97A105B1058CF42696CA
:10D530004CAD5DAD6EAD7FAD2697C8010E94527DAA
:10D54000B80182E693E10E949758C8010E94D15821
:10D55000CE0101960E94464F61E87CE088E693E1A7
:10D560000E944758DE0111961D01C12CD12C760175
:10D57000F10181909190A190B1901F01A5019401BA
:10D58000C501B4010E94DBA69B01AC01C701B60135
:10D590000E9406A86B017C0123E0B501A401C8012B
:10D5A0000E94D658B801CE0143960E940D5967E6F5
:10D5B0007CE0CE0143960E940B58BC0188E693E1C3
:10D5C0000E944158CE0143960E94D158C8010E9442
:10D5D000D1580215130561F6C701B6010E94C4AA0D
:10D5E0006B017C01FDE24F16F1E05F0661047104FE
:10D5F00034F00E94A48160E080E00E94277D23E057
:10D60000B701A601CE0143960E94D65865E77CE09B
:10D61000C8010E94155962E673E1C8010E942258B0
:10D6200068E77CE00E940B58BE016D5E7F4F0E9450
:10D6300022586DE77CE00E940B58BC0188E693E11C
:10D640000E944158C8010E94D158CE0143960E94C1
:10D65000D1582DEC3CEC4CE45FE3C701B6010E94CD
:10D66000BBA929813A814B815C812DA33EA34FA3A5
:10D6700058A718160CF0A9C12AE939E949E95FE36E
:10D68000C701B6010E9476A687FF9FC1CDA8CC2016
:10D6900009F49BC189849A84AB84BC8420E030E087
:10D6A000A901C501B4010E9476A6CD80DE80EF807D
:10D6B000F884882309F12DA13EA14FA158A5CA01E4
:10D6C000B9010E94DBA66EAB7FAB88AF99AFA70113
:10D6D0009601C701B6010E94DBA69B01AC016EA9B1
:10D6E0007FA988AD99AD0E9406A80E94C4AAA50191
:10D6F00094010E9479A804C06BED7FE089EC9FE360
:10D7000020EE3EE245E652E40E94DBA66EAB7FAB24
:10D7100088AF99AF20E030E0A901C701B6010E94AF
:10D7200076A6882309F12DA13EA14FA158A5CA01D3
:10D73000B9010E94DBA66AAF7BAF8CAF9DAFA5019C
:10D740009401C501B4010E94DBA69B01AC016AAD46
:10D750007BAD8CAD9DAD0E9406A80E94C4AAA70116
:10D7600096010E9479A804C06BED7FE089EC9FE3ED
:10D7700020EE3EE245E652E40E94DBA66AAF7BAFB4
:10D780008CAF9DAF20E030E0A9016DA17EA18FA1FB
:10D7900098A50E9476A68823F9F0A5019401C501F9
:10D7A000B4010E94DBA64B015C01A7019601C701F1
:10D7B000B6010E94DBA69B01AC01C501B4010E9429
:10D7C00006A80E94C4AA2DA13EA14FA158A50E945F
:10D7D00079A86B017C0108C08BEDC82E8FE0D82E94
:10D7E00089ECE82E8FE3F82E66E77CE0C8010E9402
:10D7F000155962E673E1C8010E94225860E87CE096
:10D800000E940B58BC0188E693E10E948258C8012F
:10D810000E94D15866E77CE0C8010E94155962E673
:10D8200073E1C8010E9422586AE97CE00E940B580B
:10D83000BC0182E693E10E948258C8010E94D1583F
:10D8400021E04EA95FA968AD79ADCE014F960E9447
:10D85000D65821E04AAD5BAD6CAD7DADCE014996A9
:10D860000E94D65820EE3EE245E652E4C701B601DA
:10D870000E94DBA6AB01BC0121E0C8010E94D65882
:10D88000B801CE0143960E940D5967E67CE0CE01B7
:10D8900043960E940B58BE01675E7F4F0E9422583C
:10D8A00067E67CE00E940B58BE01615E7F4F0E94DC
:10D8B0002258BC018CE593E10E948258CE01439628
:10D8C0000E94D158C8010E94D158CE0149960E94A9
:10D8D000D158CE014F960E94D1582DE2421621E038
:10D8E00052066104710474F469A57AA58BA59CA500
:10D8F00025E030E040E050E00E94A8A7672B682BAD
:10D90000692BA9F562E673E1C8010E940D5945E053
:10D9100050E06FEF7FEFC8019FD7C8010E94D15838
:10D9200063EA7CE0C8010E94155945E050E061EFD0
:10D930007FEFC801ECD6C8010E94D1586FEC7CE0A3
:10D94000C8010E941559C801B1D1C8010E94D1581F
:10D950006CE573E1C8010E940D5945E050E060E0BC
:10D9600070E0C8010E94D381C8010E94D1586CE5C3
:10D9700073E188E693E10E9441583FE14316510468
:10D980006104710434F4C9A4DAA4EBA4FCA4F7FC88
:10D9900011C068E673E1C8010E940D59C8010E94D8
:10D9A0001577C8010E94D1586FEC7CE088E693E1BE
:10D9B0000E946D58B201C30177FE04C069A97AA91B
:10D9C0008BA99CA90E944793A9C023E04DA15EA109
:10D9D0006FA178A5CE0143960E94D65866E77CE0F9
:10D9E000C8010E94155962E673E1C8010E942258DD
:10D9F00065EA7CE00E940B58BE016D5E7F4F0E947D
:10DA000022586EE77CE00E940B58BC0182E693E14D
:10DA10000E948258C8010E94D158CE0143960E94AC
:10DA2000D15849855A856B857C8523E0CE0149967E
:10DA30000E94D6584D815E816F81788523E0C801B0
:10DA40000E94D658B801CE0143960E940D596AEA49
:10DA50007CE0CE0143960E940B58BE01675E7F4F6B
:10DA60000E9422586EE77CE00E940B58BC018CE5B6
:10DA700093E10E948258CE0143960E94D158C8017A
:10DA80000E94D158CE0149960E94D1582DE24216EB
:10DA900021E052066104710474F469A57AA58BA58E
:10DAA0009CA525E030E040E050E00E94A8A7672B4D
:10DAB000682B692BE9F462E673E1C8010E940D59F5
:10DAC0004AE050E06FEF7FEFC801C6D6C8010E9460
:10DAD000D1586CE573E1C8010E940D594AE050E04D
:10DAE00060E070E0C8010E94D381C8010E94D15853
:10DAF00068E673E1C8010E940D59C8010E941577BC
:10DB0000C8010E94D1586FEC7CE088E693E10E9446
:10DB10006D58C301B2010E9447931DAA0E947F93D2
:10DB20006B017C0122962CAD3DAD4EAD5FAD2297D1
:10DB3000C21AD30AE40AF50AC9A6DAA6EBA6FCA61D
:10DB4000C8CC62E673E1CE010D960E940D594AE001
:10DB500050E06FEF7FEFCE010D96D9D5CE010D9637
:10DB60000E94D158CDA8CC2099F163EA7CE0CE0187
:10DB70000D960E94155945E050E061EF7FEFCE0110
:10DB80000D96C5D5CE010D960E94D1588091830D7A
:10DB9000882389F069E77CE0CE010D960E94055943
:10DBA00045E050E060E070E0CE010D96B0D5CE01CA
:10DBB0000D960E94D1586FEC7CE0CE010D960E942C
:10DBC0001559CE010D9672D0CE010D960E94D158F6
:10DBD0006CE573E1CE010D960E940D594AE050E0CC
:10DBE0006FEF7FEFCE010D960E94D381CE010D968F
:10DBF0000E94D158CB5BDF4F0FB6F894DEBF0FBE4B
:10DC0000CDBFDF91CF911F910F91FF90EF90DF90EB
:10DC1000CF90BF90AF909F908F907F906F905F90CC
:10DC20004F903F902F90089590915D0E9111FCCFF1
:10DC300091E090935D0E90935C0E2FEF20935B0E1E
:10DC400010925A0E260F2093590E9093380E9091F1
:10DC5000380E880F892B8093380E8091370E8130D3
:10DC600061F41092370E8091380E8093BB00809142
:10DC7000BC0083FDF8CF85EC01C085EE8093BC002D
:10DC800080915D0E8130E1F380915A0E861710F479
:10DC900060915A0EA9E3BEE0EAEAFDE080E0861753
:10DCA00021F09D9191938F5FFACF0895CF93DF93E9
:10DCB0002091DD042223A9F02091DC04222389F0A5
:10DCC000EC016FED83E694E10E946C598C819D819B
:10DCD000892B39F0BE0183E694E1DF91CF910C945A
:10DCE0007359DF91CF910895CF93DF93EC010E9498
:10DCF0003B55EA89FB8980818F7E8083EA89FB8995
:10DD00008081877F8083EA89FB8980818F77808308
:10DD1000EA89FB8980818F7D80838A8D898FDF915D
:10DD2000CF9108953F924F925F926F927F928F9220
:10DD30009F92AF92BF92CF92DF92EF92FF920F939A
:10DD40001F93CF93DF9300D01F921F92CDB7DEB702
:10DD5000982E0E947F932B013C0120ED420E27E07C
:10DD6000521E611C711C60E080914D140E949392C0
:10DD700045E0842ECE0101966C01AA24A394B12C17
:10DD8000F601282D11922A95E9F7860135E0332E08
:10DD900027E0E22EF12C80914E140E946B920197A5
:10DDA00039F40E947F93641575058605970598F3ED
:10DDB00080914E140E946B92892B39F40E947F93BC
:10DDC000641575058605970598F380914F140E9498
:10DDD0006B92892B51F0F8012081C5010E2C01C0F6
:10DDE000880F0A94EAF7822B8083F1E0EF1AF1089A
:10DDF00090F63A940F5F1F4F3110CACF0E947F9365
:10DE0000641575058605970550F061E080914D1405
:10DE10000E94939260E070E080EC9FE72CC08981C3
:10DE20008911AECF9A818B81890F890D9C818913CD
:10DE3000A7CF8D818D3009F0A3CF61E080914D1483
:10DE40000E9493926A818B8170E0762F6627680F1B
:10DE5000711D072E000C880B990B0E947CA620E0F8
:10DE600030E040E85DE30E94DBA623E333E948E8C5
:10DE700053E40E9405A80F900F900F900F900F9001
:10DE8000DF91CF911F910F91FF90EF90DF90CF9096
:10DE9000BF90AF909F908F907F906F905F904F90CA
:10DEA0003F900895613208F060E2BEDE1092A90D45
:10DEB0008093A80D0895CF93C82F87E70E940C7D0B
:10DEC0006C2F85EF90E10E94D38B0E94057D87E740
:10DED0000E940C7D61E070E087E790E0E3DF85EF72
:10DEE00090E10E948B8BC82F0E94057D8C2FCF91D3
:10DEF0000895CF93DF93C82F87E70E940C7D6C2F86
:10DF000085EF90E10E94D38B0E94057D87E70E94F8
:10DF10000C7D62E070E087E790E0C4DF85EF90E180
:10DF20000E948B8BD82F80E0C82F85EF90E10E9454
:10DF30008B8BC82BD92B0E94057DCE01DF91CF9111
:10DF4000089587E70E940C7D64EF85EF90E10E94C1
:10DF5000D38B6EE285EF90E10E94D38B0E94057D0A
:10DF600065E070E080E090E00E94479386EFC1CFCB
:10DF70004F925F926F927F928F929F92AF92BF92D9
:10DF8000CF92DF92EF92FF920F931F93CF93DF9385
:10DF900000D01F921F92CDB7DEB7D3DF4C01A12C6A
:10DFA000B12C209186132295220F220F207C2C5C0D
:10DFB000298387E70E940C7D64EF85EF90E10E9442
:10DFC000D38B698185EF90E10E94D38B0E94057D00
:10DFD00080918613811105C065E070E080E090E0DB
:10DFE00012C0813029F468E070E080E090E00BC05E
:10DFF000823029F46EE070E080E090E004C06AE1D5
:10E0000070E080E090E00E94479386EF72DF6C0141
:10E01000E12CF12CFE2CED2CDC2CCC2488EF4BDFFA
:10E02000C82A309186133D8380919B1390919C1355
:10E03000A5019401281B390B41095109A09199139D
:10E04000B0919A130E94C4A72B013C01AFE07594D4
:10E05000679457944794AA95D1F760919313709160
:10E060009413CB01770FAA0BBB0BBC01CD01BBE016
:10E07000660F771F881F991FBA95D1F720919513C6
:10E08000309196138901330F220B330BA9019801AC
:10E09000240D351D461D571D0E94A8A7420E531E74
:10E0A000641E751E40EA441A4FE0540A6108710864
:10E0B000A3019201C301B2010E941EAB9B01AC01FE
:10E0C0001CE055954795379527951A95D1F72983E3
:10E0D0003A834B835C83E0918713F0918813A0917E
:10E0E0008B13B0918C13A30192010E94CEA74B0118
:10E0F0005C010DE0B594A794979487940A95D1F7A5
:10E10000A0918D13B0918E1329813A814B815C814E
:10E110000E94CEA7BB2797FDB095AB2F880D991D08
:10E12000AA1DBB1D0296A11DB11D32E0B595A79594
:10E13000979587953A95D1F79C01AD0130584F4F8F
:10E140005F4FA0919713B09198130E94C4A74B0101
:10E150005C014FE0B694A794979487944A95D1F7C1
:10E1600088E090E03D81831B910904C0F694E79418
:10E17000D794C7948A95D2F7A0918F13B09190133A
:10E1800029813A814B815C810E94CEA79B01AC0121
:10E190006BE055954795379527956A95D1F7298373
:10E1A0003A834B835C83A0918913B0918A13A301B6
:10E1B00092010E94CEA7DC01CB017BE0B595A7952B
:10E1C000979587957A95D1F749815A816B817C81A2
:10E1D000480F591F6A1F7B1FCF01FF0FAA0BBB0BF4
:10E1E000E2E0880F991FAA1FBB1FEA95D1F7840FA1
:10E1F000951FA61FB71F0D8004C0880F991FAA1F67
:10E20000BB1F0A94D2F7BC01CD016E5F7F4F8F4FC9
:10E210009F4F24E030E040E050E00E94A8A7D701E3
:10E22000C601821B930BA40BB50B9C01AD0180E5CD
:10E2300093ECA0E0B0E0BC01CD010D8004C0969548
:10E240008795779567950A94D2F70E941EAB97FD44
:10E250000BC0660F771F881F991FA50194010E94AC
:10E26000D4A749015A010AC0A50194010E94D4A76C
:10E2700049015A01880C991CAA1CBB1C9927B7FCA0
:10E280009A958B2D7A2D692D9B01AC010E941EABB6
:10E290009B01AC01AEEDBBE00E94C4A76B017C0109
:10E2A000A3E4B3EEA50194010E94D0A7BB2797FD7C
:10E2B000B095AB2F6701FF24D7FCF094EF2C8C0DA9
:10E2C0009D1DAE1DBF1D8153914FAF4FBF4F44E009
:10E2D000B595A795979587954A95D1F7BC01CD013E
:10E2E000680D791D8A1D9B1D0F900F900F900F9048
:10E2F0000F90DF91CF911F910F91FF90EF90DF90E2
:10E30000CF90BF90AF909F908F907F906F905F90D5
:10E310004F900895CF92DF92EF92FF920F931F9349
:10E3200010DEAC0160E070E0E6E8F3E185899689F3
:10E330009A01AB01281B390B41095109A389B48902
:10E340000E94C4A76B017C018FE0F594E794D794F9
:10E35000C7948A95D1F765857685CB01770FAA0B8F
:10E36000BB0BBC01CD012BE0660F771F881F991FE7
:10E370002A95D1F7278530898901330F220B330B7A
:10E38000A90198012C0D3D1D4E1D5F1D0E94A8A7DF
:10E39000DA01C9018C0D9D1DAE1DBF1D0896A11D82
:10E3A000B11DBC01CD0134E09595879577956795B2
:10E3B0003A95D1F70E947CA620E030E040E251E49B
:10E3C0000E94CCA81F910F91FF90EF90DF90CF900B
:10E3D00008951092A90D1092A80D10925F0E109240
:10E3E000800E10925D0E81E080935C0E1092370ECD
:10E3F00061E084E10E94939261E085E10E94939242
:10E40000E9EBF0E080818E7F808380818D7F808347
:10E4100088E48093B80085E48093BC0089E79BE89A
:10E420009093A70D8093A60D8AE79BE89093A50D86
:10E430008093A40D08950F931F93CF93DF93CDB7CF
:10E44000DEB762970FB6F894DEBF0FBECDBF8C016A
:10E45000CB01F8011182108213821282158214827C
:10E460004AE0BE016F5F7F4F0E9436A2BE016F5F20
:10E470007F4FC8010E946D5862960FB6F894DEBFB8
:10E480000FBECDBFDF91CF911F910F9108956132E3
:10E4900008F060E2C9DB1092A90D8093A80D0895E1
:10E4A000AF92BF92CF92DF92EF92FF920F931F93A2
:10E4B000CF93DF93C82FD62F1092C4131092C51399
:10E4C0001092C6131092C7131092C81361E00E94F5
:10E4D000C19260E08C2F0E9493926D2F70E080E0DB
:10E4E00090E00E94479360E08C2F0E94C1928BE9DC
:10E4F00090E00197F1F700E911E08C2F0E946B92F8
:10E50000892B31F401501109C1F78EEF9FEF4CC0F8
:10E5100000E911E08C2F0E946B92019709F43FC033
:10E5200018E2D0E800E090E9E92EFF24F3948C2F64
:10E530000E946B92892B29F481E0E81AF108B9F75F
:10E54000E4CF0E9422936B017C0180E9A82EBB24BA
:10E55000B3948C2F0E946B92019729F481E0A81A42
:10E56000B108B9F7D2CF0E942293DC01CB018C19FC
:10E570009D09AE09BF098997A105B10538F0E02FC3
:10E58000F0E0E454FC4E80858D2B8087D69511F405
:10E590000F5FD0E8115039F680E090E005C00150DF
:10E5A000110909F0B7CFB1CFDF91CF911F910F9132
:10E5B000FF90EF90DF90CF90BF90AF900895EF92D3
:10E5C000FF920F931F93CF93DF93C82F8B017A0194
:10E5D00083E50E940C7D6C2F85EF90E10E94D38B28
:10E5E0000E94057D83E50E940C7DB80183E590E0E3
:10E5F00059DCE701CE018E199F093091A80D2091B9
:10E60000A90D321731F085EF90E10E948B8B899331
:10E61000F1CF0817190729F01092CA1381E08093EF
:10E62000CB13DF91CF911F910F91FF90EF900C943E
:10E63000057DCF93DF934AE050E0BC0188E590E18F
:10E640000E94025AEC0188E590E10E94947C8C0FB4
:10E650009D1FDF91CF9108951F93CF93DF931F925A
:10E66000CDB7DEB7162FAE014F5F5F4F61E070E0B0
:10E67000A6DF898190E002C0959587951A95E2F70B
:10E6800081700F90DF91CF911F910895CF93DF9309
:10E69000D82FC62F83E50E940C7D6D2F85EF90E16A
:10E6A0000E94D38B6C2F85EF90E10E94D38BDF917A
:10E6B000CF910C94057D0F931F93CF93DF9300D0E0
:10E6C00000D0CDB7DEB72091CE0D2223A9F08C016A
:10E6D00065E57CE0CE0101960E941559B801CE0196
:10E6E00001960E942258BC0188E590E10E94987C26
:10E6F000CE0101960E94D15826960FB6F894DEBF3F
:10E700000FBECDBFDF91CF911F910F910895BF92A2
:10E71000CF92DF92EF92FF920F931F93CF93DF93ED
:10E72000CDB7DEB762970FB6F894DEBF0FBECDBF90
:10E730006C018B017A018091DD04882309F47CC08F
:10E740008091DC04882309F477C077FF07C0009527
:10E75000109560E0802F0E94277D4DC060E080E032
:10E760000E94277D0E947F9328EE33E040E050E036
:10E770000E94A8A7CA01B90120E831E541E050E0B4
:10E780000E94A8A7AB01BC01CE0107960E94527D52
:10E79000BE01695F7F4FCE0101960E940D596CEC5E
:10E7A00076E0CE0101960E940B58BC01CE010D9679
:10E7B0000E940D59CE0101960E94D158CE010796B4
:10E7C0000E94D158BE01635F7F4F83E694E10E94AF
:10E7D0007359B98860E08B2D0E94277D01151105C2
:10E7E00011F40B2D04C060E0802F0E94277DCE0124
:10E7F0000D960E94D158B60183E694E10E947359A8
:10E800006BEE7CE083E694E10E948159F6018481FD
:10E8100060E0800F0E94277D0E947F936093CA0D65
:10E820007093CB0D8093CC0D9093CD0DB701FF0C61
:10E83000880B990B0E94479362960FB6F894DEBF3F
:10E840000FBECDBFDF91CF911F910F91FF90EF9041
:10E85000DF90CF90BF900895AF92BF92CF92DF929A
:10E86000EF92FF920F931F93CF93DF93CDB7DEB755
:10E8700062970FB6F894DEBF0FBECDBF2091DD04C6
:10E88000222309F491C02091DC04222309F48CC0D6
:10E890006A017B015C010E947F930091CA0D109177
:10E8A000CB0D2091CC0D3091CD0D0C591F4F2F4F1A
:10E8B0003F4F061717072807390708F075C0F7FEFE
:10E8C00008C087010095109560E0802F0E94277D89
:10E8D0004AC060E080E00E94277D0E947F9328EE7E
:10E8E00033E040E050E00E94A8A7CA01B90120E847
:10E8F00031E541E050E00E94A8A7AB01BC01CE0188
:10E9000001960E94527DBE016F5F7F4FCE01079638
:10E910000E940D596CEC76E0CE0107960E940B58D0
:10E92000BC01CE010D960E940D59CE0107960E94A2
:10E93000D158CE0101960E94D158BE01635F7F4F2E
:10E9400083E694E10E94735909891A89E114F1045C
:10E9500031F00E0D1F1D60E0802F0E94277DCE013B
:10E960000D960E94D158B50183E694E10E94735937
:10E970006AED7CE083E694E10E948159F50184818F
:10E9800060E0800F0E94277D0E947F936093CA0DF4
:10E990007093CB0D8093CC0D9093CD0DB601DD0C13
:10E9A000880B990B0E94479362960FB6F894DEBFCE
:10E9B0000FBECDBFDF91CF911F910F91FF90EF90D0
:10E9C000DF90CF90BF90AF9008958F929F92AF92BB
:10E9D000BF92CF92DF92EF92FF920F931F93CF934C
:10E9E000DF938C01862F0B30110509F06EC09091DA
:10E9F000C913992309F0F89462E152DD2091C913FB
:10EA0000222309F07894009709F071C0E090C413B4
:10EA1000F090C5136F2D70E080E090E00E947CA61E
:10EA20002DEC3CEC4CEC5DE30E94DBA64B015C0161
:10EA30006E2D70E080E090E00E947CA69B01AC010E
:10EA4000C501B4010E9406A86093BC137093BD1366
:10EA50008093BE139093BF13C091C613D091C71378
:10EA60006C2F6F7770E080E090E00E947CA64B01F5
:10EA70005C016D2F70E080E090E00E947CA62DECA0
:10EA80003CEC4CEC5DE30E94DBA69B01AC01C501B4
:10EA9000B4010E9406A8C7FD09C06093C01370931B
:10EAA000C1138093C2139093C3130BC0DC01CB013D
:10EAB000B0588093C0139093C113A093C213B09326
:10EAC000C313FE0CCF0DCD0F70C00631110509F038
:10EAD000B3C09091C913992309F0F89461E0E0DC88
:10EAE0002091C913222309F078940097A9F040E0FF
:10EAF00050EC69E774EC4093BC135093BD136093E2
:10EB0000BE137093BF134093C0135093C11360930F
:10EB1000C2137093C31395C0F090C513D091C41362
:10EB20006091C4137091C51376276727762780E01C
:10EB300090E00E947AA62DEC3CEC4CEC5DE30E9448
:10EB4000DBA66093BC137093BD138093BE139093A8
:10EB5000BF13E090C713C091C6138C2F8F776E2D13
:10EB600070E0782B80E090E00E947AA62DEC3CECDF
:10EB70004CEC5DE30E94DBA6C7FD09C06093C013A7
:10EB80007093C1138093C2139093C3130BC0DC0125
:10EB9000CB01B0588093C0139093C113A093C213BC
:10EBA000B093C313DF0DED0ECE0D8091C813C813C3
:10EBB00046C0C090BC13D090BD13E090BE13F0903F
:10EBC000BF1320E030E048EC52E4C701B6010E94D8
:10EBD000BBA918161CF0C0E0D0E002C0CBEFDFEFFD
:10EBE00020E030E0A901C701B6010E9476A687FFA8
:10EBF00002C0CAEFDFEFC090C013D090C113E09005
:10EC0000C213F090C31320E030E048EC52ECC7018F
:10EC1000B6010E9476A687FF02C0C9EFDFEF20E0B1
:10EC200030E040EF52E4C701B6010E94BBA91816BC
:10EC3000ACF4C8EFDFEF12C0CFEFDFEF0FC08FEF04
:10EC40009FEF8F3FFFEF9F0709F4D2C0009709F4B1
:10EC5000B0CF029609F4D8C0CCEFDFEF0C3011052D
:10EC600009F0D5C08CE5D8D680E090E0D0D6CDD6DE
:10EC700065E08CE50CDCC82FD0E02097A1F0C53012
:10EC8000D105A4F00FEC1DE085EF90E10E948B8B85
:10EC9000F80180870F5F1F4FC8018F5C9D408C1764
:10ECA0009D0794F306C0CEEFDFEFB1C0CDEFDFEFED
:10ECB000AEC0C091D70D0091D80D602F70E080E0FC
:10ECC00090E00E947CA62DEC3CEC4CEC5DE30E94B5
:10ECD000DBA66B017C016C2F70E080E090E00E946D
:10ECE0007CA69B01AC01C701B6010E9406A86093F7
:10ECF000CF0D7093D00D8093D10D9093D20DD09104
:10ED0000D90D1091DA0D6D2F6F7770E080E090E0F3
:10ED10000E947CA66B017C01612F70E080E090E096
:10ED20000E947CA62DEC3CEC4CEC5DE30E94DBA643
:10ED30009B01AC01C701B6010E9406A8D7FF5BC0CA
:10ED4000DC01CB01B0588093D30D9093D40DA093E8
:10ED5000D50DB093D60D8C2F800FC82FCD0FC10FBE
:10ED60008091DB0DC81344C0C090CF0DD090D00D62
:10ED7000E090D10DF090D20D20E030E048EC52E46C
:10ED8000C701B6010E94BBA918161CF0C0E0D0E074
:10ED900002C0CBEFDFEF20E030E040EA50E4C701F3
:10EDA000B6010E9476A687FF02C0CAEFDFEFC090CF
:10EDB000D30DD090D40DE090D50DF090D60D20E07D
:10EDC00030E040EF51ECC701B6010E9476A687FF04
:10EDD00002C0C9EFDFEF20E030E040EF52E4C701AE
:10EDE000B6010E94BBA9181694F4C8EFDFEF0FC05C
:10EDF000CFEFDFEF0CC06093D30D7093D40D8093F1
:10EE0000D50D9093D60DA7CFCEEFDFEF27CFCE0154
:10EE1000DF91CF911F910F91FF90EF90DF90CF90F6
:10EE2000BF90AF909F908F900895CF93DF93FC0198
:10EE300024813581232B59F0EC01BC0188E590E158
:10EE400077D5BE0181E89EE0DF91CF9171C5DF915A
:10EE5000CF910895CF92DF92EF92FF92CF93C0911E
:10EE60000212C43014F5C1300CF04DC0C11179C08C
:10EE70000E948765BC01990F880B990B0E947CA6A4
:10EE800020E030E040EA50E40E94DBA620E030ECD5
:10EE90004FE754E40E94CCA8209103123091041251
:10EEA000409105125091061259C0C43009F059C062
:10EEB0000E948765BC01990F880B990B0E947CA664
:10EEC00020E030E040EA50E40E94DBA620E030EC95
:10EED0004FE754E40E94CCA820E030E040EA50E440
:10EEE0000E94CCA820E030E040E851E40E94DBA67C
:10EEF00020E030E040E850E40E9406A820E030E046
:10EF00004AE754E42BC00E948765BC01990F880B27
:10EF1000990B0E947CA62AE137E64CE950E40E9456
:10EF2000DBA62091031230910412409105125091FA
:10EF300006120E9405A86B017C01EC2FEE0FFF0B5F
:10EF4000E15BFA4F60817181072E000C880B990BF1
:10EF50000E947CA69B01AC01C701B6010E94CCA80F
:10EF600003C060E070E0CB01CF91FF90EF90DF90A5
:10EF7000CF900895CF92DF92EF92FF92CF93DF93DD
:10EF8000EC018091FF11082E000C990B0E94E3A167
:10EF900003971CF5CE010E948765EC016091001279
:10EFA00070910112072E000C880B990B0E947CA611
:10EFB0006B017C01BE01DD0F880B990B0E947CA6C2
:10EFC0009B01AC01C701B6010E94DBA620E030EC3A
:10EFD0004FE754E40E94CCA803C060E070E0CB018E
:10EFE000DF91CF91FF90EF90DF90CF9008958F92B7
:10EFF0009F92AF92BF92CF92DF92EF92FF92CF9308
:10F00000DF93CDB7DEB72C970FB6F894DEBF0FBEF7
:10F01000CDBF61EB7DE0CE0101960E9405594CE227
:10F0200051E06FEF7FEFCE0101960E94D381CE01B8
:10F0300001960E94D1586091D0047091D1048091C2
:10F04000260590912705C1DC84E1882E912CA12C06
:10F05000B12CE12CF12C2FEFE21AF20AC501B40118
:10F060000E9447936091D0047091D104809126054D
:10F0700090912705AADC23E0E216F10434F02AE09F
:10F08000E216F10444F4892B49F084E1880E911CC6
:10F09000A11CB11CE0CF892B09F088C18091260505
:10F0A000909127058B309105C9F48091C013909100
:10F0B000C113A091C213B091C3138093E00D90933C
:10F0C000E10DA093E20DB093E30D8091BC139091FC
:10F0D000BD13A091BE13B091BF131DC08631910521
:10F0E00021F30C9701F58091D30D9091D40DA0914F
:10F0F000D50DB091D60D8093E00D9093E10DA093C6
:10F10000E20DB093E30D8091CF0D9091D00DA091C1
:10F11000D10DB091D20D8093DC0D9093DD0DA093B5
:10F12000DE0DB093DF0D4091E00D5091E10D609147
:10F13000E20D7091E30D21E0CE0107960E94D658B2
:10F1400060EF7BE0CE0101960E941559BE01695F18
:10F150007F4FCE0101960E942258BC0188E693E1C0
:10F160000E948258CE0101960E94D158CE01079686
:10F170000E94D1584091DC0D5091DD0D6091DE0D63
:10F180007091DF0D21E0CE0107960E94D65866E30C
:10F190007AE0CE0101960E941559BE01695F7F4F4A
:10F1A000CE0101960E942258BC0188E693E10E949C
:10F1B0004158CE0101960E94D158CE0107960E9477
:10F1C000D15868EF79E088E693E10E9433586FECFC
:10F1D0007CE0CE0101960E94155944E150E060E0C8
:10F1E00070E0CE01019693DACE0101960E94D158CB
:10F1F000C090E00DD090E10DE090E20DF090E30DB5
:10F2000020E030E0A901C701B6010E94BBA920E0BF
:10F2100030E040E05FE387FD05C0C701B6010E9412
:10F2200006A804C0C701B6010E9405A80E9465A9EE
:10F23000AB01BC01CE01019635D4BE016F5F7F4F9B
:10F2400082E693E10E949758CE0101960E94D15820
:10F2500060E087E0FCD362E673E183E694E10E941C
:10F2600073596FED83E694E10E946C596CE37AE088
:10F2700083E694E10E944C5A6091DC0D7091DD0DA3
:10F280008091DE0D9091DF0D0E9465A94AE050E06B
:10F2900083E694E10E94025A68EF79E083E694E104
:10F2A0000E944C5A64E670E080E090E00E94479330
:10F2B000C090E00DD090E10DE090E20DF090E30DF4
:10F2C00020E030E040EF51E4C701B6010E94BBA945
:10F2D00087FD03C062EA7DE054C020E030E040EDED
:10F2E00051E4C701B6010E94BBA987FD1FC062E9B6
:10F2F0007DE0CE0101960E9405594AE050E06FEF93
:10F300007FEFCE0101960E94D381CE0101960E942B
:10F31000D1588091C104882331F06CED75E080E014
:10F3200090E00E94479362E87DE02BC020E030E04F
:10F3300040EB51E4C701B6010E94BBA987FD03C0A1
:10F3400064E77DE01EC065E67DE0CE0101960E9487
:10F3500005594AE050E06FEF7FEFCE0101960E9421
:10F36000D381CE0101960E94D1588091C104882397
:10F3700031F06CED75E080E090E00E94479367E526
:10F380007DE0CE0101960E9405594AE050E06FEF02
:10F390007FEFCE0101960E94D381CE0101960E949B
:10F3A000D15862E370E080E090E0D7C0CDD76EE145
:10F3B00070E080E090E00E9447930E948A716B01A8
:10F3C0007C0164E670E080E090E00E94479360EF8B
:10F3D0007BE088E693E10E946D5821E0B701A60129
:10F3E000CE0101960E94D658BE016F5F7F4F88E61E
:10F3F00093E10E944158CE0101960E94D15868E6DF
:10F4000073E1CE0101960E940D594AE050E060E0A0
:10F4100070E0CE0101967BD9CE0101960E94D158B1
:10F420008091DD04882379F08091DC04882359F0F1
:10F430006FED83E694E10E946C5963E77CE083E61C
:10F4400094E10E944C5A62E77CE088E693E10E94D6
:10F450003358C092E00DD092E10DE092E20DF092AF
:10F46000E30D20E030E040EF51E4C701B6010E9417
:10F47000BBA987FD03C067E47DE052C020E030E017
:10F4800040ED51E4C701B6010E94BBA987FD1EC033
:10F4900067E37DE0CE0101960E9405594AE050E005
:10F4A0006FEF7FEFCE0101967ED7CE0101960E94CD
:10F4B000D1588091C104882331F06CED75E080E073
:10F4C00090E00E94479367E27DE02AC020E030E0B0
:10F4D00040EB51E4C701B6010E94BBA987FD03C000
:10F4E00069E17DE01DC06AE07DE0CE0101960E94E9
:10F4F00005594AE050E06FEF7FEFCE01019653D7F8
:10F50000CE0101960E94D1588091C104882331F028
:10F510006CED75E080E090E00E9447936CEF7CE03A
:10F52000CE0101960E9405594AE050E06FEF7FEF4F
:10F53000CE01019638D7CE0101960E94D1586CE2D7
:10F5400071E080E090E00E9447938091C10488239D
:10F5500031F068EE73E080E090E00E9447932C96D3
:10F560000FB6F894DEBF0FBECDBFDF91CF91FF90F5
:10F57000EF90DF90CF90BF90AF909F908F900895C5
:10F58000DF92EF92FF920F931F93CF93DF93CDB74C
:10F59000DEB762970FB6F894DEBF0FBECDBF8C0109
:10F5A0001092E40D6FEC7CE0CE010D960E9415598F
:10F5B000FF24F39488E590E10E949D542091E40D8E
:10F5C00018161906D4F5211138C088E590E10E947B
:10F5D0007B548A3041F08D3031F0682FCE010D968A
:10F5E0000E94135423C089899A89892BF9F0F092DB
:10F5F000E40D6DEA7CE0CE0101960E941559BE0132
:10F60000635F7F4FCE0101960E942258BC01CE015C
:10F6100007960E940D59CE0107964DD8CE01079648
:10F620000E94D158CE0101960E94D1586AE070E044
:10F6300080E090E00E944793BDCF211174C0E12C7F
:10F64000F12CDD24D39481E89EE00E949D5418168D
:10F65000190614F581E89EE00E947B548A3079F007
:10F660008D3069F09091E40D911109C0682FCE01A1
:10F670000D960E9413548FEFE81AF80A06C0898984
:10F680009A89892B11F0D092E40D65E070E080E05A
:10F6900090E00E944793D7CF64E170E080E090E073
:10F6A0000E944793EF2849F189899A89892B29F18A
:10F6B0008091CE0D8823B9F066EB7CE088E590E17F
:10F6C0000E944C5ABE01635F7F4FCE0101960E949B
:10F6D0000D59BE016F5F7F4F88E590E129D1CE01C2
:10F6E00001960E94D15881E89EE00E943B5564E15A
:10F6F00070E080E090E00E9447938091E40D8111DA
:10F7000012C089899A89892B71F464E670E080E0DF
:10F7100090E00E9447930E947F936FEC7CE0C801C9
:10F720000E94155957C089899A89019709F045C0E7
:10F730006FEC79E0CE0107960E941559BE01695F12
:10F740007F4FCE010D960E942654811116C068EDA0
:10F7500077E0CE0101960E941559BE016F5F7F4F81
:10F76000CE010D960E942654FF24F3948111F12CB2
:10F77000CE0101960E94D15801C0F12CCE0107960E
:10F780000E94D158FF2099F040E050E0BE01635F35
:10F790007F4FCE0101969BD6BE016F5F7F4F84E7FE
:10F7A00093E10E949758CE0101960E94D15864E1DE
:10F7B00070E080E090E00E944793F801118210828F
:10F7C0001382128215821482BE01635F7F4FC801CB
:10F7D0000E949758CE010D960E94D158C80162969A
:10F7E0000FB6F894DEBF0FBECDBFDF91CF911F9152
:10F7F0000F91FF90EF90DF900895DF92EF92FF92CC
:10F800000F931F93CF93DF93CDB7DEB72C970FB62F
:10F81000F894DEBF0FBECDBF8C011092E40D6FECEB
:10F820007CE0CE0107960E941559E12CF12CDD24D5
:10F83000D39481E89EE00E949D541816190614F591
:10F840008091E40D81111EC081E89EE00E947B54EE
:10F850008A3059F08D3049F0682FCE0107960E940A
:10F8600013548FEFE81AF80A06C08B859C85892B04
:10F8700011F0D092E40D6FE070E080E090E00E9423
:10F880004793D7CF62E370E080E090E00E94479317
:10F89000EF2851F081E89EE00E943B5564E670E05D
:10F8A00080E090E00E9447938091E40D81110AC0AE
:10F8B0008B859C85892B31F46FEC7CE0C8010E941C
:10F8C00015591FC08091CE0D882371F0BE01695F6C
:10F8D0007F4FCE0101960E940D59CE010196A5DA07
:10F8E000CE0101960E94D158F80111821082138234
:10F8F000128215821482BE01695F7F4FC8010E9487
:10F900009758CE0107960E94D158C8012C960FB681
:10F91000F894DEBF0FBECDBFDF91CF911F910F9145
:10F92000FF90EF90DF9008956DEC7CE00C94A5596A
:10F930000F931F93CF93DF93EC010E9473598C01B7
:10F94000CE01F2DF800F911FDF91CF911F910F91B8
:10F950000895282F3091800E313208F04AC08091EE
:10F960005D0E8111FCCF90916F1442E040935D0ECB
:10F9700020935C0E2FEF20935B0E10925A0E309363
:10F98000590EE0E6FEE0A9E3BEE020E0321721F0E8
:10F9900041914D932F5FFACF1092380E2091380E7F
:10F9A000990F922B9093380E9091370E913061F40D
:10F9B0001092370E9091380E9093BB009091BC003E
:10F9C00093FDF8CF95EC01C095EE9093BC0090911B
:10F9D0005D0E9230E1F390915B0E9F3F79F0809144
:10F9E0005B0E803241F080915B0E803331F084E019
:10F9F00005C081E003C082E001C083E010925F0E89
:10FA00001092800E10925E0E089581E0A2CF682FB2
:10FA100085EF90E10C94D38B91E090935E0E8093F0
:10FA20006F1410925F0E1092800E0895CF93C82F1E
:10FA3000682F607F83E694E10E94CB8C80E1C89FB1
:10FA4000B001112483E694E1CF910C94CB8CCF9339
:10FA5000DF93CDB7DEB728970FB6F894DEBF0FBEA1
:10FA6000CDBF98E0E7E5F5E0DE01119601900D923B
:10FA70009A95E1F790916C14961710F46FEF690F57
:10FA8000FE013196E60FF11DE60FF11D9081890F01
:10FA9000806828960FB6F894DEBF0FBECDBFDF9109
:10FAA000CF91C4CF0F931F93CF93DF93CDB7DEB722
:10FAB000A2970FB6F894DEBF0FBECDBF8C01CB016D
:10FAC000BA01F80111821082138212821582148207
:10FAD0002AE0AE014F5F5F4F0E9440A2BE016F5F00
:10FAE0007F4FC8010E946D58A2960FB6F894DEBFF2
:10FAF0000FBECDBFDF91CF911F910F9108950F934E
:10FB00001F93CF93DF93EC010E94A5598C01CE0186
:10FB10000BDF800F911FDF91CF911F910F910895FF
:10FB2000CF92DF92EF92FF92CF93DF936B017C0134
:10FB300097FF15C06DE288E590E10E946C59EC01D9
:10FB400044275527BA014C195D096E097F092AE03F
:10FB500088E590E10E94BA59C80FD91F08C02AE071
:10FB6000AB01BC0188E590E10E94BA59EC0188E53F
:10FB700090E1DADE8C0F9D1FDF91CF91FF90EF9027
:10FB8000DF90CF9008958F929F92AF92BF92CF92C5
:10FB9000DF92EF92FF920F931F93CF93DF936B014E
:10FBA0007C01142F9B01AC010E9405AB882319F046
:10FBB00060ED7CE027C046015701E894B7F82FEFCD
:10FBC0003FEF4FE75FE7C501B4010E9405AB81112C
:10FBD0000DC02FEF3FEF4FE75FE7C501B4010E9473
:10FBE00076A618161CF464ED7CE00CC02FEF3FEFF6
:10FBF0004FE75FE4C701B6010E94BBA9181694F451
:10FC000068ED7CE088E590E1DF91CF911F910F9145
:10FC1000FF90EF90DF90CF90BF90AF909F908F902C
:10FC20000C94A5592FEF3FEF4FE75FECC701B601EA
:10FC30000E9476A687FDE4CF20E030E0A901C7014D
:10FC4000B6010E9476A687FF0BC06DE288E590E1C1
:10FC50000E946C59EC01F7FAF094F7F8F09402C0A6
:10FC6000C0E0D0E000E060E070E080E09FE31017CB
:10FC700041F020E030E040E251E40E94CCA80F5F68
:10FC8000F6CFA70196010E9406A86B017C010E9495
:10FC90006AA94B015C012AE0AB01BC0188E590E157
:10FCA0000E94BA59C80FD91F1123C9F1C501B40167
:10FCB0000E947AA69B01AC01C701B6010E9405A86B
:10FCC0006B017C016EE288E590E10E946C59C80FDF
:10FCD000D91F20E030E040E251E4C701B6010E94A4
:10FCE000DBA64B015C010E946AA96B01E12CF12C9F
:10FCF0002AE0B701A60188E590E10E94BA59C80F31
:10FD0000D91FC701B6010E947AA69B01AC01C501AB
:10FD1000B4010E9405A86B017C011150D1F6CE01FF
:10FD2000DF91CF911F910F91FF90EF90DF90CF90D7
:10FD3000BF90AF909F908F9008952F923F924F92D7
:10FD40005F926F927F928F929F92AF92BF92CF926B
:10FD5000DF92EF92FF920F931F93CF93DF93CDB774
:10FD6000DEB728970FB6F894DEBF0FBECDBFC090A8
:10FD7000E70DD090E80D4091E90D5091EA0DC416C1
:10FD8000D5062CF43C2D2D2D6A01432F522FEBEE7E
:10FD9000FDE060E070E0CB010191119104171507BF
:10FDA00054F44A01550FAA08BB08680D791D8A1D35
:10FDB0009B1DA80115C0C016D10654F40D2C000CD3
:10FDC000EE08FF086C0D7D1D8E1D9F1D680108C08B
:10FDD000012E000C220B330B600F711F821F931F2B
:10FDE0002EE0E733F207C1F60E947CA620E030E067
:10FDF00048E152E40E94CCA88B0188879F8387EE5C
:10FE0000E82E8DE0F82E812C912C5401D7016D91B4
:10FE10007D917D01072E000C880B990B0E947CA61A
:10FE2000980148855F810E9405A89B01AC010E9452
:10FE3000DBA69B01AC01C501B4010E9406A84B01E1
:10FE40005C01E7E3FEE0EE15FF0501F720E030E09E
:10FE50004CE152E40E94CCA80E94C4AA6B017C0130
:10FE600020E030E040E85FE30E94BBA918160CF0E8
:10FE700069C027EE3DE03A832983212C312C412CA7
:10FE8000512C3201A981BA818D919D91BA83A983A8
:10FE90009C01990F440B550B2B833C834D835E8350
:10FEA000CA01B9010E947CA6980148855F810E9421
:10FEB00005A84B015C0120E030E0A9010E94BBA92C
:10FEC000181624F0B7FAB094B7F8B094A7019601C9
:10FED000C501B4010E9476A687FF0BC08B819C816F
:10FEE000AD81BE81480E591E6A1E7B1E9FEF291AE6
:10FEF000390AA7E3BEE0E981FA81AE17BF0711F620
:10FF000020E030E040EC5FE3C701B6010E94DBA6D1
:10FF10006B017C01F5E02F1631040CF4AACFC3016C
:10FF2000B2010E947CA66B017C01B101330C880BED
:10FF3000990B0E947CA69B01AC01C701B6010E94EF
:10FF4000CCA803C0B80188859F816B017C01C701E3
:10FF5000B60128960FB6F894DEBF0FBECDBFDF9175
:10FF6000CF911F910F91FF90EF90DF90CF90BF90B6
:10FF7000AF909F908F907F906F905F904F903F9049
:10FF80002F9008954F925F926F927F928F929F92DF
:10FF9000AF92BF92CF92DF92EF92FF921F93CF93D7
:10FFA000DF93CDB7DEB728970FB6F894DEBF0FBE4C
:10FFB000CDBF4B015C0111E0612E712C9301220F2A
:10FFC000331F220F331F3A832983F901EA50FB4F75
:10FFD000C080D180E280F380A5019401C701B60101
:10FFE0000E9476A687FF02C01F5FE6CFA50194019D
:10FFF000C701B6010E9476A649815A8142525B4FE1
:020000021000EC
:100000005E834D83811106C0FA0160817181828116
:1000100093814DC0F1E06F1AF0EC7F0AC301880FA5
:10002000991F880F991FFC01EA50FB4F20813181F5
:100030004281538129833A834B835C83FC01E252E2
:10004000FB4F4080518062807380A3019201ED815B
:10005000FE8160817181828193810E9405A86D83F8
:100060007E838F83988729813A814B815C81C5018A
:10007000B4010E9405A89B01AC016D817E818F8136
:1000800098850E94DBA64B015C0129813A814B8156
:100090005C81C701B6010E9405A89B01AC01C501A6
:1000A000B4010E94CCA8A30192010E9406A8289640
:1000B0000FB6F894DEBF0FBECDBFDF91CF911F9179
:1000C000FF90EF90DF90CF90BF90AF909F908F9078
:1000D0007F906F905F904F9008950F931F930E94B1
:1000E0007F936093260F7093270F8093280F909330
:1000F000290F8EE19FE00E947B5497FF1FC00E9452
:100100007F930091260F1091270F2091280F309197
:10011000290FDC01CB01801B910BA20BB30B0091CB
:10012000220F1091230F2091240F3091250F80175B
:100130009107A207B307E8F28FEF9FEF1F910F918E
:100140000895CF92DF92EF92FF92CF93DF93EC016D
:100150006A017B01E889F98982E080834115514E6B
:1001600061057105B1F060E079E08DE390E0A701F1
:1001700096010E94D4A7DA01C9010197A109B1092A
:10018000B695A795979587959C01211580E138072D
:10019000A8F0E889F989108260E874E88EE190E0BF
:1001A000A70196010E94D4A7DA01C9010197A1090C
:1001B000B109B695A795979587959C01EC85FD8526
:1001C0003083EE85FF852083188EEC89FD8986E0DB
:1001D0008083EA89FB89808180618083EA89FB8949
:1001E000808188608083EA89FB8980818068808340
:1001F000EA89FB8980818F7D8083DF91CF91FF9099
:10020000EF90DF90CF900895EF92FF920F931F939E
:10021000CF93DF931F921F92CDB7DEB703ED11E1AD
:10022000835D91417C01C701800F911FF8016191AD
:100230008F019A838983CE01019630D1F2E109358D
:100240001F0789F783ED91E10F900F90DF91CF9118
:100250001F910F91FF90EF9008950F931F93CF93ED
:10026000DF931F921F92CDB7DEB705EE1DE0F801B8
:1002700060818EED93E09A838983CE0101960ED141
:10028000F80161818FED93E09A838983CE01019615
:1002900005D1C8010F900F90DF91CF911F910F9161
:1002A0000895EF92FF920F931F93CF93DF931F92C6
:1002B0001F92CDB7DEB702E612E1825692417C0171
:1002C000C701800F911FF80161918F019A83898383
:1002D000CE010196E3D0F2E10C361F0789F782E6E2
:1002E00092E10F900F90DF91CF911F910F91FF90AE
:1002F000EF900895EF92FF920F931F93CF93DF93A8
:100300001F921F92CDB7DEB702E612E182569241EC
:100310007C01C701800F911FF80161918F019A83C1
:100320008983CE010196BAD0F3E10C351F0789F716
:1003300082E692E10F900F90DF91CF911F910F9184
:10034000FF90EF90089508958091DD048823E1F0F7
:100350008091DC048823C1F081E068DB8BE39FE1BE
:100360000197F1F760E080E072DB6DEA7EE083E602
:1003700094E10E94815961E080E069DB6DE97EE0F3
:1003800083E694E10C94815908958091DD048823DB
:1003900049F08091DC04882329F060E083E694E151
:1003A0000C94E18C08958F929F92AF92BF92EF923E
:1003B000FF920F931F93CF93DF932091DD042223AD
:1003C00009F461C02091DC04222309F45CC08A0195
:1003D000EB017C0177FF16C0C095D09561E08C2FB2
:1003E00036DBB70183E694E10E9473596CE87EE046
:1003F00083E694E10E948159F701848161E08C0FCA
:1004000026DB31C00E947F938090280D9090290DAB
:10041000A0902A0DB0902B0D24E6820E911CA11CF9
:10042000B11C86169706A806B90668F561E08C2F00
:100430000EDBB70183E694E10E9473596BE77EE01F
:1004400083E694E10E948159F701848161E08C0F79
:10045000FEDA0E947F936093280D7093290D80939C
:100460002A0D90932B0DB801110F880B990BDF917A
:10047000CF911F910F91FF90EF90BF90AF909F9001
:100480008F900C944793DF91CF911F910F91FF9024
:10049000EF90BF90AF909F908F900895FF920F9331
:1004A0001F93CF93DF93EC01F62E08811981C801C9
:1004B0000E9492A7F81621F06F2DC8010E949AA7FA
:1004C000CE01DF91CF911F910F91FF900895CF93AF
:1004D000DF93EC01FB01248135810E942959CE0173
:1004E000DF91CF9108954F925F926F927F928F929A
:1004F0009F92AF92BF92CF92DF92EF92FF920F93B3
:100500001F93CF93DF93CDB7DEB7C654D1090FB693
:10051000F894DEBF0FBECDBF8C016FEC7CE0CE0146
:10052000C7960E9415596FEC7CE0CE01CD960E94D3
:100530001559BE016F5F7F4F8DE993E10E942C56E4
:100540008D889E88AF88B88C498C5A8C6B8C7C8C3B
:100550008D8D9E8DAF8DB8A127968CAF9DAFAEAF20
:10056000BFAF2797C8010197039708F0BCC1A3014B
:100570009201C501B40190580E9479A82BED3FE08B
:1005800049EC5FE30E9406A82091B9043091BA04B7
:100590004091BB045091BC040E9406A86B017C01F1
:1005A00020E030E0A9010E9476A687FD09C0C09234
:1005B0007814D0927914E0927A14F0927B1410C0DF
:1005C0002BED3FE049EC50E4C701B6010E9406A8BC
:1005D000609378147093791480937A1490937B14B9
:1005E000C0907814D0907914E0907A14F0907B1435
:1005F0002BED3FE049EC50E4C701B6010E94BBA9D6
:10060000181684F42BED3FE049EC50E4C701B60125
:100610000E9405A8609378147093791480937A14DB
:1006200090937B1420E030E044E353E4609178142D
:100630007091791480917A1490917B140E94DBA6BA
:100640002BED3FE049E450E40E94CCA86093741481
:100650007093751480937614909377140E9465A913
:10066000CE018B960E941B726CED7CE0CE018596CC
:100670000E941559BE01655D7F4FCE0185960E948F
:10068000225866EE7CE00E940B58BC018EE693E196
:100690000E948258CE0185960E94D158CE018B9639
:1006A0000E94D158C0907414D0907514E0907614C4
:1006B000F090771420E030E044EB52E4C701B6013B
:1006C0000E9476A618168CF020E030E040E05FE350
:1006D000C701B6010E9406A80E9465A9CE018B96AB
:1006E0000E941B726DEE7CE022C020E030E044E30B
:1006F00053E4C701B6010E9476A618169CF1A70123
:10070000960160E070E884E393E40E9405A860939A
:1007100074147093751480937614909377140E94D8
:1007200065A9CE018B960E941B7260EF7CE0CE0122
:1007300085960E941559BE01655D7F4FCE01859655
:100740000E942258BC01CE01C7960E948258CE0159
:1007500085960E94D158CE018B960E94D1586FE9A0
:100760007AE061C020E030E047E853E4C701B60119
:100770000E9476A61816FCF020E030E044E353E433
:10078000C701B6010E9405A820E030E040E05FE329
:100790000E9406A860937414709375148093761465
:1007A000909377140E9465A9CE018B960E941B72CC
:1007B00060EF7CE01EC0A701960160E070E084EB72
:1007C00093E40E9405A820E030E040E05FE30E944F
:1007D00006A86093741470937514809376149093A4
:1007E00077140E9465A9CE018B960E941B726DEE54
:1007F0007CE0CE0185960E941559BE01655D7F4F54
:10080000CE0185960E942258BC01CE01C7960E9457
:100810008258CE0185960E94D158CE018B960E94B7
:10082000D15863EF7CE0CE01CD960E946D58BE0199
:10083000695C7F4FCE0185960E940D594AE050E0D9
:1008400060E070E0CE0185960E948773CE018596A8
:100850000E94D1580E947F93C090CA0DD090CB0DBA
:10086000E090CC0DF090CD0DA4E6CA0ED11CE11C99
:10087000F11CC616D706E806F90608F423C20E9442
:100880007F930E947AA66B017C016091CA0D7091E2
:10089000CB0D8091CC0D9091CD0D0E947CA620E0D7
:1008A00030E048EC51E40E9406A89B01AC01C7016E
:1008B000B6010E9476A687FD05C267E67CE0CE0100
:1008C00085960E941559BE01635C7F4FCE018596C7
:1008D0000E942258BC01CE01C7960E944158CE0109
:1008E00085960E94D158C8010297029708F0C4C1AA
:1008F00020E030E040E251E4C501B4010E94DBA6F3
:100900006B017C0120E030E040E251E4C301B20120
:100910000E94DBA64B015C0120E030E040E251E4A4
:1009200027966CAD7DAD8EAD9FAD27970E94DBA65F
:100930002B013C010E947F9320912C0D30912D0DB5
:1009400040912E0D50912F0D621B730B840B950B54
:100950000E947AA620E030E04AE754E40E94CCA846
:10096000AB01BC0123E0CE018B960E94D65866E70E
:100970007CE0CE0185960E941559BE01655D7F4FD2
:10098000CE0185960E9422586CEC76E00E940B58AE
:10099000BC018CE593E10E948258CE0185960E94AD
:1009A000D158CE018B960E94D1586CE573E1CE01EF
:1009B00085960E940D596EE673E1CE0185960E94E0
:1009C0002258BE01695C7F4F0E942258BC01CE01B3
:1009D000C7960E948258CE0185960E94D15860E742
:1009E0007EE088E693E10E94475821E0B701A60126
:1009F000CE0185960E94D658BE016B5D7F4F88E67A
:100A000093E10E944158CE0185960E94D15821E081
:100A1000B301A201CE01C1960E94D65821E0B501D2
:100A2000A401CE018B960E94D65867E67CE0CE01E9
:100A300085960E941559BE01655D7F4FCE01859652
:100A40000E94225867E67CE00E940B58BE016F5C52
:100A50007F4F0E94225865EF7CE00E940B58BC013A
:100A600088E693E10E944158CE0185960E94D158B4
:100A7000CE018B960E94D158CE01C1960E94D158CA
:100A8000A7019601C701B6010E94DBA66B017C019C
:100A9000A5019401C501B4010E94DBA69B01AC0134
:100AA000C701B6010E9406A86B017C01A301920157
:100AB000C301B2010E94DBA69B01AC01C701B601D4
:100AC0000E9406A80E94C4AA6B017C016093701466
:100AD00070937114809372149093731469EF7CE097
:100AE00088E693E10E94335821E0B701A601CE01C8
:100AF00085960E94D658BE016B5D7F4FCE018B96C6
:100B00000E940D5967E07DE0CE018B960E940B5844
:100B1000BC018EE693E10E948258CE018B960E9422
:100B2000D158CE0185960E94D1586EE673E188E6D1
:100B300093E10E944158C0907014D0907114E090DD
:100B40007214F090731420E030E04AE754E4C701D7
:100B5000B6010E94BBA987FD29C020E030E04AE72A
:100B600054E4C701B6010E94CCA8AB01BC0123E04C
:100B7000CE0185960E94D658BE016B5D7F4FCE0197
:100B80008B960E940D5968E07DE0CE018B960E9405
:100B90000B58BC018EE693E10E948258CE018B96E1
:100BA0000E94D158CE0185960E94D15820E030E6AF
:100BB0004AE656E460917014709171148091721439
:100BC000909173140E9476A6BE01695C7F4F87FFE7
:100BD0004FC0CE0185960E940D5965E77CE0CE019D
:100BE00085960E940B5868E673E10E942258BC016A
:100BF00088E693E10E948258CE0185960E94D158E2
:100C000003301105A1F468E673E1CE0185960E94D8
:100C10000D59CE0185960E941577CE0185960E94CA
:100C2000D1586FEC7CE088E693E10E946D586DEF3F
:100C30007CE0CE0185960E9415596EE673E1CE01E7
:100C400085960E942258BC01CE018B960E940D59B8
:100C50004AE050E06FEF7FEFCE018B96A4DBCE0130
:100C60008B960E94D158CE0185960E94D15804C01F
:100C700088E693E10E9482586AE070E080E090E0AC
:100C80000E944793CE01CD960E94D158CE01C796BF
:100C90000E94D158CA5BDF4F0FB6F894DEBF0FBE7B
:100CA000CDBFDF91CF911F910F91FF90EF90DF901B
:100CB000CF90BF90AF909F908F907F906F905F90FC
:100CC0004F9008956FEC7CE0CE0185960E941559F7
:100CD000CE0185960E94566ECE0185960E94D1580F
:100CE000BE01635C7F4F83E694E10E947359E5CDBA
:100CF0001F93CF93DF93CDB7DEB7A8970FB6F894C5
:100D0000DEBF0FBECDBF182F0E94E9718EE10E9499
:100D10000C7D62E085EF90E146D560E085EF90E1E3
:100D200042D50E94057D8EE10E940C7D61E085EF39
:100D300090E139D560E285EF90E135D50E94057DDF
:100D400080E290E09093A1138093A01380E090E85C
:100D5000A9E8B4E48093D8049093D904A093DA046A
:100D6000B093DB0480E090E0A5E7B4E48093D40482
:100D70009093D504A093D604B093D704BE016F5FBF
:100D80007F4F8DE993E10E94DF55112309F484C060
:100D900065E47EE088E590E10E94815988E590E174
:100DA0000E94947C65E37EE088E590E10E94815991
:100DB000BE016F5F7F4F88E590E10E947F7D65E215
:100DC0007EE088E590E10E9481596D857E858F8562
:100DD00098890E94907D65E17EE088E590E10E941F
:100DE000815969897A898B899C890E94907D65E007
:100DF0007EE088E590E10E94815920E030E040E209
:100E000051E4698D7A8D8B8D9C8D0E94DBA642E02A
:100E10000E94C37D66E07DE088E590E10E947F7DD1
:100E200065EF7DE088E590E10E94815920E030E0A7
:100E300040E251E46D8D7E8D8F8D98A10E94DBA6DE
:100E400042E00E94C37D66E07DE088E590E10E947B
:100E50007F7D65EE7DE088E590E10E94815920E08C
:100E600030E040E251E469A17AA18BA19CA10E94EB
:100E7000DBA642E00E94C37D66E07DE088E590E16C
:100E80000E947F7D6FEB7DE088E590E10E948159B3
:100E900088E590E10E94947C64EF71E080E090E04E
:100EA0000E944793A8960FB6F894DEBF0FBECDBF41
:100EB000DF91CF911F9108950C942BAC0895E3ED31
:100EC000F1E114A215A216A217A210A611A612A64D
:100ED00013A681E084A729E130E036A725A787A7DC
:100EE00080E090E0A0EAB0E480AB91ABA2ABB3AB02
:100EF00080E090E0A8EAB1E484AB95ABA6ABB7ABD9
:100F000080932C0590932D05A0932E05B0932F056B
:100F100080E090E0A0E8BFE380931D1290931E1242
:100F2000A0931F12B0932012809328059093290557
:100F3000A0932A05B0932B0510924A1210924912E1
:100F40008BE090E090934C1280934B129093270586
:100F50008093260510927C0D10927B0D80E090E02E
:100F600053C93F924F925F926F927F928F929F925E
:100F7000AF92BF92CF92DF92EF92FF920F931F93A7
:100F8000CF93DF93CDB7DEB7A8970FB6F894DEBF47
:100F90000FBECDBF81E080937C1400E010E082E0C2
:100FA000382E98EEC92E93E0D92EE12CF12C0E307C
:100FB000110508F041C3F8018827E855FF4F8F4F0E
:100FC0000C9454AB8091491290914A12892B09F5E7
:100FD0006CE87AE0CE0107960E94155967E574E146
:100FE000CE0107960E942258BC01CE0101960E94B4
:100FF0000D5948EC50E06FEF7FEFCE0101960E9453
:101000008773CE0101960E94D158CE0107960E94A7
:10101000D1588091491290914A12019709F568E7D9
:101020007AE0CE0107960E94155967E574E1CE017A
:1010300007960E942258BC01CE0101960E940D59CC
:1010400048EC50E06FEF7FEFCE0101960E9487736E
:10105000CE0101960E94D158CE0107960E94D15828
:101060008091491290914A12029709F561EA7AE05B
:10107000CE0107960E94155967E574E1CE010796E7
:101080000E942258BC01CE0101960E940D5948ECE5
:1010900050E06FEF7FEFCE0101960E948773CE0183
:1010A00001960E94D158CE0107960E94D15866EA57
:1010B0007AE0CE0107960E94155961E574E1CE01F0
:1010C00007960E942258BC01CE0101960E940D593C
:1010D00040ED57E06FEF7FEFCE01019664D9CE016E
:1010E00001960E94D158CE0107960E94D158809156
:1010F000491290914A120197E9F5CE0107960E9494
:101100009D478B859C85009789F1EF81F88520812B
:10111000222361F1079750F16DE270E1CE01019653
:101120000E94055948EC50E06FEF7FEFCE01019629
:101130000E942C74CE0101960E94D158BE01695FB5
:101140007F4FCE0101960E940D5948EC50E06FEFA1
:101150007FEFCE01019627D9CE0101960E94D1588A
:1011600060ED77E080E090E00E944793CE01079623
:101170000E94D15864E670E080E090E00E944793BE
:10118000309201111092041157C261E270E1CE0158
:1011900001960E94055948EC50E06FEF7FEFCE01B9
:1011A00001960E942C74CE0101960E94D1580E9493
:1011B0007F934B015C010E947F93A70196010E94DF
:1011C000D4A7CA01B90120E831E541E050E00E940E
:1011D000D4A720E13EE040E050E00E94A8A72DA364
:1011E0003EA34FA358A72CE330E040E050E00E941C
:1011F000A8A729013A01AB01BC01CE0101960E94CA
:10120000527DB301A201CE0107960E94527D4DA1ED
:101210005EA16FA178A5CE010D960E94527DC501F9
:10122000B40120E03CE546E255E00E94D4A7BA01B3
:10123000A901CE0149960E94527DBE01675E7F4F93
:10124000CE0143960E940D596AE07DE0CE0143969F
:101250000E940B58BE01635F7F4F0E9422586DE0D1
:101260007DE00E940B58BE01695F7F4F0E942258AB
:101270006AED7BE00E940B58BE016F5F7F4F0E94BA
:1012800022586FEC79E00E940B58BC01CE014F96BA
:101290000E940D59CE0143960E94D158CE01499625
:1012A0000E94D158CE010D960E94D158CE010796CA
:1012B0000E94D158CE0101960E94D15840ED57E0CE
:1012C0006FEF7FEFCE014F966ED8CE014F96B2C131
:1012D0008091510D9091520D019719F462E170E1E6
:1012E00002C064E070E1CE0101960E94055948EC0D
:1012F00050E06FEF7FEFCE0101960E942C74CE017B
:1013000001960E94D15864EF7FE0E3C064EE7FE075
:10131000CE0101960E94055948EC50E06FEF7FEF37
:10132000CE0101960E942C74CE0101960E94D158E4
:1013300067ED7FE0CEC06AEC7FE0CE0101960E94AF
:10134000055948EC50E06FEF7FEFCE0101960E9407
:101350002C74CE0101960E94D1586FEB7FE0B9C08A
:1013600063EB7FE0CE0101960E94055948EC50E006
:101370006FEF7FEFCE0101960E942C74CE01019693
:101380000E94D15862EA7FE0A4C08091510D9091F3
:10139000520D039719F467E97FE002C06DE87FE022
:1013A000CE0101960E94055948EC50E06FEF7FEFA7
:1013B000CE0101960E942C74CE0101960E94D15854
:1013C00062E87FE086C065E77FE0CE0101960E947B
:1013D000055948EC50E06FEF7FEFCE0101960E9477
:1013E0002C74CE0101960E94D15866E67FE071C050
:1013F0006BE57FE0CE0101960E94055948EC50E074
:101400006FEF7FEFCE0101960E942C74CE01019602
:101410000E94D1586EE47FE05CC08091510D9091A4
:10142000520D029719F46DE37FE002C06DE27FE098
:10143000CE0101960E94055948EC50E06FEF7FEF16
:10144000CE0101960E942C74CE0101960E94D158C3
:1014500060E27FE03EC064E17FE0CE0101960E9441
:10146000055948EC50E06FEF7FEFCE0101960E94E6
:101470002C74CE0101960E94D15864E07FE029C00F
:1014800069EF7EE0CE0101960E94055948EC50E0DC
:101490006FEF7FEFCE0101960E942C74CE01019672
:1014A0000E94D1586FEE7EE014C063EE7EE0CE0164
:1014B00001960E94055948EC50E06FEF7FEFCE0196
:1014C00001960E942C74CE0101960E94D15863EDC2
:1014D0007EE0CE0101960E94055940ED57E06FEF86
:1014E0007FEFCE0101960E94D381CE010196A2C06A
:1014F000B090021268EC7EE0CE010D960E94055974
:10150000B11044C08090031290900412A090051274
:10151000B090061220E030E048E452E4C501B40186
:101520000E9476A6782E771C7724771C832D871946
:10153000782EA501940160E070E080EA90E40E94BA
:10154000CCA8AB01BC01272DCE0101960E94D65834
:1015500066E77CE0CE0107960E941559BE016F5FD9
:101560007F4FCE0107960E9422586EE676E00E94D9
:101570000B58BC01CE010D960E944158CE01079632
:101580000E94D158CE0101960E94D158BE01635FDE
:101590007F4FCE0101960E940D5948EC50E06FEF4D
:1015A0007FEFCE0101960E942C74CE0101960E941D
:1015B000D1586DEB7EE0CE010D960E9447586091A8
:1015C000001270910112CE0101960E941B7260E11F
:1015D0007DE0CE0107960E941559BE016F5F7F4FD7
:1015E000CE0107960E94225869E876E00E940B58C7
:1015F000BC01CE010D960E944158CE0107960E9473
:10160000D158CE0101960E94D158BE01635F7F4F31
:10161000CE0101960E940D5940ED57E06FEF7FEF2C
:10162000CE0101960E94D381CE0101960E94D1582D
:10163000CE010D960E94D1580E943C52882319F089
:1016400010927C140CC00E948A5C80917C148823C8
:1016500031F00F5F1F4F0131110509F0A8CCA8969A
:101660000FB6F894DEBF0FBECDBFDF91CF911F91B3
:101670000F91FF90EF90DF90CF90BF90AF909F9031
:101680008F907F906F905F904F903F90089585ED81
:101690008093BC008091BC0084FDFCCF10925D0E55
:1016A000089540919D14262F30E0240F311D2132E2
:1016B0003105DCF420915D0E2430C9F4FC0180E09A
:1016C00090E0861758F430919D142191DC01A358C5
:1016D000BB4EA30FB11D2C930196F3CF80919D14A7
:1016E000680F60939D1480E0089581E0089582E082
:1016F0000895089508950895E091A90D8091A80D89
:10170000E81730F4F0E0E655F24F808190E008955C
:101710008FEF9FEF08959091A90D8091A80D9817D4
:1017200050F4E92FF0E0E655F24F208130E09F5F62
:101730009093A90D02C02FEF3FEFC901089580914A
:10174000A80D90E02091A90D821B91090895CF92D8
:10175000DF92EF92FF920F931F93CF93DF937C0161
:10176000CB018A0120915E0E222389F0EB016B01EF
:10177000C40ED51ECC15DD0561F06991D701ED9140
:10178000FC910190F081E02DC7011995F3CF642FF2
:1017900088DFC801DF91CF911F910F91FF90EF90EB
:1017A000DF90CF900895CF93DF931F92CDB7DEB730
:1017B000698320915E0E2223D1F02091800E203289
:1017C00040F021E030E0FC013383228380E090E0B0
:1017D00014C080915F0EE82FF0E0E05AF14F99813C
:1017E00090838F5F80935F0E8093800E04C061E0D2
:1017F000CE01019656DF81E090E00F90DF91CF910E
:10180000089580E090E00895FC0190810180F281CC
:10181000E02DF8948181892B81832281892F809505
:1018200028232283A7E0B0E01197F1F721818223DA
:101830008183A3E2B0E01197F1F780817894EFEC17
:10184000F0E03197F1F7982381E009F480E0089502
:10185000FC0190810180F281E02D892F809560FF4D
:1018600012C0F8942281822382838181892B818313
:10187000A3E2B0E01197F1F78281982B92837894DC
:1018800087ED90E011C0F8942281822382838181C8
:10189000892B8183AFEFB0E01197F1F78281982B0C
:1018A000928378948FE090E00197F1F70895DC013E
:1018B0002C911196ED91FC911297F8948181922FC1
:1018C00090958923818378948DE743E050E081509F
:1018D00021F1DA011197F1F730813223C1F3F89445
:1018E0008281892382838181822B81837894ABE7F3
:1018F000B7E01197F1F7F89481819823918383E100
:1019000091E00197F1F78081282381E009F080E0E0
:101910007894E3E6F6E03197F1F708951F93CF93BB
:10192000DF93EC01162F60E0812F2BD6612F70E042
:10193000FB01E653FF4EE491E883FB01EC57FF4EB9
:10194000E491F0E0EE0FFF1FE659FF4E8591949170
:101950009A8389831B861D861C86FE013B962396EF
:101960001292EC17FD07E1F7DF91CF911F910895D7
:101970001F93CF93DF93EC01162F8C810E940C7D77
:101980006B85812F862B90E00E94077DDF91CF91A0
:101990001F910C94057D0F931F93CF938C01C62F3D
:1019A000E7DF6C2F6460C801E3DF6C2F6B7FC80139
:1019B000DFDF83EC90E00197F1F7CF911F910F915A
:1019C00008950F931F93CF938C01C62F607F6160A2
:1019D000E2DF80E1C89FB00111246160C801DBDF54
:1019E00081E090E0CF911F910F9108951F920F9287
:1019F0000FB60F9211240BB60F922F933F934F9374
:101A00005F936F937F938F939F93AF93BF93EF9366
:101A1000FF93809102115FD520910511309106113D
:101A20002F5F3F4F309306112093051190910411C1
:101A3000953618F096E09093011190910111943031
:101A4000C9F128F4923069F09330D1F05EC095303E
:101A500009F451C0963009F058C091E09093D1112B
:101A600051C0811152C020910511309106112436C8
:101A7000310508F442C01092D111109204111CC01B
:101A8000813009F042C0E091041191E09E0F9093E3
:101A90000411F0E02091051130910611EE0FFF1FA7
:101AA000E95FFE4E318320831092061110920511DA
:101AB00094E029C0811117C0E091041191E09E0FBC
:101AC00090930411F0E02091051130910611EE0F72
:101AD000FF1FE95FFE4E31832083109206111092A2
:101AE000051193E010C020910511309106112536A3
:101AF000310558F007C0811108C0109206111092EC
:101B0000051103C095E09093011190910311992361
:101B100029F0811102C02F9A01C02F98FF91EF91F7
:101B2000BF91AF919F918F917F916F915F914F91F5
:101B30003F912F910F900BBE0F900FBE0F901F90F3
:101B40001895CF92DF92EF92FF92CF93DF93EC0143
:101B5000072E000C880B990B0E947CA66B017C0160
:101B600020E030E040E45FE30E94DBA620E030E0CC
:101B700048E452E40E94CCA80E9465A9C617D70782
:101B8000D4F020E030E040EA5FE3C701B6010E94F4
:101B9000DBA620E030E048E452E40E94CCA820E03C
:101BA00030E040E85FE30E9406A80E9465A921E0BA
:101BB0006C177D070CF420E0822F90E0DF91CF912D
:101BC000FF90EF90DF90CF9008950F931F93CF93E6
:101BD000DF93082F64E37AE088E590E10E944C5A95
:101BE000C7E0D0E010E0B8010C2E02C075956795F3
:101BF0000A94E2F76170772742E050E088E590E1CF
:101C00000E94025A219778F7DF91CF911F910F918F
